:020000040800F2
:1000000000A00020D514010875C5000809050108E5
:1000100073C5000871C500086FC500080000000026
:100020000000000000000000000000006DC5000896
:100030006BC500080000000069C5000817EA000849
:100040003D1501083D1501083D1501083D15010844
:100050003D1501083D1501083D1501083D15010834
:100060003D1501083D1501083D1501083D15010824
:100070003D1501084D55000827B500083D1501083C
:100080003D1501083D1501083D1501083D15010804
:10009000D5C500083D1501083D1501083D150108AD
:1000A000A1E00008CDE0000891E00008DDE00008D4
:1000B000C1E00008B1E000083D1501083D15010848
:1000C0003D1501083D1501083D1501083D150108C4
:1000D0003D15010899E200088DE2000881E2000860
:1000E00025EA00083D150108ADFE00083D15010890
:1000F0003D1501083D1501083D1501083D15010894
:100100000000000000000000000000003D15010894
:100110003D1501083D1501083D1501083D15010873
:100120003D1501083D1501083D1501083D15010863
:100130003D1501083D150108000000000000000009
:100140003D1501083D1501083D150108000000009E
:10015000000000000000000000000000000000009F
:1001600000000000000000003D1501083D150108D9
:100170003D15010800000000000000000000000024
:08018000000000003D1501081C
:100188002DE9F04F2DED068B6F4E704B3360AFB0FD
:10019800002373600DF019F918B90DF039F909F059
:1001A800CBF909F087FA6A4B6A4C1A7842F00102D7
:1001B8001A70694A4FF47001C2F888100022099237
:1001C8000A92226842F4803222600493236803F47E
:1001D80000330A93099B013309930A9B1BB9099BB6
:1001E800B3F5A04FF2D1236813F4003318BF0123ED
:1001F8000A930A9B012B7DD0DFF85C81574BC8F826
:100208000C30636AB360636ADFF884B1DFF8849105
:10021800DFF884A143F080736362636943F4FC03ED
:100228002EAD636103238DF86A3041F6FF7325F81C
:10023800503D4FF09040294605F07AFA4FF6FF738B
:1002480058462946ADF8683005F072FA4448294600
:1002580005F06EFA4348294605F06AFA42482946ED
:1002680005F066FA2946414805F062FA284606F084
:10027800D7FD1A9B3E4AB3FBF2F33E4A13603E4B4E
:100288003E4A00271F605F603D4B5A60F02288F8A5
:1002980023200722DFF804819F601A60D8F808300D
:1002A800CAF8003099E80300636985E8030043F45D
:1002B800802363612023CBF818301BA91A9805F016
:1002C80037FA64200EF094FB3946C8222D4813F003
:1002D800F4F9E3692C4A43F00303E361A36943F4A7
:1002E800A123A361636943F4C023636102F1900C05
:1002F800574655E0254B12221A60636863606368AD
:100308006360636843F480636360636823F47C1309
:100318006360636843F4E8136360236843F08073A1
:10032800236022680B4B9201FBD55A6822F0030226
:100338005A605A6842F002025A60636803F00C037C
:10034800082BFAD158E700BF58080020238E000870
:10035800C02A00200010024000ED00E00005FA0568
:1003680000080048000C004800100048001400482D
:1003780040420F00CC250020D02500203F19010065
:1003880010E000E01C260020B066010800200240B2
:1003980000040048F0460108842A0020801D00203F
:1003A800937B506892F80FE003F00701DB0800EB3D
:1003B80083038900186A4FF00F0A0EFA01FE0AFA41
:1003C80001F120EA01011962196A10324EEA0101AD
:1003D80062451962E4D10023DFF89CA20AF10C02FD
:1003E800002199540133092BF6D1FF23964A8AF844
:1003F80015308AF816308AF817308AF818308AF8D3
:100408001930924BDFF874B21360914A03930420B9
:1004180010705846302213F050F9142202218BF83C
:1004280000208BF8241001228A49039B8BF818209E
:1004380098F805B081F800B0A3F5EF71CAF81C1060
:1004480085493F68A3F58F730B60844B03EBCB039F
:100458005B78CAF82030BB0648BFCAF820200023C2
:100468007F4A40F2DC5122F813100133082BF7D1F0
:1004780013A800211C2213F020F9BBF10E0F03D0A2
:100488000BF0EF03082B02D101238DF85E30022018
:1004980005F0CEFF18B14088003018BF0120C7F31F
:1004A80040038DF85230C7F380138DF85530C7F3E9
:1004B80040338DF84C30C7F3C03300F001008DF89D
:1004C8004F3017F400638DF8510007D098F8843145
:1004D80003F1FF3EDEF1000343EB0E038DF85030CD
:1004E800C7F300438DF85630336AB8F844E1ADF8E5
:1004F80062E0003318BF01238DF85730C7F300536B
:100508008DF85830B8F84631ADF85C30B8F852314B
:10051800ADF85A30C7F380438DF8533098F854310A
:10052800181C07F00101C7F3C00218BF0120FF041F
:1005380048BF4C4F8DF85400B8F8500144BFB7F885
:100548004C71ADF86270B0F5FA7F8DF84D108DF8EA
:100558004E20ADF8600002D90BB9ADF8623098F8BA
:10056800D431414886F82430002386F8253043707A
:100578009DF85E30002B0CBF0023022301B902B1A5
:10058800013309EB83094FF0000AD9F808309A1EA5
:10059800103303920593039A32F8023F03924FF601
:1005A800FF72934200F08A819DF851004FEA132CA4
:1005B800DAB25FFA8CF378B12C4F2D4807EB0217AB
:1005C8007968814208D13889B0F5806F00F071816F
:1005D800B0F5006F00F06D819DF8560090B11001E4
:1005E800DFF888E00EEB00075EF800E0214886455A
:1005F80000F05F811E487968814203D1B87B0828E2
:1006080000F057819DF8520050B1184F07EB0217C0
:100618007868B0F1904F03D13889202800F04981DB
:100628009DF84F0050B1114F114807EB0217796838
:10063800814203D13889042800F03B81BCF1020FC4
:100648001ED19DF84C1020E0682500206E1F002068
:10065800500F0020C0020020602700209068010889
:10066800100F0020801D00207D080020B0660108C2
:100678000004004800440140580800206C25002070
:10068800BCF1010F04D19DF84D10002900F0118133
:100698009DF8571031B19DF85E1019B9911F0129C5
:1006A80098BF0423CC4F9DF858104FEA02194F44C5
:1006B80031B19DF85E1019B9043A032A40F2E2807C
:1006C800012B43D1FF2386F86C3086F86D30C24B7E
:1006D800F76703EB09024FF00008517B50688DF86B
:1006E8006A1002F1080B1289ADF868201AA90222D3
:1006F80086F8708006938DF86B2086F82880C6F8F7
:100708002C80C6F83080C6F83480C6F8688086F831
:100718006E8086F86F8005F00BF8069B9BF8021038
:1007280053F80900424604F057FE38460DF07AFEA9
:10073800AA4BAB49C6F88030AA4BC6F88430C6F835
:10074800888038460A1D0DF03DFDB2E0022B46D1E7
:100758005FFA8AF21C2101FB02FC06EB0C089E4A98
:1007680088F871A0012188F8701002EB09014FF098
:10077800000B91F80DE0486888F872B001F10802A2
:100788000989ADF8681088F87AB01AA9C8F87C7099
:10079800CDF81CC08DF86AE006928DF86B3004F035
:1007A800C7FF8D4B069A53F8090091785A4604F012
:1007B80013FE38460DF036FEDDF81CC088498A4A1B
:1007C800C8F880206144894AC8F88420C8F888B0ED
:1007D80038460A1D0DF0F6FC0AF1010A69E0032B00
:1007E8004ED19DF85330DFF83C82DFF83C9203B3DA
:1007F8009DF8543098F826C0DFF800B2CDF818C03C
:1008080053B17B4BBDF86020B3FBF2F238460821A8
:1008180092B2BDF8623003E0384608214FF6FF7205
:1008280004F0AFFFDDF818C049F82C00C0F80CB090
:1008380020E0BDF8602098F826B0BDF86230B2F527
:10084800FA7F0BD96A49B1FBF2F23846082192B215
:1008580004F097FF674B49F82B000AE06649B1FBA3
:10086800F2F23846012192B204F08BFF634B49F84B
:100878002B00C36098F82630013388F8263018E03A
:10088800042B16D196F82580BDF85A205A4B93FBB5
:10089800F2F23846BDF85C30012192B204F071FFE3
:1008A80096F8253006EB88080133C8F8500186F819
:1008B8002530039B059A93427FF46DAE96F8252068
:1008C80086F870214E4A4F4B92F800E0AEF11702BD
:1008D8000027022A1F709C461AD8F3693B44D3EDBF
:1008E800007AF5EE407AF1EE10FA02D1336A73BB62
:1008F80026E0454A07EB02080FCB88E80F009CF872
:10090800003010370133C02F8CF80030E5D1EDE707
:100918003E4B13F83E908CF8009003EBCE03D3F8CF
:1009280004A0BAF1000FE1D04F45DFDA364A3B01A7
:1009380003EB020853440FCB013788E80F00F3E7B5
:10094800334B1A6812F4805F984624D11DE0314B6E
:10095800314A13F83E00107003EBCE035E68002E98
:10096800EED000238342EBDAC3EBC3017218DFF841
:10097800BC80D2F8009041F8089001EB08079188F4
:10098800B9809279BA710133ECE70EF0EF03082BC6
:10099800224B4DD14FE09CF80020012AF5D9204B7D
:1009A80003EB0212103210339342EED053ED047A67
:1009B800B6EE007A67EE877A43ED047A53ED057A4E
:1009C80067EE877A43ED057A53ED037A67EE877A07
:1009D80043ED037AE7E700BFB066010899510008C4
:1009E800D808002079520008DD5400087151000829
:1009F80000127A009952000840420F0089520008FC
:100A0800C002002018260020FC0100209068010880
:100A1800842A00209C500108EC260020EC1A0020B3
:100A28000402002058080020E8250020ED260020B8
:100A3800BEF10E0F09D11A7842F010021A70BEF1F9
:100A4800180F09D10EF054FA06E01A7822F01002B5
:100A58001A70BEF1190FF4E70EF02EFAD8F800302C
:100A6800B84E58035EBFB84B01221A70049B049A13
:100A78001B7843F00403137063694FF0010B4FF0C8
:100A8800020943F400332946ADF868B08DF86AB01E
:100A98008DF86B904FF09040636104F049FEAB4BCA
:100AA800AB4A1A6000200DF0C5FFE36943F48043A8
:100AB800E361236943F480432361636943F480233A
:100AC8006361736A23F470037362736A43F4A00367
:100AD8007362736A23F070637362736A43F0A0638E
:100AE8007362736A23F070437362736A43F0A043BE
:100AF8007362736A23F470237362736A43F4A023E6
:100B0800002773624FF0030A4FF4604330462946CA
:100B18001A938DF86C908DF86DA08DF86E708DF825
:100B28006F7006F0EBFA4FF48052304629461A925D
:100B380003928DF86CB08DF86DA08DF86E708DF8FD
:100B48006F7006F0DBFA23698249039A43F4804305
:100B58002361236923F4804323618B8823F4805322
:100B68001B041B0C8B808B889BB243F480538B80B7
:100B78000B8803F4415343F4457343EA0A030B809B
:100B88008B8823F470631B041B0C43F4E0638B8095
:100B98008B8B23F400631B041B0C8B8307230B82B2
:100BA8000B889BB243F040030B806B4BB2616B4EDA
:100BB8001E60636943F400336361E36943F48003AF
:100BC800E361236B23F020032363236B43F08053FB
:100BD80043F0200323634FF0904318465A6A22F0EB
:100BE800F0025A625A6A42F040025A625A6A22F481
:100BF80070625A625A6A42F480625A6229464FF415
:100C080000721A9203938DF86E708DF86F708DF8DC
:100C18006C908DF86DA006F071FA039B04934FF465
:100C28008062184629461A9206F068FA326822F05D
:100C38000102326031684A4A0A403260494A3261E8
:100C4800326842EA0B023260B760F760B760B26898
:100C580042F40042B26032683260726822F0784230
:100C680022F400427260326842EA0B023260D8F81D
:100C780000503D4E05F40043102230463946039398
:100C880012F01BFD4FF6FF7215EA09050E928DF85A
:100C98003D908DF83E708DF83F708DF83CA0049B18
:100CA8000ED02EA92022184641F8802D06F026FAEB
:100CB800072386F800907770F37086F802B05D46D7
:100CC800039B7BB12EA9042341F8803D1D4806F003
:100CD80015FA0C2333710723F371012375711D4431
:100CE800B371EDB2E36A214823F4F873E362E36A6F
:100CF80043F4D873E362636943F0805343F002031B
:100D0800636105F0C2FF1AA805F094FF184B1A9307
:100D1800184B1B93022D4FF0000314BF1A46802274
:100D28001F924FF48072114C20924FF480622192EE
:100D38002022204622921AA94FF400521C931E9397
:100D48001AE000BF0004004828070020CC2A002031
:100D580075E8000800380040D40E00200058004014
:100D6800FFE0CF00300E5000E411002008040240DC
:100D780040010050F411002023922493ADF87450E0
:100D880005F065FF236843F001032360C24CA368A4
:100D980023F04053A360A36843F08053A3600A2064
:100DA8000DF026FEA36823F08043A360A368A36028
:100DB800A36843F00043A360A368B74A002BFBDB9A
:100DC8009368B64923F040539360936843F0005307
:100DD80093608868B24B034043F468338B60D168F2
:100DE800B04B0B4043F40053D360136B013D23F029
:100DF8000F0C45EA0C05156300240123321991787C
:100E080000296BD05D1C042B375DD078DFF888E2B1
:100E1800EDB20ED803EB43035A00DEF830101F235F
:100E2800934021EA030107FA02F30B43CEF830306E
:100E380031E0092B0ED8053B06225A43DEF8341060
:100E48001F23934021EA030107FA02F30B43CEF86C
:100E5800343020E00E2B4FF006010ED8A3F10A0221
:100E68004A43DEF838C01F2393402CEA030107FAEF
:100E780002F30B43CEF838300DE00F3B01FB03F2D1
:100E8800DEF83CC01F2393402CEA030107FA02F363
:100E98000B43CEF83C30092F7F4A0FD99369A7F14D
:100EA8000A0303EB430397690721994027EA0101E5
:100EB800916191699840084390610EE053697B1EE7
:100EC80003EB430357693821994027EA010151612F
:100ED800516903339840084350612B460434102C61
:100EE8008CD16D4B9A6842F001029A601A461168DB
:100EF800694BC907FBD5DA686B4D22F00202DA604C
:100F0800DA6842F00202DA60DA6842F00102DA6076
:100F18009A6842F004029A60B5F85831002B40F004
:100F2800A886B5F95A21002A40F0A386B5F95C21B4
:100F3800002A40F09E86D8F800305C4C13F4003F3D
:100F48001FD0C8200DF054FDAE200DF01DF808B1DB
:100F58000CF098F9564E84F87101C8200DF048FD40
:100F6800544BC4F8743100210C22304612F0A5FB12
:100F78000223F37007F05FFA0DF01EFD4E4B034499
:100F8800B3604E4EDFF824A133684D48B3F8629041
:100F980095F85F7100210C2212F08FFB4FF0000BC7
:100FA80000211422474812F088FB59460C2284F885
:100FB80078B10AF5BE708AF879B112F07EFB424B1F
:100FC800C4F8883123200DF013FD752001210BAAE8
:100FD8000CF02CFF002800F082803C4BCAF88031CE
:100FE8003B4BCAF884315846432301210CAA8AF89E
:100FF8007C310CF01BFF9DF8303003F07E038DF838
:10100800303040B1682B06D101238AF878311D238E
:101018008AF87C3163E09DF82C3003F07E03682B5E
:101028008DF82C3056D10223062084F878310146F9
:10103800D4F880311AAA98479DF86D1001F0010282
:101048009DF86B1001F001014B0043EA82019DF805
:10105800692002F001030B430AD05BB2012B01D1D6
:10106800002302E0022B0FD1012384F8793136E006
:101078000E4B0C20D3F8803101210EAA98479DF819
:10108800383013F00F0303D103200DF035FD26E0AF
:10109800042BE9D1E4E700BF000100500003005031
:1010A800E010FCFF07C0FFFD801D0020580800204D
:1010B800440E0020081F0020404B4C00200F002049
:1010C80090270020F41900200847010835DE0008A1
:1010D80029DE0008702B04BF042384F87831484BBC
:1010E80000221A7094F87821022A9A4617D1454BA3
:1010F800454919604548464959604649D9600270D2
:101108004549464A196103218AF80010116841F0DF
:10111800010EC2F800E09346BE461F4603E00120D8
:101128000DF0EAFC8DE072460A2A28BF002201234E
:10113800934040F2B23E03EA0E0EBEF1000F16D104
:1011480013F04D0F13D0364B364A1A60364A5A60A0
:1011580094F87921002A0CBF6F226E221A72032399
:10116800324A437019431370CBF8001006E0012A85
:101178004FF0000ED7D82D4B83F800E0DBF8003095
:101188009B0702D5264B1B689847294B00224FF432
:101198007A7184F88C211960BC203B6803929847C7
:1011A800244B039A1A7095F855210AB18AF8002041
:1011B80095F856210AB11D490A7095F8572102B1D0
:1011C8001A70DBF80030180738D50FFA89F964224D
:1011D80099FBF2F302FB139212B207EE902AB8EED3
:1011E800E77A07EE903ADFED146AF8EEE77AE7EE71
:1011F800267AB2EE047A67EE877AC4ED647A20E044
:10120800081A0020F419002081CE000804010020EB
:1012180065DD000849DD000890C1793DDC0E00203D
:101228009027002021CF0008ADDD0008E22A002029
:10123800480F0020DF2A00208988883C0023C4F852
:101248009031CA4A137843F002031370C84B202226
:101258009A610A27DFF81893B9F814309BB283F023
:101268002003A9F8143019200DF0C2FB01200DF05D
:10127800E1FB19200DF0BCFB013F00200DF0DAFB6B
:1012880017F0FF07E6D12023C9F81830B94B9FEDB6
:10129800BA8AD3F80090DFEDB98A99F80C3000EEDD
:1012A800103AB8EEC00A20EE080A08F0E3F8B44B8A
:1012B80083ED000AB34B1B8807EE903AF8EEE77A05
:1012C800B7EE007AC7EE277AAF4BB0EE680AC3EDE7
:1012D800007AAE4BD3ED047AAD4B67EE887AC3ED56
:1012E800007A99F8003007EE903AF8EEE77AA94BC1
:1012F800C7EE277AC3ED007A77EE677AA64BC3ED7F
:10130800007AA64B83ED027AC3ED008AC3ED018A09
:10131800A34B83ED027AC3ED008AC3ED018A08F07E
:10132800A9F8B0EE408AB0EE680A08F043F820EE5B
:10133800006A68EE086A66EE007A9A4BE6EE887AEA
:10134800FF211B2220EE087AC3ED007A67EE007AAF
:10135800F0EE675AD7EE085AE7EE087A28EE468A82
:10136800C3ED015AA6EE808AC3ED027A83ED038AA3
:101378008D4B1F708D4B184612F09FF98C4ADFF881
:101388005CE212680770012112F0020F8EF800105B
:101398001FBF417003218EF80010022118BF817011
:1013A800510741BF9EF800104F1C8EF800700327AC
:1013B80048BF475412F00A0F73460ED09EF800201B
:1013C80004218154511CC9B205274754D11C02324B
:1013D800D2B28EF8001006218154D8F800108A067F
:1013E80041BF1A78571C1F70072748BF87546F7969
:1013F800082F01D00E2F08D11A7802F1010E83F8B8
:1014080000E04FF00B0E00F802E01A7811F4803F6C
:101418004FF00C0C00F802C002F1010E1CBFDFF8FF
:10142800BCC102325FFA8EFE83F800E01FBF8CF861
:1014380000205E4A4FF00E0C02F80EC04A0741BF6A
:101448001A7802F1010E83F800E04FF0100E48BF41
:1014580000F802E01A7802F1010E5FFA8EFE4FF0F2
:10146800120C11F4806F83F800E000F802C00ED06F
:1014780095F810C2BCF1000F09D0DFF860C1023244
:101488008CF80020494A4FF0130C02F80EC08A0568
:1014980041BF1A7802F1010E83F800E04FF0150EF3
:1014A80048BF00F802E0182F13D11A784FF0160E33
:1014B80000F802E002F1010E5FFA8EFE4FF0170C01
:1014C80000F80EC002F1030E0232D2B283F800E037
:1014D80087540F0341BF1A78571C1F70192748BF3C
:1014E8008754CA0541BF1A78511C19701A2148BF80
:1014F80081541A78511C197014238354002198229E
:101508002C4812F0DAF80DF07BF82B4B2B492C48BD
:1015180019602C4BB5F84E2101602B491A80002325
:101528002A4A37680B70B5F89611138093701FFA22
:1015380081FC07F18502264E26483668DFF8A0E0D0
:1015480020F813C006F596764EF823600133122B67
:10155800F1D1214ED6F800E01EF4805F08BFB5F83F
:101568009CC1A0F806C0D5373CE000BFC02A0020C7
:1015780000040048F01A002035FA8E3C00000000F4
:10158800E81A002008000020A01A0020F419002002
:10159800A41A0020041B0020F41A0020081B0020B5
:1015A800F81A0020D81A00205E1A0020E90E002040
:1015B800DC0E0020E81C0020340E0020081F00204C
:1015C800802A0020380E00206F0D0020942A002069
:1015D800902A0020C21C0020842A0020E80E002047
:1015E800B80D00201378F3B992F802C0D3789C455F
:1015F80019D2BCF1000F08D00CF1FF3C0CEB8C0C9D
:101608000CEB8C0C0CF5617306E0013303EB8303E0
:1016180003EB830303F5617392F801C00CF1040C2A
:101628009BB220F81C300432BA42DBD11EF0080FFE
:1016380000F0E08095F89031062B00F2D580DFE8C5
:1016480003F004070E35506E6E0045F2F05201E0CB
:1016580042F6F822424B1A800DF070F8C3E0404B76
:1016680042F6F8221A8009010A2391FBF3F10023BC
:10167800A1F5B0613B4A42F823100133122BF9D18E
:10168800394A3A4911603A4A4020137004F0ACFFD5
:10169800002800F0A98001234FF0070E90F9000000
:1016A800344A8DE808404021334B97E02C4B42F6F2
:1016B800F8221A802C4B314A1A602D4B10224020F8
:1016C8001A7004F091FF002800F08E800123002793
:1016D80090F900002A4A8DE8880040214FF4E13350
:1016E8007CE01F4B42F6F8221A801F4B254A1A60ED
:1016F8001F4B082240201A7004F076FF002873D090
:101708000123002590F900001F4A8DE82800402198
:101718004FF4E13304F08CFDC4F8940160E0104A02
:10172800DFF87480DFF874C0DFF874E0174F184DE5
:10173800184842F6F82111800D490C22062B0A7030
:1017480030D0002388F800308CF800308EF8003054
:101758001B233B7005232A7003704FF4E1352DE0FD
:10176800BA010020AC290020A4000020B50201081D
:1017780060250020C9030108A08601006D680008E3
:101788001D03010855680008A169000872110020AE
:10179800F310002073110020F410002071110020B4
:1017A80070110020002188F800108CF800108EF8C5
:1017B80000102A702121C34D39700370C24BC34AEF
:1017C8001A60402004F010FF70B101210023C04AC4
:1017D80090F900008DE80A0040212B4604F028FD0E
:1017E800003018BF012028B9082007F06BFEB64B5F
:1017F800B84A1A603268B84B12F4804F1FBF1221E2
:101808001970B149B54818BF086042F2010111408A
:1018180002F0010002F4005579B1B14944F620679D
:101828000F8025B108211970A749AE4D0D6020B170
:101838000C211970A449AC4808601978AB4F0439D9
:101848005970AB49AB4B0B60AB498033002512F4A0
:10185800803F0B603D700DF1680800F0AE8007F026
:10186800EFF8DFF8CCC2DFF8CCA2CDF814C040F214
:101878002A334FF001091A4660462946049387F82F
:10188800009011F01AFFDAF814209C489C4F42F49B
:101898008022CAF81420426A22F00F024262426A89
:1018A800032142EA090242624FF4807B02228DF84A
:1018B80035100CA98DF8342003928DF83650CDF8E8
:1018C80030B08DF8379005F019FCDAF81810039A43
:1018D80041F40031CAF81810398821F4407109041C
:1018E800090C39801D21F96238463A850EA93D86D2
:1018F8006022C7F814900E92ADF83E501095ADF8DE
:101908004450ADF84650ADF84850ADF84A50ADF8DF
:101918003C9005F047FABA6942F00802BA617A6C5D
:1019280042F400427A64DAF8142042EA0902CAF85A
:101938001420AAF57D6A504605F0A7F9404605F03F
:1019480079F9049B6F4AADF8743080231A92DDF858
:1019580014C01F9310224FF400535046414623935E
:10196800CDF86CC01C921E95CDF880B021952295BB
:10197800249505F06CF9FB6843F40073FB60DAF812
:10198800003043F00203CAF800300BA80D238DF88D
:101998002C308DF82D908DF82E508DF82F900CF05E
:1019A80023FD594B1A68594B43F825200135202D42
:1019B800F7D103F0DFFD03F0DDFD33685A0542D5AA
:1019C800534BD4F8C4741F60042004F00DFE0421A6
:1019D800C4F8C80404F0E2FD4E4B84F8CC04082097
:1019E8001F6004F001FE4C4B4C4D1860082104F0B8
:1019F800D5FD2C22002184F8CD04284611F05DFE87
:101A08007C232B708E236B70E023EB7010207D23DA
:101A180085F82B30C4F8D07404F0E6FD1021C4F822
:101A2800D40404F0BBFD84F8D8042020C4F8DC7486
:101A380004F0DAFD2021C4F8E00404F0AFFD84F8D6
:101A4800E40406F0CFFB364A138823F040031B0456
:101A58001B0C1380138823F038031B041B0C138002
:101A680013889BB243F04003138000259F23322044
:101A78008DF838308DF839508DF83A508DF83B5044
:101A88000CF0B6FF8DF869501C4D4FF480570422B6
:101A98002F8540460EA90CF071FCAF619DF86A30A5
:101AA8009DF869201B0243EA02429DF86B301343FC
:101AB8001C4A93421C4A53D044D81C498B4248D0F4
:101AC8003AE000BF90D00300A4000020716700082E
:101AD800816800081903010860250020E90201084F
:101AE800BA01002009030108F9020108B307002020
:101AF800C8120020A01F0020C412002000040048C3
:101B0800004401403444014020470108B407002044
:101B180034070020700700208C07002040070020B1
:101B28000038004018BA20000C00002015202000C2
:101B3800F00900200010024001F51A4102318B42E1
:101B480009D01BE082498B4205D001318B4207D076
:101B580014E0202300E0802313804FF4807302E018
:101B68004FF4807313805380938811881B0293600D
:101B78004B43D360012384F8E53404E00023138049
:101B880053809360D360D4680CB3E40A27464FF0BF
:101B98000009A14509DA09EB04056D10E802414680
:101BA80010220BF049FB0F2806DC07F09DF8694B63
:101BB800FF02C3F8E8740AE0002358F82320013232
:101BC80053D10133042BF8D12F462C46E1E7336873
:101BD800614A13F4002318BF012313700CF0ECFEC4
:101BE8005E4B18605E4B5A79052A194602BF5D4B59
:101BF8004FF4C8721A805C4B4FF47A721A805B4AB1
:101C0800137843F008031370594A137823F002033A
:101C18001370326840F6020313406BB1554B5648B7
:101C28001860564B03201870554B01201870554802
:101C38000023038054480380930341BF534B03227E
:101C48001A71DA7844BF42F00102DA708B683360A7
:101C58004F4B01221A704F4A137863F07F031370B9
:101C68002FB0BDEC068BBDE8F08F05F101092546C4
:101C7800ABE71BB208EE103AB5F95A31DFED467AF8
:101C8800464A09EE103AB5F95C31B8EEC88A08EE52
:101C9800903A28EE278AB8EEC99AF8EEE88A002129
:101CA800B0EE480A29EE279A68EEA78A117007F065
:101CB800E1FBF0EE40AAB0EE480A07F07BFBB0EE7D
:101CC800408AB0EE490A07F0D5FBF0EE409AB0EE34
:101CD800490A07F06FFBB0EE40AAB0EE680A07F0B9
:101CE800C9FBB0EE409AB0EE680A07F063FB60EEFD
:101CF8002A6A68EE097AF0EE665AE7EE8A5A284BA5
:101D080029EE2A6A28EE007AC3ED035AF0EE465A05
:101D180029EEC00AE7EE4A5AE6EE8A7AA6EE4A7A31
:101D280029EE299A83ED010A28EE698A29EEAA0A82
:101D380083ED009A83ED02AAC3ED045A83ED058A68
:101D480083ED067AC3ED077A83ED080AFFF7F3B847
:101D58001740EF0058080020B62700208C0100200B
:101D6800801D0020721A0020DC2A0020EC1A0020B6
:101D7800E02A0020DC110020FA1E00208C27002019
:101D880008010020A80E0020AA0E0020440E002002
:101D980028070020C02A002035FA8E3C7000002059
:101DA800B81100202DE9F04FA249A34C0A6802F5AA
:101DB8009C432DED028B20332360A04B87B01E7807
:101DC8000091C6B19E4909688A4240F20581013EE8
:101DD8001E7001E1D9F800309A48072D98BF595D67
:101DE800994B88BF29461B689847032D0CD904EBEB
:101DF80045050136A880934BDFF870921A78F5B242
:101E0800AA421946E6D820E0D9F8002005F10E03C9
:101E180002EB83039988DA880028E8D04FF47A73B4
:101E2800401A5843531A90FBF3F040F6C90300F5E3
:101E38007A70984205DC40F2EE239842B8BF184603
:101E480001E040F6CA0080B2D1E7804B1B6842F23D
:101E5800010803EA08087E4BB8FA88F84FEA5818D0
:101E68001B68B8F1000F06D194F8292084F82820BF
:101E7800784A5078107094F828701FB1754A17780E
:101E880087F0010794F82BB091F800A00F220326E1
:101E9800BBFBF6F606EB460684F82A20C6EB0B06D3
:101EA800D9F80020DFF8CC91F6B20025554559DA6B
:101EB8004FEA450C1FB1684931F8150000E0384673
:101EC800918ADFF8B4E1814202D8D18A81421ED2D8
:101ED8005EF825005849834203D2604931F80C0066
:101EE80019E0E8B20292019303910EF091FA032DE2
:101EF800019B029A0FDC03994FF0010C91F82AE03C
:101F08000CFA05FC2EEA0C0E81F82AE003E003F532
:101F180096714EF82510B8F1000F1CD194F8BC103A
:101F280029F8160031B9BBF1020F14D94249012032
:101F380081F8BC00B9F80210B9F800000844B9F8F3
:101F480004100844464980B221F8150000B2032164
:101F580090FBF1F080B2414909F1060921F815001A
:101F68000135A3E794F82A2039493E4BA2F10F0E18
:101F7800DEF1000242EB0E0284F8D6206AB13A4A3A
:101F88001268570109D40A68D9689A60521AC82A8F
:101F98001DD9012283F8212019E02E4A0120507012
:101FA80010700A689968DA605B68521A9A4282BFB0
:101FB8002C4B002283F821200025554507DAE8B28A
:101FC8000EF026FA254B23F815000135F5E794F8AD
:101FD8002B30013384F82B301C4B1A6812F4805FC5
:101FE800984605D0204B1B68DE0701D40DF06FFD25
:101FF800009B19681D4B1F68BB7A002B3ED0013B24
:1020080016483A7B30F813301AB1C3F53B630833EE
:102018009BB21BB2A3F57A73B3F57A7FA8BF4FF4CE
:102028007A7323EAE37307EE903A9FED117AF8EE9C
:10203800E77A5CE0C42A0020440D00208C2A0020A6
:10204800882A002060250020A4000020842A00207F
:10205800902A002003000020480D0020C21C002008
:10206800020E0020942A0020E40E0020802A00207E
:1020780000007A44700D0020B80D0020D8F8002028
:10208800150440D5D4F8D800934E081A00283ADB36
:10209800924A01F59C402030C6F8D8005079904A01
:1020A80032F81050A8B2FD7A90FBF5F596F8DC00EE
:1020B800013000F00F0286F8DC20324482F8DD504F
:1020C8001A468848185C01330244102B92B2F8D1A2
:1020D80012B292FBF3F31BB2642BA8BF642323EA6A
:1020E800E37307EE903A9FED807AF8EEE77AC7EE51
:1020F800877A7E4A9FED7E7A67EE877AFCEEE77AEA
:1021080017EE903A1380D8F800307A4F13F4807F96
:1021180000F00981784BDFF8E491994205D999F8E4
:10212800022012B9012289F8022099F80220002A17
:1021380000F0F980714A3E7892F82150704A681E82
:10214800454211684541002DC1F38063C6F38006FE
:102158000093924614BF4FF0000B4FF0030B99F811
:102168002020052A00F2D980DFE802F0034D5275DD
:1021780084A1002E3AD0D4F8F000B4F8F4100CF092
:10218800D6FB012809D15F495F4A09681268C988E6
:10219800642000FB0122C9F81020009B6BB1594A4A
:1021A800126812794AB10EF063F8032289F82020E8
:1021B8004FF47A72C9F81C20D1E7002D40F0AD80A9
:1021C800514AD9F8101010684C4A88420AD901922D
:1021D8000EF04EF8019A032182F8201040F6B8312B
:1021E800D161BCE7012182F82010B8E7009B4FF4C9
:1021F800806013B107F056F901E007F043F90022B7
:10220800C9F8102089E0002D46D10EF031F8A6E774
:1022180025B1052289F82020012000E0284666B172
:10222800D4F8F020D189394A1180518091803549FC
:1022380009684988D1804FF0020B334A1168D9F8F0
:102248001420914201D8002E64D147F23052C9F8C7
:102258001C20032221E03A7842F002023A700DF085
:1022680036FC294AD9F81C1012680A44C9F8182003
:10227800042212E0244A9DB11168D9F8182091422D
:102288004BD9234A92781AB9DAF80020D10744D4F6
:102298003A7822F002023A70052289F820205EE797
:1022A8001268D9F81C100A44C9F8182035E01549F5
:1022B800154A09681268C988642000FB0122C9F818
:1022C80010204FF48060002289F8202089F803202C
:1022D80007F0D8F843E700BF440D0020E4110020C0
:1022E800F4110020210E00200000C842420F0020F7
:1022F80000C07F44E02A0020404B4C00942A002074
:10230800E40E0020A8290020902A0020C21C0020EA
:102318000300002000287FF422AFBBF1000F02D099
:1023280058460CF0A1FB8D4D05F5C470B5F84E115B
:102338000CF0FDFA834668B90DF08CFF884BC3F8A2
:1023480000B0C3F804B0C3F808B0864B00221A6086
:102358005A609A603B785A0736D5D8F80030DB06C1
:1023680032D5814B1B78DE062ED4804B9B7893B1F7
:1023780095F8E031BBF1000F15D17BB17C4B1A68A1
:10238800D4F8F8309B1A002B08DA0DF0A0FB794B33
:1023980083F8FCB018E0BBF1000F0DD110200CF051
:1023A80063FB01230EE03BB1714A12684FF47A7166
:1023B80001FB0323C4F8F83094F8FC3023B10CF087
:1023C8003FFB002384F8FC30002295F8DEA195F845
:1023D800DF11B5F898E1B5F89AC113466648009040
:1023E80030F912609B087645C4BF63F07F03DBB207
:1023F80001326645B8BF43F04003042AEED194F891
:10240800FD205C489A4205D190F8FE20F92A04D8AC
:10241800013200E0002280F8FE2084F8FD30534BA2
:10242800564E9A789946E2B93368D80708D5BBF171
:10243800000F16D13B78DA0713D50DF0C9F910E073
:102448003B785B070DD54B4B93F828304BB14C4B81
:10245800DB7833B911B10DF03AFB02E0BBF1000FA4
:10246800F9D094F8FE30434ADFF82CB1142B40F031
:10247800A58099F802301AF1000A18BF4FF0010A36
:102488006BB392F8FD305F2B11D13B7803F0040356
:1024980003F0FF0113B10DF01AFB08E00B200291C5
:1024A80001920CF0E1FA019A029982F8FE10BAF151
:1024B800000F14D094F8FD307D2B10D13B7803F039
:1024C800040303F0FF0213B10DF001FB07E00B203A
:1024D80001920CF0C9FA274B019A83F8FE203B7849
:1024E80003F0040303F0FF01002B67D194F8FD30DB
:1024F800204A572B0BD1234B4FF47A721A80224B68
:102508001B6813F0080359D1204A138056E0D8F805
:102518000000400716D55A2B14D11D4B187820B14E
:1025280019701C4B01221A7048E092F8FF3083F0B2
:10253800010382F8FF300BB10C2000E00D200CF0F5
:1025480093FA3BE05D2B00F034845B2B00F033847E
:102558005E2B23D1032000F02FBC00BF801D00207C
:10256800981900203C130020EC1A002003000020DA
:10257800902A0020440D0020C21C0020E40E0020F8
:10258800942A0020DC2A0020DC0E0020400F0020C6
:102598009D1A00209E1A0020200F0020562B01D1E2
:1025A80007F01AFA99F80230002B00F01A8494F810
:1025B800FD306F2B40F00F840DF00AF9D8F8003089
:1025C8005A0732D594F8FF30A3B13B785B0711D591
:1025D800009BB3F90620B5F898319A420ADD3368B2
:1025E80013F0010301BFAC4A32211180AB4A08BF86
:1025F80082F8FF303368D8030AD5A94B1A782AB96C
:10260800A84A127812B9A44A3221118001220BE09B
:10261800A44A13784BB13B7803F0040303F0FF019D
:102628001BB9A14B117001221A70DBF800A000231E
:1026380033600AF187090AF1D70B99F8002099F855
:10264800013019F8010C9A420BD249460CF038F9BE
:1026580038B119F8022C012303FA02F23368134344
:10266800336009F10409D945E7D1904B1B782BB1A8
:102678008F4E3368990700F13D8334E30AF1D6069B
:102688000AF58F793278737816F8010C9A4225D2B8
:1026980031460CF015F908B3B37896F804C0854AAA
:1026A80096F803A07D480C21013B01FB0C4103EB8C
:1026B80043031344D1F810219A420FD0C1F81031C6
:1026C800002390F83C21C1F81431012303FA0CF3DC
:1026D80022EA030381F80CA180F83C3106364E4506
:1026E800D0D1754B1E68754B1B68029394F828303F
:1026F8000393734B009300230193009B1A68002AED
:1027080000F0E68292F800A0BAF1000F00F0E08233
:102718005B680299CB1A002B0CDB01F5FA73009960
:102728004B60019901238B4094F83C1121EA030383
:1027380084F83C31039B002B00F0CA82009B51783F
:1027480013F8043C0433DBB2002940F080825D4971
:1027580031F91310B5F8963103F1C800814202DD52
:1027680092F802B015E0C83B994203DA9178C1F1BA
:10277800000B0EE0019A0123934094F83C2122EAD1
:10278800030384F83C31029B009A03F5FA73536003
:102798009EE2019A94F83C311341DA0700F19882DD
:1027A800BBF1000FCCBF022001200CF08DF90AF11B
:1027B800FF33DFF8E890132B00F28282DFE813F092
:1027C8001400250037004B0064008A00ED0050011A
:1027D800B701E501150280024B005A008A00ED009E
:1027E8005001BF002201870196F80090D944B9F141
:1027F800FA0FA8BF4FF0FA0929EAE979304686F8B6
:1028080000900CF043F801200FE096F80190D944AD
:10281800B9F1640FA8BF4FF0640929EAE979304695
:1028280086F801900CF032F802204946DAE196F871
:1028380003A0DA44BAF1640FA8BF4FF0640A2AEA89
:10284800EA7A86F803A03046D9F8401103F0D4FE9E
:1028580003205146C6E1717959446429A8BF64210F
:1028680021EAE17171710D200CF092F8BAF10D0FA7
:1028780000F02682317959446429A8BF642121EAED
:10288800E17131710E20ADE1B179594481F308014C
:10289800B1710520A6E100BF841A0020440D002074
:1028A8009C1A00209D1A00209E1A0020E12A002070
:1028B800E40E0020504701084C0F0020902A002009
:1028C800540E0020C21C002000007A440000C842B8
:1028D80000000000D9F844311A78022A20D107EE06
:1028E80090BAB8EEE70A5FED077A93ED097A80EEC1
:1028F800270A30EE070AB5EEC00AF1EE10FA07D43F
:10290800B4EE670AF1EE10FAC8BFB0EE670A01E04C
:102918001FED110A83ED090A0F200CF023F80AE0D5
:1029280099785944C829A8BFC82121EAE17199704A
:102938000F200CF02DF8BAF10F0F00F0C181D9F873
:1029480044311A78022A1ED107EE90BAB8EEE78A07
:102958005FED227A93ED080A88EE278A38EE000A9E
:10296800B5EEC00AF1EE10FA07D4B4EE670AF1EE3C
:1029780010FAC8BFB0EE670A01E01FED2B0A83ED1D
:10298800080A122056E159785944C829A8BFC82115
:1029980021EAE1715970122024E1D9F844311A78FA
:1029A800022A20D107EE90BAB8EEE70A5FED397A2D
:1029B80093ED0C7A80EE270A30EE070AB5EEC00ACE
:1029C800F1EE10FA07D4B4EE670AF1EE10FAC8BFB8
:1029D800B0EE670A01E01FED420A83ED0C0A1020F1
:1029E8000BF0C0FF0AE0197B5944C829A8BFC821C9
:1029F80021EAE171197310200BF0CAFFBAF1100F28
:102A080000F05E81D9F844311A78022A1ED107EE07
:102A180090BAB8EEE78A5FED537A93ED0B0A88EE29
:102A2800278A38EE000AB5EEC00AF1EE10FA07D48C
:102A3800B4EE670AF1EE10FAC8BFB0EE670A01E01B
:102A48001FED5D0A83ED0B0A1320F3E0D97A594490
:102A5800C829A8BFC82121EAE171D9721320C1E0B1
:102A6800D9F844311A78022A22D107EE90BA1FED1C
:102A78006A0AF8EEE77A87EE800AD3ED0F7A30EE2D
:102A8800270AB5EEC00AF1EE10FA09D45FED717AA3
:102A9800B4EE670AF1EE10FAC8BFB0EE670A01E0BB
:102AA8001FED750A83ED0F0A11200BF05BFF0AE09A
:102AB800997D5944C829A8BFC82121EAE1719975AF
:102AC80011200BF065FFBAF1110F00F0F980D9F869
:102AD80044311A78022A20D107EE90BA1FED860AEF
:102AE800B8EEE78A88EE008A93ED0E0A38EE000AFF
:102AF800B5EEC00AF1EE10FA09D45FED8C7AB4EEA7
:102B0800670AF1EE10FAC8BFB0EE670A01E01FEDE0
:102B1800900A83ED0E0A14208CE0597D5944C82987
:102B2800A8BFC82121EAE171597514205AE0D9F8E3
:102B380044311A78022A1ED107EE90BAB8EEE78A15
:102B48005FED9E7A93ED0A0A88EE278A38EE000A2E
:102B5800B5EEC00AF1EE10FA07D4B4EE670AF1EE4A
:102B680010FAC8BFB0EE670A01E01FEDA70A83EDAF
:102B78000A0A09205EE0D9785944C829A8BFC821A3
:102B880021EAE171D97009202CE0D9F844311A788A
:102B9800022A1ED107EE90BAB8EEE78A5FEDB57A41
:102BA80093ED0D0A88EE278A38EE000AB5EEC00AC2
:102BB800F1EE10FA07D4B4EE670AF1EE10FAC8BFC6
:102BC800B0EE670A01E01FEDBE0A83ED0D0A0A2088
:102BD80030E0597B5944C829A8BFC82121EAE171CE
:102BE80059730A200BF0D4FE6AE0D9F844311A78F8
:102BF800022A22D107EE90BA1FEDCD0AB8EEE78A75
:102C080088EE008A93ED100A38EE000AB5EEC00A85
:102C1800F1EE10FA09D45FEDD37AB4EE670AF1EE5B
:102C280010FAC8BFB0EE670A01E01FEDD70A83EDBE
:102C3800100A0B200BF096FE42E0D97D5944C829B2
:102C4800A8BFC82121EAE171D9750B20CAE701297B
:102C580036D190788F4A32F91390B9F5617F05DB48
:102C680040F633039945A8BF994601E04FF46179CE
:102C7800BAF10C0F24D1884A4FF4966393FBF0F015
:102C88001378A9F5617999FBF0F95FFA89F94B4551
:102C980016D0B9F1040F34BF4B46022313707F4A94
:102CA8000AFB035303F2AA73136006F0DFFC5046D5
:102CB80049460BF06DFE09F10100C0B20BF004FFAC
:102CC800019A0123934094F83C21134384F83C3142
:102CD800019B01330193009B0C330093019B042B50
:102CE8007FF40BADC4E4D8F80030DB0511D56C4B8C
:102CF800DB7873B16B4B1B689C070AD56A4B1B8842
:102D080013F001040AD10DF0A5FA012006F0CAFB60
:102D180004E0012006F0B6FB012300E0002332683E
:102D280050070DD563B1012006F0ACFB5E4B1B8844
:102D3800990708D40DF08EFA022006F0B3FB02E0E2
:102D4800022006F09FFB33681A054FF4807002D505
:102D580006F0A8FB01E006F095FB6B79082B01D083
:102D68000E2B02D1402006F08DFBD8F800305B0511
:102D780040F18B8095F810321BB93B7813F0040FA3
:102D880002E0336813F4002F0AD0484B00221A706F
:102D98003C200BF019FD002877D00CF037FAF7E744
:102DA80005F020FA07B0BDEC028BBDE8F04F0BF040
:102DB80027BC012000E002205FFA80F909F1FF3307
:102DC80085F8A83706F0B8FB06F074FC48460BF007
:102DD8007BFEFFF7F3BBBAF1000F02D07E2B3FF466
:102DE800EBAB94F8FD30324A972B05D1314B4FF4B9
:102DF800C8721A80FFF7E2BBA72B06D12E4A1378B8
:102E080043F004031370FFF7D9BB0021BB2B0591D6
:102E180001D1022303E0B72B04D14FF6FE73ADF8BE
:102E2800163009E0BE2B01D1022303E0BD2B1AD1D5
:102E38004FF6FE73ADF81430DBF80030BDF814100F
:102E4800B3F864200A44A3F86420BDF81610B3F858
:102E580066200A44A3F8662006F0BEFD002384F825
:102E6800FE30FFF7ABBB792B04D192F8033123F086
:102E7800010306E07A2B7FF4A1AB92F8033143F00B
:102E8800010382F80331FFF799BB07B0BDEC028B51
:102E9800BDE8F08FC21C0020642700204C0F0020E2
:102EA800942A0020DC0E0020E00E0020652500207A
:102EB800440D0020721A0020EC1A00202DE9F04F72
:102EC800BB4BB3F90610BB4B2DED028B1F687A89FB
:102ED80091B0914201930EDBB1F5FA6FFC79BDBF59
:102EE8008B1A6343A2F5FA64C4F16404BCBF93FB74
:102EF800F4F4643400E06424AF4AB04BB2F896A10D
:102F080092F95E211868049092B205920546002253
:102F18000293A74B33F912300393CAEB030303F26E
:102F2800F31640F2E63086424FEA420B03D8002BF4
:102F3800B8BF5B4201E04FF4FA73022A00934FF0E6
:102F48006400049B9E4E31D093F81DE1BEF1000F42
:102F580006D0009B7345CCBFCEEB03030023009340
:102F6800009BDFF8A0E293FBF0FC6FF063093EF8EA
:102F78001C8009FB0C390CF1010C3EF91CE00FFA1E
:102F880088FCCCEB0E0E0EFB09FE9EFBF0FEC64441
:102F980026F80BE0BE18367973438A4E93FBF6F396
:102FA80064339BB2634393FBF0F031E093F81EE186
:102FB800BEF1000F06D0009B7345CCBFCEEB0303D8
:102FC80000230093009BDFF8288293FBF0F06FF05A
:102FD800630C38F910E00CFB00390130BDF81430EF
:102FE80038F91000CEEB000000FB09F999FBFCF959
:102FF800CEEB090919FB03F9009BA6F80490B879F0
:10300800002BB8BF5B4243436E4893FBF0F064303B
:103018006B786D4E4FF0640E434393FBFEF3B3544D
:103028006A4EEB7A434393FBFEF3B3546B7D644ED5
:103038005843674B90FBFEF0022A9854654B0FD11A
:1030480083F802E0039B53450EDB5B4CB4F89821F0
:10305800914215DBB1F5FA6FA8BF4FF4FA6110E0A1
:103068009C54039B534504DA36F80B305B4226F830
:103078000B300132032A05F101057FF44AAFE4E77A
:103088001146891A4FF47A73DFF87CE14C4D5943A5
:103098006FF06303C2F5FA626427B1FBF2F191FBAA
:1030A800F7F23EF8120003FB0211013203B23EF9B7
:1030B8001220D21A514391FBF7F30344F380464B95
:1030C8001B885B0635D5454B454A1B881288DFEDC2
:1030D800457A9B1A1BB208EE103AB8EEC88A28EE59
:1030E800278AB0EE480A06F0C5F9F0EE408AB0EE3D
:1030F800480A06F05FF9B5F9023006EE903AB5F9DC
:103108000030F8EEE66A07EE903A20EE667AF8EEBE
:10311800E77AA7EEA87A67EE807ABDEEC77AE6EE80
:10312800A87A17EE103AFDEEE77A2B8017EE903A60
:103138006B802D4D2B689F0740F1A1802B4B2C4FA6
:103148001A687B6945F20721D31A8B4240F39780AE
:103158007A6104F0E7F8274BDFF8B0901A78032A71
:103168009846B9F8003053D10A2B5BD900232820A0
:1031780088F800300BF03CFC04F0D4F81E4B18889B
:1031880004F0BAF81D4B1A68D37890FBF3F00130BD
:1031980008281B4BA8BF08201870537980B213FB6E
:1031A80000F33B83137913FB00F078833AE000BF08
:1031B800C21C00204C0F0020801D0020200F002082
:1031C800801900200CFEFFFF501300209E0E0020E7
:1031D8006413002088190020E00E0020400F002012
:1031E800B427002035FA8E3C842A0020C42A002007
:1031F800900E00208C270020FC110020DC110020FC
:1032080008010020BC2500209E1000208812002004
:103218000A2B07D80323A04A88F80030002313702C
:103228003B837B8398F800309C4A012B0CD002D357
:10323800022B1BD023E03A8BB9F800309A421EDDEE
:10324800012388F800300FE0B9F800107B8B8B421F
:1032580002DD022313700FE0914B1B8B013399425F
:1032680002DD002313700AE0082006E07B8BB9F822
:10327800002001339A42E3DC07200BF0F5FBD5F878
:1032880000B0884D1BF4006F78D0874B844F1B68C3
:10329800FA69C2EB030845F2072290456EDDFB612F
:1032A800824BB6F906C0D3F80090B4F84E1199F8DD
:1032B8000A307F4E012BACF57A7C03D045D3022B24
:1032C80020D044E07B4B396A5A7B7B4B33F8122081
:1032D800082092B291FBF0F3C91A8B18BA843B62AA
:1032E80040F6E44293FBF0F39BB25343B9F808204D
:1032F800C2EB13334FF47A725343B9F9062093FBA8
:10330800F2F323E02B78B9F808A0C6F800A0580714
:103318001DD56A48CDF800C00BF009FBDDF800C0E8
:1033280020B91BF0100F18BF4FF0000C32220CFB15
:103338000CF393FBF2F3B9F9062063445A434FF4B4
:103348007A7392FBF3F3534400E000233360D7E928
:103358000A01336803FB08F84FF47A7398FBF3F813
:1033680010EB080241EBE873C7E90A231046194637
:10337800534A00230DF0E6FA524B1860524F00975B
:103388003B6813F4805F02D00A200BF06DFB4F4EB0
:103398003268002A57D04E494E4B08681F6887424A
:1033A800894698464FD84C4BDFF838A118785168B1
:1033B80008BB01201870BAF80030CB5C5BB31378F7
:1033C800013B00FA03F2D4F8D4371A4201D10BF0CA
:1033D80031FB424B01221A700DF06CF8BAF800303C
:1033E800CBB933681B78053B012B14D80BF0E4FAF2
:1033F8003B4B18600FE04FF0000B83F800B0BAF8B1
:103408000030CB5C3BB158460BF014FB334B83F8D0
:1034180000B00DF04FF83268BAF800305268314801
:10342800D25CFE2A01D100230CE0FF2A02D10BF066
:1034380007FB08E0D9F800600A2111FB0262C8F80E
:103448000020013303802B78590703D5264B20220F
:103458001A8561E0009A1268D2075EBF114A43F0EC
:1034680001031370214B1B781F075EBF2B7823F0D5
:1034780001032B701E4B1A88184B1AB11D4A12688B
:10348800960702D41C4A1288C2B302221A702B78FB
:1034980023F001032B7036E0080100208C27002060
:1034A800900E0020E02A0020C42A0020DC11002011
:1034B800440F0020E4110020F4110020081F002010
:1034C800407E0500E0110020E40E0020E4250020E5
:1034D800902A0020DC250020D8250020B82A0020CA
:1034E8003C290020E025002000040048EC1A0020B8
:1034F800721A0020DC0E0020DC2A00202978C80778
:1035080058BF02221A700BF057FAB44B1B68C01A46
:10351800002801DB0CF0CEFFB14F04F063FE3E78CB
:10352800002E00F0AC80AF4B1A689846002A00F0D5
:10353800BD86D8F800000BF02DFB002800F0B686F9
:10354800A84BA94C18680BF022FB092801D03F288A
:1035580052D14FF0000A2668DFF8C892554636B1B6
:10356800A248D9F80010324610F0F4F810B9CA464B
:1035780005B94D469E4B09F110099945EFD3EDB1B8
:10358800D5F800C0DAF8009023681CF803E019F8B1
:103598000300704512D15A1C944958B92D2B09D8EB
:1035A800DFF844E2CEF800204FF0200E01F803E0E7
:1035B800885403E001F803E02260E5E723680BB1D3
:1035C800554510D08B480BF019FF554507D855F8CD
:1035D800100B0BF013FF09200BF008FFF5E78648E6
:1035E8000BF00CFF002623689E42A2D27F4B985D09
:1035F8000BF0FCFE0136F6E72368002B40F03C8612
:10360800042840F05E86794803F0E8FF00F04EBEDB
:10361800D9F80000DFF8ECA10BF0BCFA28B3DAF80F
:1036280000000BF0B4FADBF8003093F848100246BB
:10363800A9BB24286CD1012283F84820DBF800308C
:10364800DFF8E4A193F84820062AE1D193F849006D
:1036580000F0C2FE8346002800F083800BF022FEB3
:10366800D8F80030002283F84820644B93F83730AC
:10367800002B40F0EF854C36982E00F01786604BF3
:10368800F21892F84A100129F5D1DFF89C81F35815
:10369800C8F800205B4AC34613609146B8E7012981
:1036A80004D14D2814BF00220222C5E7022904D103
:1036B8003C2814BF00220322BEE703290CD140286E
:1036C8004FF0000102D983F84810B7E75871197113
:1036D800D97198710422AFE7042906D1997983F842
:1036E80049004A409A710522A6E70529A6D15879CA
:1036F80019798842987906D950409871481C1871F0
:103708000B441A729AE790420CBF0622002293E7F4
:103718002B783D495B0791D42328DAF8003013D180
:103728000090012038702F480391036033480363E9
:1037380036480BF063FE30480BF060FE0399009AA0
:103748000B7843F002030B70314B1B681B789342D4
:1037580001BF304B304A1A60304B04BF304ADA6040
:103768006CE7DAF8002092F849304A2B00F06D85B2
:1037780000F28580332B00F0718421D8292B00F0CA
:10378800F68309D8252B00F0CE83272B00F0D183B0
:10379800232B40F0928569E22D2B00F0F98307D89E
:1037A8002B2B40F08A850BF051FD607100F04DBD68
:1037B8002F2B00F0BF84312B00F0D18400F07DBDA9
:1037C8003E2B00F03D8146D8372B00F07A842DD867
:1037D800352B00F0868200F070BD00BFBC2A0020A7
:1037E800E12A002088270020C01200209012002023
:1037F800DC4F01084067010845670108900E00206A
:10380800E81C002084270020E02A002075670108B2
:1038180068250020FC9F0020EFBEADDE00ED00E033
:103828000400FA050C4E010880270020392B00F00F
:103838008D833C2B40F04185DFF81894D9F800A01F
:103848000BF004FD8AF80000D9F80030187808F069
:1038580043FE00F0FABC432B00F0118405D8412B3D
:1038680040F02B854FF00009FDE3442B00F0AC84B9
:10387800482B40F0228509F0B7FC00F0E6BCD02BBD
:1038880000F02F835FD8CA2B00F0E38016D84E2BA8
:1038980000F0B683C82B00F0A2804C2B40F00D85B9
:1038A8000BF0D4FC84F8D6010BF0D0FC84F8D701D7
:1038B8000BF0D6FCA4F8D80100F0C7BCCD2B00F063
:1038C8001B8304D8CC2B00F0348200F0F6BCCE2B3E
:1038D80000F01B83CF2B40F0F0840BF0C1FC6FF499
:1038E800AF6E00EB0E039BB2C62B98BFA4F89601EF
:1038F8000BF0B6FCA4F840010BF0B2FCA4F84201AE
:103908000BF0AEFCA4F844010BF0AAFCA4F8D80113
:103918000BF09CFC0BF09AFC0BF098FC0BF096FC5F
:1039280084F885010BF092FC84F892010BF08EFC70
:10393800C84BD3F800900BF093FC00EB80004000DC
:10394800A9F8620002E3D82B00F015810FD8D32B19
:103958003FD003D8D22B29D000F0AFBCD42B00F035
:103968004782D62B40F0A9844FF0000935E2F22BAC
:1039780000F08C8212D8EF2B40F09F84DFF8D492AD
:10398800D9F800A00BF06CFCAAF86600D9F80090F2
:103998000BF066FCA9F8640000F057BCF32B00F0AC
:1039A8001884FA2B00F0BB8200F087BC2B7803F058
:1039B800040303F0FF09002B40F047840BF046FC9A
:1039C800022884F8A80740F29282A34B83F8A897AC
:1039D8008DE20BF045FCA14B988600F036BC92F8BE
:1039E80005904FEA5909B9F1120F03D90AF0E8FE18
:1039F80000F02BBC4FF0000ACA4507D20BF030FC90
:103A080007AB23F81A000AF1010AF5E74A46002332
:103A18004B4507DA07A931F81300914921F813003B
:103A28000133F5E7122A05D08D4B002123F8121037
:103A38000132F7E7894B012283F8362000F005BCF4
:103A48000BF004FC84F8E0010BF000FC84F8DF01C3
:103A5800FBE3804B1A681278022A824699466FD196
:103A6800D9F800B00BF0F2FB07EE900AF8EE677A8F
:103A7800B2EE048AC7EE887A0BEB8A0BCBED087A94
:103A8800D9F800B00BF0E2FB07EE900A9FED757ACB
:103A9800F8EE677A0BEB8A0BC7EE877ACBED0B7AD9
:103AA800D9F800B00BF0D2FB07EE900A9FED6E7AC2
:103AB800F8EE677A0BEB8A0BC7EE877A0AF1010AF0
:103AC800BAF1030FCBED0E7ACAD1BAF1070FD9F8C4
:103AD80000B01CD10BF0BAFB07EE900AF8EE677A3B
:103AE800C7EE887ACBED117AD9F800B00BF0AEFBAF
:103AF80007EE900AF8EE677AC7EE887ACBED127A6D
:103B0800D9F800B00BF0A2FB8BF84C0012E00BF0D8
:103B18009DFBD3448BF80100D9F800B00BF096FB5D
:103B2800D3448BF80B00D9F800B00BF08FFBD344CB
:103B38008BF815000AF1010ABAF10A0FC5D184E31E
:103B4800D9F800B00BF082FBD3448BF80100D9F808
:103B580000B00BF07BFBD3448BF80B00D9F800B016
:103B68000BF074FBD3440AF1010ABAF10A0F8BF87F
:103B78001500E5D169E38246DFF8D8909FED3A8ACF
:103B8800D9F800B00BF06CFB07EE900AF8EE677AF4
:103B98000BEB8A0BC7EE887ACBED087AD9F800B020
:103BA8000BF05EFB07EE900AF8EE677A0BEB8A0BD8
:103BB800C7EE887ACBED0B7AD9F800B00BF050FB42
:103BC80007EE900AF8EE677A0BEB8A0BC7EE887A55
:103BD8000AF1010ABAF1030FCBED0E7ACCD1BAF192
:103BE800070FD9F800B01CD10BF03AFB07EE900A8A
:103BF800F8EE677AC7EE887ACBED117AD9F800B07B
:103C08000BF02EFB07EE900AF8EE677AC7EE887A7B
:103C1800CBED127AD9F800B00BF022FB8BF84C00F0
:103C280012E00BF01DFBD3448BF80100D9F800B06B
:103C38000BF016FBD3448BF80B00D9F800B00BF04F
:103C48000FFBD3448BF815000AF1010ABAF10A0FE9
:103C5800C5D1FAE2200F0020801D0020900E002020
:103C6800F42900200000C84200007A440BF0EEFA64
:103C7800132883463FF6BAAEDFF870A3DAF800904F
:103C88000BF0E4FA0023D44A0C2101FB0322117A39
:103C9800814222D10FFA8BFB09EB8B09137889F843
:103CA80085300BF0D3FA89F886000BF0CFFA89F843
:103CB80087000BF0CBFAC94BC94A1A6089F888000B
:103CC800C84BDAF800001860002185300AF01EFEA3
:103CD800C54B80F001001870B7E201331C2BD2D11C
:103CE80084E60BF0B3FA0B2882463FF67FAEBF4B53
:103CF800D3F800900BF0AAFA03283FF677AE062314
:103D080003FB0A9989F8DA000BF0A0FA89F8D500C4
:103D18000BF09CFA89F8D6000BF098FA89F8D700CE
:103D28000BF094FA89F8D8000BF090FA89F8D900CA
:103D38008BE25379092B7FF659AE019BD3F800909B
:103D48000BF084FA019B89F80000D3F800900BF07F
:103D58007DFA89F801000BF079FA019B64281B6849
:103D6800A8BF642018710BF071FA019B64281B68C6
:103D7800A8BF642058710BF069FA019BFF281B68E3
:103D8800A8BFFF2098710BF061FA019B6428D3F853
:103D9800009028BF642089F807000BF057FA019BB0
:103DA80089F80200D3F800900BF050FA019B89F8CB
:103DB8000300D3F800900BF053FAD8F80030A9F8B4
:103DC8000A005B790A2B40F24082894BD3F80090B5
:103DD8000BF03CFA89F8080037E20BF041FA854B02
:103DE80023F8190009F10109B9F1080FF5D12CE2FE
:103DF80053790F2B7FF4FAAD0BF028FA0728814688
:103E08003FF6F4AD029BD3F800A00BF029FA0E237D
:103E180003FB09F9CA44029BAAF82501D3F800A0BC
:103E28000BF01EFACA44029BAAF82701D3F800A097
:103E38000BF016FACA44029BAAF82901D3F800A08D
:103E48000BF004FACA44029B8AF82B01D3F800A0AD
:103E58000BF0FCF9CA44029B8AF82C01D3F800A0A5
:103E68000BF0F4F9CA44029B8AF82D01D3F800A09C
:103E78000BF0ECF9CA44029B8AF82E01D3F800A093
:103E88000BF0F8F9D144C9F82F01DEE10BF0DEF9A7
:103E98000F2881463FF6AAADC9EBC9090BF0D6F940
:103EA80004EB090303F1D00983F8D0000BF0CEF935
:103EB80089F801000BF0CAF989F802000BF0C6F97D
:103EC80089F803000BF0C2F989F804000BF0BEF979
:103ED80089F805000BF0BAF989F806000BF008F824
:103EE800B3E12B78580700F1B08109F091FA05F099
:103EF80023FB05F0DFFBA8E12B78590700F1A5812A
:103F08003D4B4FF4C8721A809FE12B785A0700F195
:103F18009C813A4A137843F00403137095E12B7897
:103F28005B07E4D5C9E1A0600BF0A4F905F0D2FA6B
:103F38008BE10BF095F9A4F858010BF091F9A4F86E
:103F48005A010BF08DF9A4F85C017EE10BF07EF9C3
:103F580084F87A010BF07AF984F87E010BF076F98F
:103F680084F87D010BF072F984F87F016DE10BF0A4
:103F780077F9A4F880010BF073F9A4F882010BF02B
:103F880065F984F884010BF06BF9A4F886015CE10B
:103F98000BF05CF984F890010BF062F9A4F89A012F
:103FA8000BF05EF9A4F896010BF05AF9A4F8980101
:103FB8000BF04CF9DAF8003084F891015B79082BA2
:103FC80040F243810BF04CF9A4F89C010BF048F93E
:103FD800A4F89E0139E100BFBC470108840E002007
:103FE800C01E0020880E002005000020200F0020A1
:103FF8004C0F002066270020721A0020EC1A0020BF
:1040080092F805900323B9FBF3F9B9F1120F3FF6C3
:10401800EDACDFF8C0A34FF0000BCB4580F0158165
:104028000BF014F98AF8A0010BF01AF940F2ED230D
:10403800984205DD40F6CA039842A8BF184601E039
:1040480040F2EE20A0F2EE2019230BF1010B90FBB9
:10405800F3F00AF1020A8AF89F01DEE70BF0F6F89E
:1040680084F89201F1E00BF0F1F804EB090309F18F
:104078000109B9F1080F83F88801F4D1E5E00BF0E4
:10408800E5F8C4F808B060710BF0F4F805F022FA0E
:104098000BF0DCF884F890010BF0E2F8A4F8580172
:1040A8000BF0DEF8A4F85A010BF0DAF8A4F85C017A
:1040B8000BF0D6F8A4F880010BF0D2F8A4F882012E
:1040C800C3E053794FF0070AB3FBFAF2C2EBC2021E
:1040D8009A1A12F0FF0F7FF489ACB3FBFAFA0AF1CF
:1040E800FF3A5FFA8AFABAF1FF0F00F0AE800BF0E0
:1040F800ADF85FFA80FB4FFA8BF002F099F9814630
:1041080000283FF473AC80F800B00BF0A9F8A9F8C8
:1041180002000BF09BF889F804000BF097F889F877
:1041280005000BF093F889F807000BF08FF889F871
:104138000600D4E7DFF89C9209F1400A0BF090F8EA
:10414800A9F8A0020BF082F889F8A2020BF07EF819
:1041580009F1040989F89F02D145EFD175E00BF008
:1041680075F81F2881463FF641ACD8F800305B79D6
:10417800082B7FF43BAC0BF073F809F1880904EBCA
:10418800890A00F03F00AAF802000BF069F8BAF8B3
:104198000230800100F4FE501843AAF802000BF028
:1041A80055F8000104F829000BF050F814F82930EC
:1041B80000F00F00184304F829000BF047F88AF8BC
:1041C800010004F03DFC40E0724B012283F83720E7
:1041D8003BE00BF03BF8FF28824622D100238DF804
:1041E8001B309DF81B30072B14D89DF81B006A4A1A
:1041F8009DF81B3052F8300002EBC30301215B68C5
:10420800994089B2042201F08DFF9DF81B300133DB
:10421800DBB2E4E74FF090400121002201F082FF79
:1042280013E007283FF6E2AB00200BF05FF80BF035
:1042380039F8D9F800000AF0A7FC18B932200AF0BA
:10424800D7FBF6E7504601F07BFF00200BF04EF855
:10425800FFF704BA514B98590AF096FC18B9322066
:104268000AF0C6FBF6E70AF003FE05F03BF94C4BF3
:104278004C4ADA60FFF7FFB90C2824D00A2826D167
:10428800494D4A480BF0BAF8284623210FF04BFA5B
:1042980008B1401B20602368E3B94348236000212C
:1042A80030220FF00AFA3B78002B46D1404B9B682E
:1042B800002B69D03F48984766E00AF081FAFFF77B
:1042C800CDB90C2847D13C480BF098F835E00D28BB
:1042D80035D1D5E75A1EA95C202901D11346DBE761
:1042E800314A23600021D154344B354DD3F800A016
:1042F800D5F800B0DFF8B09058460FF022FA06461D
:104308003246484659460FF025FA2E4A28B919F878
:10431800063053445B78590703D010359542E7D3EC
:1043280006E0954204D2701CEB684844984702E0C6
:1043380025480BF063F80023AFE7244807E07F28FF
:104348000DD1013B184A224823600021D1540BF0BB
:1043580055F8FFF7EEB87F2804D1FFF7EAB82F2BFE
:104368003FF6E7A8A0F12002D2B25E2A3FF6E1A804
:1043780013B920283FF4DDA85A1C22600A4AD054F9
:104388000BF034F8FFF7D5B811B0BDEC028BBDE8DF
:10439800F08F00BF900E0020686A0108E81C00201A
:1043A80000ED00E00400FA059012002036760108BE
:1043B800F4190020C80E00204A6701080C010020EB
:1043C8000C4E0108DC4F01085567010845670108D4
:1043D80071670108801D00202DE9F0472DED028B43
:1043E8004728A0B0044600F0528600F2CE802E285E
:1043F80000F0018667D8222800F0AC8423D803286F
:1044080000F03A8214D8012800F02B82022840F0EC
:104418008A8604200AF06AFF43200AF034FF4C2001
:104428000AF031FF46200AF02EFF4C2000F0B5BDFF
:10443800042800F02B82052840F075861A200AF01F
:1044480055FF002432E2282800F06E8515D824286C
:1044580000F05585262840F06686C34C06200AF0F1
:1044680045FFB4F858010AF044FFB4F85A010AF0BD
:1044780040FFB4F85C0100F0A1BD2A2800F0678570
:104488002C2840F05086B84C0C200AF02FFF94F8E6
:1044980090010AF0F8FEB4F89A010AF02AFFB4F87D
:1044A80096010AF026FFB4F898010AF022FF94F862
:1044B80091010AF0E8FEB4F89C010AF01AFFB4F87A
:1044C8009E0100F07BBD3A2800F0DB821DD834281D
:1044D80000F070840DD8302800F0A385322840F011
:1044E800228601200AF002FF9F4B93F8920100F008
:1044F80054BD362800F06585382840F0148604201D
:104508000AF0F4FE984C00F000BD402800F0488501
:1045180011D83B2800F017843D2840F00486924CBF
:1045280002200AF0E3FE94F8E0010AF0ACFE94F8E9
:10453800DF0100F032BD452800F0E28500F29685E3
:10454800422840F0F085884C10200AF0CFFE6079B0
:104558000AF099FEA0680AF0D5FE94F890010AF0D6
:1045680092FEB4F858010AF0C4FEB4F85A010AF0F1
:10457800C0FEB4F85C010AF0BCFEB4F880010AF091
:10458800B8FEB4F8820100F019BD6F2800F0CA82A5
:1045980000F2F280662800F0C58100F2BE804D2846
:1045A80000F0DB8415D8492800F0B5824B2840F08C
:1045B800BA856D4C04200AF099FE94F8D6010AF0E9
:1045C80062FE94F8D7010AF05EFEB4F8D80100F054
:1045D800F5BC642800F08381652840F0A485634C0D
:1045E8000B200AF083FE20880AF083FE6268604B85
:1045F8009A420CBF2089608980B20AF07AFEE3688B
:10460800C3F3C000C3F38002800040EA4200C3F352
:1046180040021043C3F3401240EAC20003F0100303
:1046280018430AF066FE228A6369247E02F00801B4
:1046380003F4475949EA010903F4804149EA0109A9
:1046480003F4004149EA010903F4803149EA010908
:1046580003F4003149EA010903F4802149EA010918
:1046680003F4002149EA010903F4801149EA010928
:1046780003F0007349EA0303DFF8F89099F8009013
:1046880012F0010FC9F3800914BF4FF002084FF070
:10469800000843EA090312F0020F43EA080314BFB3
:1046A8004FF0040C4FF0000C12F0040F43EA0C0C0E
:1046B80014BF4FF0100E4FF0000E12F0400F14BF51
:1046C800202700274CEA0E0E12F0100F14BF4FF4EB
:1046D800007600264EEA070712F0200F14BF4FF4A9
:1046E800806500253E4312F4807F14BF4FF40060BC
:1046F8000020354312F4007F14BF4FF4001100214D
:10470800284312F4806F41EA000114BF4FF0806320
:104718000023002019430346F1E0692800F097813F
:104728000AD8672800F01E81682840F0FC84102011
:104738000AF0DCFD002482E16D2800F09B8100F284
:10474800BD816C2840F0EF84084C06200AF0CEFDAD
:10475800B4F86C000AF0CDFDB4F86E000AF0C9FD9B
:10476800B4F8700000F02ABC801D0020D00E002094
:1047780000540040E02A0020772800F079834BD8C5
:10478800732800F095833CD8702800F0F5817228D2
:1047980040F0C984BD4C16200AF0A8FDB4F8960173
:1047A8000AF0A7FDB4F840010AF0A3FDB4F84201ED
:1047B8000AF09FFDB4F844010AF09BFDB4F8D80153
:1047C8000AF097FD00200AF05EFD00200AF05BFD6C
:1047D80000200AF058FD94F885010AF054FD94F879
:1047E80092010AF050FD00200AF04DFDA84B1B6D08
:1047F8000A20B3F9623093FBF0F080B20AF079FD39
:1048080083E3742800F0FB82752840F08C842F2005
:104818000AF06CFD9F4C8EE2A02800F062830AD853
:10482800782800F0AB807B2840F07D843C200AF09B
:104838005DFD002429E2F12800F0DB80FE2800F06D
:104848004283F02840F06F84914C04200AF04EFD1A
:10485800236DB3F866000AF04CFD236DB3F86400CD
:10486800ACE303200AF042FD00200AF00CFD2046CC
:104878000AF009FD0D2090E30AF038FD01200AF046
:1048880002FD0B200AF0FFFC002086E306200AF058
:104898002DFD4D200AF0F7FC4F200AF0F4FC5420BF
:1048A8000AF0F1FC4F200AF0EEFC18E37A4B185D91
:1048B80001340AF0E8FC0B2CF8D10024774B185D82
:1048C80001340AF0E0FC082CF8D10024744B185D80
:1048D80001340AF0D8FC072CF8D100F022BC0720DC
:1048E8000AF004FDE7200AF0CEFC684B58790AF07C
:1048F800CAFC00200AF0C7FC042000F010BCA34248
:104908000AD2684A9D5C012202FA05F50D421CBFD5
:104918009A4010430133F2E70AF0F4FC5B4B93F83A
:10492800A8073AE312200AF0E1FC5F4B1B88B3F5B5
:10493800806F8CBF082601260025554C04F13403EE
:1049480033F9150090FBF6F0013580B20AF0D1FC7E
:10495800032DF2D1608F0AF0CCFCA08F0AF0C9FCBD
:10496800E08FB4E210200AF0C1FC00244F4B185D20
:1049780001340AF088FC102CF8D1D2E370200AF038
:10498800B5FC0026424D0E242B6D7443234401369A
:10499800B3F825010AF0ADFC2B6D2344B3F82701C9
:1049A8000AF0A7FC2B6D2344B3F829010AF0A1FCF7
:1049B8002B6D234493F82B010AF065FC2B6D2344DF
:1049C80093F82C010AF05FFC2B6D234493F82D011A
:1049D8000AF059FC2B6D234493F82E010AF053FC7E
:1049E8002B6D1C44D4F82F010AF08CFC082EC9D179
:1049F80097E37020254C0AF079FC04F1700594F8CF
:104A0800D0000AF040FC94F8D1000AF03CFC94F87D
:104A1800D2000AF038FC94F8D3000AF034FC94F879
:104A2800D4000AF030FC94F8D5000AF02CFC0734C6
:104A380094F8CF000AF027FCAC42E0D171E31C4B9C
:104A4800185D01340AF01FFC102CF8D169E3194DE8
:104A58002878400000F0FE000AF048FC00242B787B
:104A68009C4280F05E83144B33F814000AF041FC3A
:104A78000134F4E706200AF039FC00200AF042FC71
:104A88002DE204200AF032FC48E300BF801D00201C
:104A9800D00E00208B47010857650108636501089F
:104AA8003B650108E90E002008000020100F0020D7
:104AB800240F002060250020C21C002007200AF0D7
:104AC80015FCB54BB54C1888FF28A8BFFF20C0B20D
:104AD8000AF0D9FBB24B18684FF6FF75A842A8BF79
:104AE800284620EAE07080B20AF003FCB4F87200AD
:104AF8000AF0FFFBAB4B606F93F885313BB10A239B
:104B08005843A842A8BF284620EAE07001E000F315
:104B18000F0080B252E202200AF0E8FB9F4BB3F884
:104B280078004BE29D4C0B200AF0E0FBE36F18780D
:104B38000AF0A9FBE36F58780AF0A5FB0026254682
:104B4800EB6F964C3344013618790AF09CFB032E20
:104B5800F6D1E36FD8790AF096FBE36F98780AF0FC
:104B680092FBE36FD8780AF08EFBE36F58890AF05E
:104B7800C0FBE36F187A10E2884C1E200AF0B6FBDF
:104B8800236D1B78022B4FF000056BD1236D03EBCF
:104B9800850393ED080AB2EE048A20EE080A0EF0A7
:104BA8009BFF80F30800C0B20AF06DFB236DDFEDB8
:104BB8007E7A03EB850393ED0B0A20EE270A0EF0AD
:104BC8008BFF80F30800C0B20AF05DFB236DDFEDB8
:104BD800777A03EB850393ED0E0A20EE270A0EF091
:104BE8007BFF80F30800C0B201350AF04CFB032DAF
:104BF800CCD1072D236D23D193ED110A20EE080A9D
:104C08000EF06AFF80F30800C0B20AF03CFB236D87
:104C180093ED120A20EE080A0EF05EFF80F30800FA
:104C2800C0B20AF030FB236D93F84C3000EE103A16
:104C3800B8EE400A0EF050FF80F30800C0B20BE057
:104C48002B4458780AF01FFB236D2B44D87A0AF0BE
:104C58001AFB236D2B44587D01350AF014FB0A2DED
:104C6800C7D15EE2236D2B4458780AF00CFB236D04
:104C78002B44D87A0AF007FB236D2B440135587D65
:104C88000AF001FB0A2DEDD14BE2444D9FED478A16
:104C98002B6D03EB840393ED080A20EE080A0EF04F
:104CA8001BFF80B20AF025FB2B6D03EB840393ED09
:104CB8000B0A20EE080A0EF00FFF80B20AF019FB6B
:104CC8002B6D03EB840393ED0E0A20EE080A0EF019
:104CD80003FF013480B20AF00CFB032CD5D1072C5A
:104CE8002B6D16D193ED110A20EE080A0EF0F4FE92
:104CF80080B20AF0FEFA2B6D93ED120A20EE080A34
:104D08000EF0EAFE80B20AF0F4FA2B6D93F84C002C
:104D18000BE0234458780AF0ECFA2B6D2344D87A38
:104D28000AF0E7FA2B6D2344587D01340AF0E1FAC2
:104D38000A2CD4D1F5E114F8010F002800F0F18114
:104D48000AF0A1FAF7E701200AF0D0FA134B1B6D1D
:104D5800187822E150200AF0C9FA00250F4B1C6D83
:104D6800134B04EB85040C2194F8852001FB0233D6
:104D7800013593F838000AF086FA94F886000AF0AC
:104D880082FA94F887000AF07EFA94F888000AF00C
:104D98007AFA142DE2D1C4E188120020D00E002046
:104DA800E0110020801D00200000C84200007A4465
:104DB8008C47010848200AF099FA0025C54B1C6D5C
:104DC800062303FB0544013594F8DA000AF05BFA80
:104DD80094F8D5000AF057FA94F8D6000AF053FA76
:104DE80094F8D7000AF04FFA94F8D8000AF04BFA72
:104DF80094F8D9000AF047FA0C2DDFD191E14FF071
:104E0800000801260027B34B1A7E974227DA193388
:104E18000024FA5CB04D0C2305F130016343595C62
:104E2800914207D12B44586B0EF08BFC82462EB969
:104E3800B14605E001341C2CECD10EE080440CE0B6
:104E4800D1450ADA0C2303FB04535B6B13F8090002
:104E58000AF019FA09F10109F2E70137D3E7002E40
:104E680000F05F815FFA88F00AF040FA0026C9E78F
:104E7800984D287E0AF03AFA00242B7E9C4280F056
:104E88005081964BE65C002193480C2200F13007D4
:104E980002FB01F3DA5DB24205D1034493F838000E
:104EA8000AF0F1F902E001311C29EDD10134E4E7FF
:104EB80008200AF01BFA0124E0B201340AF0E3F9F1
:104EC800092CF9D12DE108200AF010FA00200AF087
:104ED80010FA00200AF00DFA00200AF00AFA002061
:104EE8006CE00C200AF002FA7D4B18680AF00AFA06
:104EF8007C4B18680AF006FA7B4B18680FE104200F
:104F08000AF0F4F9794B986809E194F87A010AF003
:104F1800BAF994F87E010AF0B6F994F87D010AF01E
:104F2800B2F994F87F0138E0704C07200AF0DEF9F6
:104F3800B4F880010AF0DDF9B4F882010AF0D9F971
:104F480094F884010AF09FF9B4F8860136E001204C
:104F58000AF0CCF9654B58791FE0654C654D20780F
:104F680000EB4000C0B20AF0C1F9002623789E4247
:104F780005F1020580F0D58015F8020C0AF083F9D6
:104F880015F8010C00EB800000EB800000F2EE2029
:104F980080B20AF0AEF90136E8E70AF074F9C0E029
:104FA80008200AF0A3F90024504B2344013493F855
:104FB80088010AF068F9082CF6D1B2E00AF099F9EC
:104FC800AFE0444B494C93F88000C0EBC000C0B23E
:104FD8000AF08CF904F1200594F8F0010023464A00
:104FE800D25C904200F0A1800C33302BF7D108340A
:104FF800AC42F1D195E040203C4C0AF077F904F13D
:105008004005B4F8A0020AF074F994F8A2020AF074
:105018003AF9043494F89F020AF035F9AC42F0D119
:105028007FE0E020314C0AF061F904F18005B4F822
:10503800220200F03F000AF05CF9B4F82202C0F343
:1050480086100AF056F994F8200200090AF01BF9B4
:1050580094F8200200F00F000AF015F9043494F8CF
:105068001D020AF010F9AC42E1D15AE0234C0D20A0
:105078000AF03CF907F0BAFF0AF005F9A0880AF02F
:1050880041F920690AF03EF907F090FF47E00AF07D
:10509800F1F8054684200AF029F928460AF032F981
:1050A800164B1C6905F18003A3428CBF641B802446
:1050B80003F01AFE28462246694608F0BDF8002487
:1050C8000546AC422DDA1DF804000AF0DCF801347C
:1050D800F7E700BFD00E00208C470108E90E00203A
:1050E800ACF7FF1FB0F7FF1FB4F7FF1F801D0020AC
:1050F80060250020201F00206C25002008000020CB
:1051080013200AF0F3F80024164B185D01340AF056
:10511800BAF80B2CF8D100200AF0F4F800200AF0B5
:10512800F1F8012018E0002016E00AF0ACF8B4F815
:10513800F2010AF0DEF894F8F4010AF0A4F894F801
:10514800F5010AF0A0F894F8F7010AF09CF894F831
:10515800F6010AF098F84AE720B0BDEC028BBDE8EA
:10516800F08700BF5765010810F80A3C0133DBB22D
:105178000A2B84BF10F8131C044A00F80A3C82BFAB
:10518800002322F8113000F80A3C7047182A002042
:10519800334A136C90681944081A40F68C239842D5
:1051A80070B513469160D06051603BD9127893F97D
:1051B80045108A4210460BD1111F082908D893F8C8
:1051C8004610182901D8013103E083F8442002E091
:1051D800002183F8461093F944402149A24219D18D
:1051E80091F84740B4B10C310024944206DA1D4DC1
:1051F80051F8046F25F814600134F6E70C2805D03F
:105208001849002421F810400130F7E716480178C2
:105218000131017083F84520002201211A7083F8BA
:10522800471070BD92F84710C9B1A0F2EF2440F2C0
:10523800DA518C4208D811780B2905D80B1D013199
:10524800117042F8230070BD002283F84720074BF5
:1052580003F13002002143F8041F9342FAD170BDD4
:1052680080080020182A00207D0100208C080020DA
:10527800024A136C013319441164704780080020F6
:10528800024B53F820301B6819607047E82500204E
:10529800064B53F820301A681B89A1F57A715943D7
:1052A8004FF47A7391FBF3F111607047E825002001
:1052B800F0B5046D8668236823F0010323608379C1
:1052C800054613F0020F40790CBF4FF0000E4FF463
:1052D800005E13F0040F14BF4FF48067002710F02E
:1052E800010F14BF042100218307206820F001006A
:1052F8002060626822F440524EEA0202626022682C
:1053080022F4B05323F00C0348BF41F008013B439B
:105318000B432360A36895B023F44073A3606846E9
:1053280001F07EFD284B9C4201D10C9B0EE0274BDF
:105338009C4201D10D9B09E0254B9C4201D10E9B5B
:1053480004E0244B9C420CBF0F9B109B2268A87959
:10535800170448BF5B00B3FBF6F206FB1233B3EB4E
:10536800560F236828BF01321E0441BF4FF6F07361
:10537800C2F34201134041EA03026B7992B213F07F
:10538800020FA28100F0010114BF4FF40032002285
:10539800DC0748BF42F480322B6D11B159680A43CB
:1053A80002E0596821EA02025A609A6801074CBF74
:1053B80042F0080222F008029A601A6842F00102DC
:1053C8001A6015B0F0BD00BF00380140004400402D
:1053D80000480040004C00403D4B1B78012B30B585
:1053E80014BF00240324B1B9036A23F00103036244
:1053F8008169036A21F0F30123F00A0341F00101F6
:1054080042F001021A4341EA041181610262836990
:1054180023F00C031BE004291DD1016A4FF6EF733A
:105428000B4003628169056A120121F473414FF64A
:105438005F7342F0100241F480712B4092B2134323
:1054480041EA043181610362836923F44063836123
:105458008369836130BD0829016A1AD14FF6FF6359
:105468000B400362C169036A9BB289B223F42063CB
:1054780043F4807321F0F30143EA022241F0010171
:1054880092B241EA0411C1610262C2694FF6F37334
:1054980019E04EF6FF730B400362C369056A40F6D4
:1054A800FF41194045F6FF732B4043F4805343EA0C
:1054B800023241F4807192B241EA0431C161026260
:1054C800C2694FF2FF331340C361C369C36130BD82
:1054D8007C08002038B510F80E2C50F8043C04461F
:1054E80052B9012200F80E2C20F80C1C997A186881
:1054F8000222BDE838406FE730F80C2C20F80A1C6F
:10550800891A89B220F8081C074A10F80F0C0025E0
:1055180022F8101004F80E5C1868997A2A46FFF7EA
:105528005BFF04F8065C38BD182A0020044B53F8CA
:1055380020301BB107289CBF1B681960704700BF4B
:10554800A8090020084A13689B050BD5074B0021C2
:105558001970074908684FF6FE7303400B604FF453
:1055680000735360704700BF00000240DE2A00202D
:10557800300002402DE9F047664D2B6866490A78ED
:10558800581C02F0FF068E460AB10346F6E72B6068
:10559800687BAB6895F80C80AA7B374639B220291E
:1055A80000F09B80DFF880C10CEB81033CF82110F0
:1055B800DC789B78C3F1FF039BB2002B65D0C3F165
:1055C800FF0363434FF03C0C1B12B1FBFCF9B9F12C
:1055D800050F5DD8DFE809F0030B1A293A4AE01AEB
:1055E800DAB24143B1FBFCF01044C0B251E0B1FB68
:1055F800FCF00CFB101189B2DAB2C1F13C01E31ADC
:105608004B432046B3FBFCFC94442CE0B1FBFCF07C
:105618000CFB10115FFA83F8E21A89B24A43B2FB15
:10562800FCF24244D2B2204632E0B1FBFCF90CFB5A
:10563800191189B25FFA83F8E01AC1F13C014843B5
:10564800B0FBFCF04044C0B2224621E0B1FBFCF8BC
:105658000CFB1811D8B289B2E31A01FB03F2B2FBB2
:10566800FCFC224684445FFA8CF412E0B1FBFCF89F
:105678000CFB181189B2D8B2C1F13C01E31A4B43B3
:10568800B3FBFCF20244D2B203E02246204600E01B
:1056980044464FEA042C4CEA004C4CEA020C17230F
:1056A80006F117014FF0010808FA03F8C91A18EAB9
:1056B8000C0F89B2DFF8748014BF4FF011094FF056
:1056C800090913F1FF3308F80190E9D218360137B8
:1056D800B6B2BFB2114BA04660E7AA73AB60104ADE
:1056E800E98001238EF800300E4985F80C8040F2DD
:1056F8002A336873AE80536000234B620B889BB2D9
:1057080043F001030B80136843F001031360BDE805
:10571800F08700BF540F0020DE2A0020600F002011
:105728003000024000440140B4070020F009002086
:1057380073B506460D46002401232A88A340134268
:105748001AD0AA78009302F003038DF80430EB789E
:10575800022B03D0032B0CBF032301238DF8053044
:105768003046C2F301136946C2F381028DF8063050
:105778008DF8072001F0C2FC0134102CDCD102B0F6
:1057880070BD2DE9F04F734EF57B07460C4687B088
:1057980011469A4600686B1C914622464FF0020B50
:1057A800F37308F09FFC3B897868ADF8043001A9D1
:1057B8008DF806B08DF807B0FFF7BAFF0023ADF8F3
:1057C8000A30ADF81230ADF8163070230193BA7A6A
:1057D8003C68CDF80CA0012306F110082D01ADF8A6
:1057E80008304FF48073A844ADF810B0ADF8143009
:1057F8000C2A7ED8DFE802F0077D7D7D0F7D7D7D58
:10580800387D7D7D5E00204601A901F0CBFAA369B1
:1058180043F0080326E0236A4F4823F0100323626D
:10582800236A6168A26922F0807222F4E642844207
:1058380042F4E04206D000F50060844202D043F012
:10584800300307E023F0E00321F4406143F0300324
:1058580041F480616160A261C4F838A02362A36941
:1058680043F40063A36144E0236A3B4823F4807354
:105878002362226A6168E369844223F0730343F078
:10588800700306D000F50060844202D042F44072F2
:1058980007E022F4606221F4405142F4407241F47E
:1058A80080516160E361C4F83CA02262E36943F07F
:1058B80008031DE0236A284823F480532362226AE0
:1058C8006168E369844223F4E64343F4E04342F425
:1058D800405203D000F50060844201D141F4804178
:1058E8006160E361C4F840A02262E36943F40063A5
:1058F800E3613A7B3B681AB15A6C42F400425A643D
:105908001A8892B242F001021A80BA7A0C2A18D880
:10591800DFE802F0071717170B1717170F171717D6
:105928001300721903F134010AE0721903F1380106
:1059380006E0721903F13C0102E0721903F140011B
:10594800116135444046A5F818906B6107B0BDE871
:10595800F08F00BF540F0020002C0140054B9842E7
:105968000CBF054A054A138801339BB213800020F7
:10597800704700BF00540040D80E0020DA0E002007
:10598800400070B5C5B22D482D4B00684FF4204437
:105998001C608669360404D52646013C002EF8D1E1
:1059A80012E04668274C344044F0807444F4903444
:1059B8002C4344604FF420441C608669B60726D403
:1059C8002646013C002EF8D11C601AE02146013C15
:1059D8000029F9D081690E06F8D544681949214093
:1059E80041F0007141F48031294341604FF4204176
:1059F80019608469A4070FD40C460139002CF8D12A
:105A08001960FFF7ABFF003018BF012070BD4FF4DD
:105A1800204481621C60DDE782624FF420421A60F4
:105A28008169890605D41146013A0029F8D11A601E
:105A3800E7E71A602023C361012070BDD40E00205F
:105A4800B81B0020009800FCF8B504460E4617461F
:105A58000025204620210DF066FE0446D0B1013411
:105A680020460DF0C5FEB0F5617F05DB40F6340336
:105A78009842A8BF184601E04FF46170A0F5617024
:105A8800192390FBF3F00DB9307000E070703B788B
:105A980001333B700DB90125DBE72046F8BD30B571
:105AA80005460C461346294622460248BDE83040C2
:105AB80003F0EEBB606901087FB504780646E4B9D7
:105AC800354B1B6803EB8403192193F8870093F87F
:105AD800886093F8852093F886304FF4617511FB40
:105AE800005011FB0651009001912C4821460134C9
:105AF80003F0CEFB142CE3D14BE00DF079FE132814
:105B0800054641DC244B701C1C68202100238DF8BD
:105B18000F300DF008FE2035064670B101363046CC
:105B28000DF066FE1A289FBF04EB850358719DF897
:105B38000F30013398BF8DF80F30304620210DF01B
:105B4800F2FD064670B1013630460DF051FE0D28C3
:105B58009FBF04EB850398719DF80F30013398BF00
:105B68008DF80F3004EB85043046E11D0DF10F026E
:105B7800FFF76AFF9DF80F30042B0AD0601D002143
:105B880004220DF09AFD04E0054800211322FFF7D6
:105B980086FF04B070BD00BF200F00207F69010898
:105BA80094690108014809F029BC00BF9A690108F5
:105BB800F8B50478064674B9304DB5F8C421B5F87F
:105BC800C6312F482146013403F062FB042C05F14D
:105BD8000405F2D1F8BD2B490DF078FDA8B9274B83
:105BE8004FF47A714FF4FA62A3F8C411A3F8C621EE
:105BF800A3F8C811A3F8CA21A3F8CC11A3F8CE21A1
:105C0800A3F8D011A3F8D221F8BD30460DF0F0FD6D
:105C1800032805462BD8304620210DF084FD044684
:105C280030B1013420460DF0E3FD0126074600E0BF
:105C38000646204620210DF076FD10B9BDE8F84053
:105C4800B0E701300DF0D4FD012EF7D1A7F2EE2216
:105C580040F2DC539A42F1D8A0F2EE229A42EDD8F3
:105C6800064B703503EB85039F80D880F8BD064846
:105C780000210322BDE8F84011E700BF801D002085
:105C8800A8690108BB690108567701082DE9FF4199
:105C980004780546002C39D17348744D09F0AEFBE1
:105CA800D5ED047AF5EE407AF1EE10FA00F0D880DE
:105CB80021466F4803F0ECFA95ED040A684603F0B4
:105CC80067F901466B4803F0E3FA95ED050A684663
:105CD80003F05EF90146674803F0DAFA95ED060A23
:105CE800684603F055F90146624803F0D1FA95ED8C
:105CF800070A684603F04CF9013401465E4803F090
:105D0800C7FA0C2C05F11005CAD1A9E05B49052298
:105D18000DF020FD40B9554B03F1C002002143F8B6
:105D2800101F9342FAD19BE02846554904220DF0F2
:105D380011FD04462846002C40D120210DF0F3FC2B
:105D4800002800F08D80451C28460DF0FAFC074617
:105D58004C4B53F824601EB94B4809F04FFB7FE0C9
:105D680028463146FAB20DF0F5FC01340028EFD18F
:105D78003E4B03F1C0029E46002143F8101F934298
:105D8800FAD1424B03EBC4029846D2F804C0BCF1E6
:105D9800000F04D131463E4803F07AFA57E0002755
:105DA80018F834309F42F5DA3B010EEB03056344E3
:105DB8000FCB103585E80F000137F1E70DF018FD1E
:105DC8000B28064647DC284620210DF0ACFC05468A
:105DD80050B10135284603F051F8244B03EB061364
:105DE80083ED040A012400E00446284620210DF032
:105DF8009AFC054648B10135284603F03FF81B4B8D
:105E080003EB061383ED050A0134284620210DF023
:105E18008AFC054648B10135284603F02FF8134B94
:105E280003EB061383ED060A0134284620210DF002
:105E38007AFC10B9FFF7B6FE12E0013003F01EF845
:105E48000A4B032C03EB061686ED070AF2D111481C
:105E5800FFF71CFF04E0104801210C22FFF71FFE8A
:105E680004B0BDE8F08100BFC1690108801D0020B1
:105E7800DC690108E2690108DA740108BB690108F4
:105E8800E6690108DC4F0108EB6901089068010820
:105E9800FA6901087467010894690108F0B5047883
:105EA80087B006461CBB514B1968062303FB041137
:105EB800192091F8D65091F8D77091F8DA2091F816
:105EC800D5304FF4617610FB056510FB076000952F
:105ED800019091F8D8000290D0314548497A039151
:105EE8002146013403F0D4F90C2CDCD17CE00DF010
:105EF8007FFC0B28044672DC3C4B701C1D6820217B
:105F080000238DF817300DF00EFC064680B10136DF
:105F180030460DF06DFC03289FBF062303FB045396
:105F280083F8DA009DF817309CBF01338DF81730DD
:105F3800304620210DF0F7FB074680B1013738467F
:105F48000DF056FC0D289FBF062303FB045383F86E
:105F5800D5009DF817309CBF01338DF81730062601
:105F68006643A9193846D6310DF11702FFF76CFDC3
:105F780020210DF0D8FB074670B1013738460DF0E7
:105F880037FC14289FBF9DF817307619013386F81F
:105F9800D80098BF8DF81730384620210DF0C3FB84
:105FA80078B101300DF024FC0D289FBF062303FBB8
:105FB800045383F8D9009DF817309CBF01338DF83E
:105FC80017309DF81730062B0ED0062202FB04501E
:105FD8000021D5300DF071FBFFF7E4FD04E0054822
:105FE80000210B22FFF75BFD07B0F0BD200F00205A
:105FF800066A0108946901082DE9F3470478074601
:106008004CB9204601A908F0CDFA0134FFF7F4FF96
:10601800122CF6D179E00DF0EBFBC5B2112D6FD83B
:10602800781C20210DF07FFB394C3A4F05F1D00642
:10603800034614F8168030B9A8F10202D2F100081C
:1060480048EB020843E000F1010A597838460DF0A0
:106058006AFB60B1032D8CBF03230023C01B3B44A4
:1060680053FA80F090F80490B9F1030F02D1FFF7CA
:1060780099FD4AE0A9F10203D3F1000850464FF018
:10608800200148EB03080DF04EFBD8B1B8F1000F22
:10609800EDD001300DF0ACFB40F2ED2380B2984218
:1060A80005DD40F6CA039842A8BF184601E040F251
:1060B800EE2004EB4603A0F2EE20192290FBF2F04A
:1060C800587002E0B8F1000FD1D104F8169014F816
:1060D8001630FA5CB8F1000F0DD00D4B0E4803EBEB
:1060E80046062946737840F2EE24192505FB03433A
:1060F80003F0CEF809E02946084803F0C9F804E09F
:10610800074800211122FFF7CAFC02B0BDE8F0875A
:10611800801D00201C490108266A0108386A010808
:106128005677010807B50123ADF8041001A98DF8C9
:1061380006208DF80730FFF7FBFA03B05DF804FB83
:106148002DE9F041064672B62D4D8021402729855C
:10615800284604222F85FFF7E5FF28463946012205
:10616800FFF7E0FF274850F8364000EBC6002368E9
:1061780042680126510006FA01F848EA03039640EE
:106188002360A661AF612B8A1F06FCD4236848EA06
:10619800030323601A4B4022B1B221851A852022BD
:1061A8009A6140F60557164D2B8A180603D4002F1E
:1061B800F9D0013FF7E7A66120460422FFF7B2FFB6
:1061C80087B10F4B1A8A1206E0D5228A92B216427C
:1061D8004FF040014FF0200215BF996119859A616F
:1061E8001A85EEE740212023A9612846AB610222E7
:1061F800FFF798FF62B60A20BDE8F04108F0F8BB47
:1062080000040048686A0108002208490C2303FBBF
:1062180002135968814204D10022C2621A725A607C
:1062280070470132042AF0D1704700BF6C25002066
:106238002DE9F04F87B0074602919DF8444011467A
:106248001A469DF8403000250C20674E684300EB45
:10625800060E8057B842B14605D19EF808A0BAF19B
:10626800000F04D0BBE00135042DEDD1B7E0012FBC
:1062780000F0A48005DC002F40F0B18000945B485A
:10628800A1E0022F00F09D80142F40F0A880584E06
:10629800B36943F00103B36173694FF0904443F469
:1062A8000033736103224FF0010B4FF4805804A9A7
:1062B8004FF090408DF815200392CDF810808DF89E
:1062C80014B08DF816B08DF817A000F017FFA4F8D9
:1062D8002880C82008F08CFBC4F818807369039ADA
:1062E80043F40033736120464FF4C0538DF81520F2
:1062F80004A902228DF81420039204938DF816A0A5
:106308008DF817A000F0FAFE636A23F47043636205
:10631800636A43F460436362636A23F470236362CD
:10632800636A43F460236362324B334C4FF4802139
:1063380019601223A36404F14800082384F84D303F
:1063480084F84EB008F09AF82C4B2D49C3F800A0F9
:10635800F369039A43F40003F3612A4B04A8D96054
:106368008DF810708DF811208DF812A08DF813B0EB
:1063780008F03AF82A238DF810309DF813308DF87C
:1063880011B08DF812A01BB104A808F02DF804E094
:106398001D4B4FF48062C3F884201C4A1C4B1360C9
:1063A80002221A721B4A1C4B13601C4A1C491B68A8
:1063B800116098471B4B23600F4807E000941A4868
:1063C80001E01A48009405F0CBF840B10C2303FB18
:1063D80005959DF8083007712B72686000E0002071
:1063E80007B0BDE8F08F00BF6C25002000380140E1
:1063F80000100240140401404C100020D800424212
:106408000005FA0500ED00E000E100E0BC1C0020FA
:106418009C250020241B0020D0000020201B0020E9
:106428001C000020284901080044004000480040A2
:1064380010B5084B1968002201EBC20393F902401A
:10644800844201D1981C10BD0132042AF4D10020E5
:1064580010BD00BF68250020F0B5027887B08AB962
:106468004A4C04F1200694F8F02100234849595673
:1064780050B281426ED00C33302BF7D10834B4427D
:10648800F1D181E0002204920592451C0DF0B0F98B
:10649800C4B260B2FFF7CCFF074618B18DF81040C0
:1064A800012400E00446284620210DF03CF9054669
:1064B80038B1013528460DF09BF90134ADF81200CA
:1064C800E4B20026284620210DF02DF9B0B3451C72
:1064D80028460DF08DF900222E4951F822308342CA
:1064E8005FFA82FE04D00132082AF5D1002300E0C9
:1064F800734651F82320824220D1022E0FD0032E5A
:1065080012D05A1E012ED2B204D0042A13D88DF804
:1065180014300EE0042A0ED88DF8153009E0052B4A
:1065280009D88DF8173004E09A1E052A03D88DF88B
:1065380016300134E4B20136042EC3D1052C04D838
:1065480007B0BDE8F040FFF72DBB04AB03CB3860C4
:10655800796019E094F8F5010E4B94F8F45153F86A
:106568002000B4F8F221009094F8F70153F82000C5
:10657800019094F8F60153F82000029053F8253062
:10658800054802F085FE79E707B0F0BD801D0020C0
:106598006C2500205C560108476A010838B1438819
:1065A80011EA030003D08B420CBF01200220704780
:1065B80030B50B4B0B491C6891F85020032A0BD8B7
:1065C800134604EBC303551CEAB29D882842F5D054
:1065D80081F85020981C30BD81F85020002030BD33
:1065E800682500204C100020024B002283F8502020
:1065F800DEE700BF4C1000202DE9F047877890F8BF
:1066080003C0214DBBB2C7F1640E03EB83065C42A5
:10661800C3F178005FFA8EFE7600CCF16408A4B26C
:1066280080B2A3B20FFA83F9B9F1000F05DC002B91
:1066380014BFBA464FF0010A00E0F24613FB03F319
:1066480003FB0CF21AFB0AF392FBF3F3434403FB3C
:1066580009F30A2293FBF2F333449BB225F8023F75
:10666800B1F800904A880A34C9EB020AA4B21AB2F7
:1066780002FB0AF24FF47A73844292FBF3F34B4421
:106688002B80CED1BDE8F0879C10002010B5214AA0
:1066980018B9136802221A8210BD1F481468002313
:1066A8000380217811F07F0102460DD1637A9906A3
:1066B80044BF0221017013F0400F037814BF43F068
:1066C800010323F0010315E0012921D002291ED17D
:1066D800637913F0800F03F00F034FEA830303F18C
:1066E800804303F5B8431B6806D003F03003102B32
:1066F80007D10123137004E003F44053B3F5805F1E
:10670800F6E7064B1B681B699847034810BD1846F7
:1067180010BD00BFBC1C0020B8100020201B0020AA
:1067280010B5064C18B9236801221A8210BD044B13
:106738001B689B68984720680C3010BDBC1C002063
:10674800201B002010B5064C18B9236801221A82B4
:1067580010BD044B1B681B68984720680A3010BDA1
:10676800BC1C0020201B002003788B4283BF034BF6
:1067780003EB410148880020704700BFB810002093
:1067880070B500221346244914180C44A47E83EAE9
:106798000423082413F4004F4FEA430318BF83F47B
:1067A800815304F1FF3418BF83F0010314F0FF0490
:1067B8009BB2EFD10132192AE5D100F1190200F19B
:1067C8001A050A440D44967EAA7E02EB062292B26E
:1067D8009A421FD1104B93F83B50E2B2AA4216D20C
:1067E800431C03EB4203DBB2CA1801330B44927E0D
:1067F8009B7E03EB02239BB24FF4AF6253431B1300
:10680800064A03F5487322F814300134E5E70123FA
:1068180081F83C3070BD00BFB8100020BA100020CD
:1068280003788B420BD9074B1A78074B8900194418
:10683800086C02B1400800F5777080B270470020FC
:10684800704700BF64250020B810002007299DBFAD
:10685800034B03EB8101B1F870000020704700BFC3
:10686800B8100020034B03EB4101B1F89000C008B9
:10687800704700BFB810002070B5334C054608F0CB
:106888009BF8D4F8B030C4F8B000C31AB3F5FA5F77
:10689800C4F8B43082BF002384F8B83084F8B93023
:1068A80094F8B8302BB9A12D02BF274A012182F8EC
:1068B800B91094F8B910244A29B1D118EDB20133AE
:1068C8008D7682F8B83094F8B85094F8BA30AB4264
:1068D80039D11D4B93F8BB30052B02D0062B03D0C2
:1068E8002CE00020FFF74CFFE37E1E2B26D1002072
:1068F8000246C1B26B1E994219DA21448B7E0821E7
:10690800DBB283EA0206F60744BF83F01803C3F339
:10691800460301F1FF3154BF5B0843F0800311F0D7
:10692800FF01C2F34702ECD101301A46E1E72344E4
:106938009B7E9A4202D10320FFF722FF002384F8AE
:10694800B93084F8B83070BDB810002010B50446CE
:1069580008F032F80F4BD3F8BC20C3F8BC00821AF9
:1069680041F288318A42C3F8C02084BF002283F8EC
:10697800C42093F8C420074913440F2AE4B218BF6F
:10698800013283F8C54012BF81F8C420012381F881
:10699800D53010BDB810002010B5044608F00CF82A
:1069A8000F4BD3F8D820C3F8D800821A41F28831A7
:1069B8008A42C3F8DC2084BF002283F8E02093F8E1
:1069C800E02007491344142A18BF013283F8E14034
:1069D80012BF81F8E020012381F8F63010BD00BF16
:1069E800B81000202DE9F843324F3D682A8A2E7AE4
:1069F800B2B9042E14D1304C30482378012B0BD176
:106A08002F4B19682F4B89B20B445B0019681A6029
:106A180030230380227048E010230380072644E0D7
:106A2800AC8AAB69A24294BF04260226944228BFCE
:106A380014461FFA84F840469847214A13689BB2C7
:106A480003F1005303F540535B0004F1010E1B688A
:106A58009BB203F1005303F540534FEA6E0E5B00FF
:106A68000021714500F1020009D010F8019C10F8CE
:106A780002CC4CEA092C23F821C00131F1E7126855
:106A8800104B92B213445B001A681C602B8AC8EB47
:106A980003032B826B8A9844084BA5F81280302296
:106AA8001A80094B4FF440521A803B681E72BDE8A9
:106AB800F88300BFBC1C0020E32A00201A1B00201A
:106AC800505C004002300020181B00200E4B0F4A7B
:106AD8001B689BB203EBC00002443E294FEA420206
:106AE80009D94B09C80604BF03F1FF339BB29B02C7
:106AF80043F4004304E04B08C90748BF01339B0235
:106B080011681360704700BF505C004006300020D9
:106B180010B5454B1A68107810F07F0004D1537AED
:106B280023F02003537210BD02287AD15388002B1A
:106B380078D11379002B75D1537923F08000840024
:106B480004F1804101F5B84113F0800F096814BFC2
:106B580001F0300101F44051032862D8002960D0C7
:106B6800927A002A5DD004F1804404F5B8441906ED
:106B7800226825D502F03002102A4CD103F07F0399
:106B88009B0003F1804303F5B8431A68510641BFDF
:106B9800196840F60F720A4042F4004244BF42F0BE
:106BA800C0021A601A6822F4E04222F0400292B24F
:106BB80082F0300242F4004242F080021A602AE079
:106BC80002F44052B2F5805F25D128B9174B93F8EB
:106BD8002C10FFF77BFF11E09B0003F1804303F5C6
:106BE800B8431A68520441BF196840F60F720A4048
:106BF80042F4404244BF42F080021A60236823F402
:106C0800804323F070039BB283F4405343F4004362
:106C180043F080032360064B1B685B69984700209C
:106C280010BD022010BD00BFBC1C0020D0000020F9
:106C3800201B00200023036043608360838103617D
:106C480043618361C36103624362836270478A68F8
:106C5800036810B50C6A14430A6914434A6914435B
:106C68008A691443CA6914434A6A14438A6A23F432
:106C7800FF4323F070032243134303608B8943606F
:106C88000B6883604B68C36010BD02684FF6FE73E3
:106C9800134003600023036043608360C360294B93
:106CA800984201D1284A27E0284B984201D1264A28
:106CB8002AE0274B984201D1234A2DE0254B9842E0
:106CC80001D1214A30E0244B984201D11E4A33E0D9
:106CD800224B984204D11C4A536843F470032EE0B7
:106CE8001F4B984204D1184A536843F0706326E05A
:106CF8001C4B984204D11C4A536843F00F031EE012
:106D08001A4B984204D1184A536843F0F00316E02E
:106D1800174B984204D1144A536843F470630EE049
:106D2800144B984204D1104A536843F4704306E068
:106D3800114B984204D10C4A536843F470235360B2
:106D4800704700BF08000240000002401C000240DB
:106D58003000024044000240580002406C000240EB
:106D68008000024008040240000402401C04024063
:106D7800300402404404024058040240084BDA68D8
:106D8800D10709D4DA68D20608D4DB6813F0040FF7
:106D980014BF032004207047012070470220704769
:106DA80000200240036A23F001030362036A70B5FE
:106DB800446882690D6822F4803222F07302154318
:106DC8008A8923F0020313438A881343134A9042A3
:106DD8000FD002F5006290420BD002F5406290425B
:106DE80007D002F58062904203D002F5806290429B
:106DF8000DD1CA89CE8823F0080313430A8A24F4E4
:106E0800407414434A8A23F00403334314438A68C2
:106E1800446085614263036270BD00BF002C01407D
:106E2800994A536803F00C03042B2DE9F04105D06F
:106E3800082B06D095490160B3B916E0934B03605F
:106E480012E053685468C3F38343991CE30349BFB2
:106E5800D36A8F4B8D4C03F00F0344BF0133B4FB4F
:106E6800F3F34B43036000E000235168894FC1F3FB
:106E780003117D5C0168EDB221FA05F4446056689F
:106E8800C6F30226BE5D24FA06FEC0F808E056687E
:106E9800C6F3C226BE5DF6B2F440C460D2F82C80B8
:106EA800C8F3041808F00F0C07EB4C0C18F0100F7F
:106EB800BCF810C01FFA8CFC07D0BCF1000F04D03E
:106EC800B3FBFCFCC0F810C000E00161D2F82CC094
:106ED800CCF3442C0CF00F0807EB48071CF0100FFC
:106EE8003F8ABFB204D01FB1B3FBF7F7476100E098
:106EF8004161176BFF065ABF644F87618161176B49
:106F0800BF065ABF614FC761C161176B7F065ABF81
:106F18005E4F07620162176BFF0506D5994204D1DF
:106F2800AE4202D14F00476200E04462176BFF0493
:106F380006D5994204D1AE4202D14F00876200E0E3
:106F48008462176BBF0506D5994204D1AE4202D1BF
:106F58004F00C76200E0C462176B7F0506D59942EF
:106F680004D1AE4202D14F00476400E04464176B7D
:106F78003F0506D5994204D1AE4202D14F0087643D
:106F880000E08464176BBF0406D5994204D1AE4271
:106F980002D14B00C36400E08464156B3A4BAD0723
:106FA80001D1046315E01C6B04F00304012C01D12A
:106FB80001630EE01C6B04F00304022C02D14FF4B1
:106FC800004305E01B6B03F00303032B01D12F4B98
:106FD8000363146B2C4B14F4403F02D1C0F834E027
:106FE80018E01C6B04F44034B4F5803F01D14163D0
:106FF80010E01C6B04F44034B4F5003F02D14FF4A8
:10700800004306E01B6B03F44033B3F5403F01D166
:107018001E4B4363146B1C4B14F4402F02D1C0F871
:1070280038E018E01C6B04F44024B4F5802F01D13B
:10703800816310E01C6B04F44024B4F5002F02D1E6
:107048004FF4004306E01B6B03F44023B3F5402FD5
:1070580001D10E4B8363146B0B4B14F4401F02D108
:10706800C0F83CE020E01C6B04F44014B4F5801F29
:1070780001D1C16318E01C6B04F44014B4F5001F7F
:107088000AD14FF400430EE00010024000127A00CB
:1070980000093D00400000201B6B03F44013B3F5CA
:1070A800401F01D1134BC363126B134B12F4400FF3
:1070B80003D1C0F840E0BDE8F0811A6B02F4400249
:1070C800B2F5800F02D10164BDE8F0811A6B02F4B9
:1070D8004002B2F5000F02D14FF4004306E01B6BEB
:1070E80003F44003B3F5400F01D1024B0364BDE83C
:1070F800F08100BF00127A0000100240F0B50023B2
:107108000E681C460125A54005EA060EAE452BD1A2
:107118000F797A1E012A15D8856803229A4025EA34
:10712800020282604D7982689D401543856082889D
:1071380092B222EA0E0282808A798588A2402A4386
:1071480092B28280032205689A40D24315400560B6
:1071580005689F402F430760C7681740CA7902FA3D
:1071680003F547EA0502C2600134102C03F102035B
:10717800C8D1F0BD38B52DED048B4A4C0368C4F86E
:10718800F8308388A4F8FC30023A0D46062A05D860
:10719800DFE802F00A101822292F3500B4F8F83079
:1071A8000B80B4F8FA3013E0B4F8FA300B80B4F876
:1071B800F83005E0B4F8F8305B420B80B4F8FA30E8
:1071C8005B4205E0B4F8FA305B420B80B4F8F83063
:1071D8006B80B4F8FC301DE0B4F8F8305B420B80EB
:1071E800B4F8FA3012E0B4F8FA300B80B4F8F8309A
:1071F8000CE0B4F8F8300B80B4F8FA3005E0B4F8D5
:10720800FA305B420B80B4F8F8305B426B80B4F81C
:10721800FC305B42AB80244B93F83030002B3ED1DE
:10722800B5F9003094ED430AD4ED407A09EE103AEE
:10723800B5F9023008EE103AB8EEC88AB5F904304C
:10724800B8EEC99A28EE000A08EE903AA7EE890A25
:10725800F8EEE88AD4ED467AA7EEA80A0CF03CFCD2
:1072680094ED440AD4ED417A288028EE000AA7EE6E
:10727800890AD4ED477AA7EEA80A0CF02DFC94ED04
:10728800450AD4ED427A688028EE000AA7EE890AFA
:10729800D4ED487AA7EEA80A0CF01EFCA880BDEC35
:1072A800048B38BDB810002040000020104BDFEDE3
:1072B800117AD3F82421D3F82831928983F3100363
:1072C800D31A07EE103AB8EEC77A27EE277A07EEF8
:1072D800902AF8EEE77AC7EE277AFDEEE77A17EEFE
:1072E800900A6428A8BF642020EAE070C0B2704702
:1072F800B81000200000C842094BD3F824211378A5
:1073080044F6FB7103EB431300FB03135078C0EB07
:107318000030B3FBF0F39078B3FBF0F080B2704725
:10732800B810002010B50A4C94F82D3104EB430333
:107338000A22B3F83C1104F5A47089B2A4F84411E8
:1073480007F02EFC80B2FFF7D7FFA4F8D00110BDDC
:10735800B810002038B500240B4D6059254408F0BA
:107368004DF8696811B1094801F092FFA96811B197
:10737800074801F08DFF0748103408F03FF8B4F5CE
:10738800E87FE9D138BD00BF0C4E0108A86A0108A2
:10739800AE6A01083676010870B5054628460CF035
:1073A800D0F9064658B91A4B1A485A791A4B03EBC2
:1073B8008203BDE87040D3F8CC1101F069BF2846BC
:1073C800164932460CF0C6F960B91548154C08F054
:1073D80015F854F8041F19B1134801F059FFF8E7DC
:1073E800124805E00024124B53F8241021B9114823
:1073F800BDE8704008F002B8284632460CF0AAF9F9
:1074080001340028EFD1024B0B4D5C71C6E700BF79
:10741800801D0020B46A01080C4E0108C06A0108EA
:10742800C56A0108D84F0108D86A010836760108EC
:10743800DC4F0108EB69010874670108F0B585B0F5
:1074480004460CF07EF9082826D1621EE01D1F496B
:1074580012F8013F09681944497801F0030102292B
:1074680008BF203B82421370F1D1254604F108077A
:1074780015F8016B164831460CF055F920B128462D
:1074880031460CF050F910B1FEF78CFB1CE0BD4200
:10749800EED1204607F034F90E4807F0AFFF00237D
:1074A8000D4A1A4404A992F888210A440849595CEB
:1074B80002F80C1C0133082BF2D1002307488DF881
:1074C8000C3001A901F0E4FE05B0F0BD0C0100206C
:1074D8004E740108DC6A0108801D0020DA74010876
:1074E8002DE9F04105460CF02CF92F4B04469E6817
:1074F80088B92E4807F082FF2D4B53F8241041B16C
:107508000123A340334202D02A4801F0C1FE0134CE
:10751800F2E7294821E02846284922460CF01AF9C2
:1075280058B92748274C07F069FF54F8041F002969
:10753800EFD0204801F0ACFEF7E72B782D2B03BFE6
:10754800013504F1FF344FF001084FF00008002620
:10755800174B53F8267027B91B48BDE8F04107F0D0
:107568004DBF2846394622460CF0F4F8C8B9012028
:10757800B040020601D51548EFE78305FBD4B8F102
:10758800000F03D001F09EFF114802E001F0A2FFB6
:10759800104807F033FF39460F48BDE8F04101F0C5
:1075A80077BE0136D4E700BF801D0020E26A0108DB
:1075B80044500108D86A010836760108C06A0108F3
:1075C800EC6A010840500108EB690108F86A0108F3
:1075D800066B01080F6B0108D974010810B508483B
:1075E80007F00CFF074B00241C701C63064B1C7033
:1075F80007F062FC08F0B4F8044B1C6010BD00BF33
:10760800176B010890120020E12A0020882700202B
:1076180070B5064600240B4BE518AA8816420AD016
:10762800E158094801F034FE2846002107F073FEAE
:10763800064807F0E3FE143440F6CC339C42EAD106
:1076480070BD00BFBC580108436B010836760108BD
:1076580008B5084801F01CFE05F0C6FD05F0C6FC9B
:1076680018B9642007F0C4F9F8E70348BDE80840F2
:1076780001F00EBE4D6B01085A6B01082DE9FF4160
:107688000A48068885684488B0F80480C76805F009
:107698008DFCCDF800800290019731462A4623469A
:1076A800034801F0F5FD04B0BDE8F0810C000020AE
:1076B800626B0108F0B504788BB005460CB1002464
:1076C80036E04B4B19680E2303FB041101F590704B
:1076D800B1F92951B1F92521B1F92731009591F86E
:1076E8002C51019591F82D51029590F90B000390BA
:1076F80001F594713F4891F906100491214601342F
:1077080001F0C6FD082CDCD170E02D2B14D1072C1C
:107718001BDC28460CF06CF80AAB661C03EB44042F
:1077280024F8100C15F8013F303B092BFAD93446E0
:107738002B78002BE9D104E0A3F13002092A09D8FB
:10774800E5E7082CBDF8182009D00BB0BDE8F040DB
:10775800FEF728BA202BF8D101352646E7E7072A95
:10776800F3D8BDF81A00224BA0F2EE2189B240F2FC
:10777800DC55A9421B68E8D8BDF81C10A1F2EE241C
:10778800A4B2AC42E1D8BDF81E6004B237B2A74239
:10779800DBDB0DB2AF42D8DCA542D6DBBDF82470E6
:1077A80007F16404A4B2C82CCFD8BDF826E00FFABC
:1077B8008EF4112CC9DCBDF82050B42DC5D8BDF805
:1077C8002240B42CC1D812B24FF00E0C0CFB02337D
:1077D800A3F82501A3F82711A3F8296183F82C51F0
:1077E80083F82D4183F82B7183F82EE10BB0F0BD9F
:1077F800200F0020BF6B0108F0B504468FB020466B
:107808000BF09FFFC5B225BBAF48B04C07F0F6FDA3
:1078180094F8D21009B9AE4854E049B294F8D0208F
:1078280094F8D130009194F8D310019194F9D410C0
:10783800029194F9D510039194F8D6100491A548B3
:107848002946013501F024FD102D04F10704DFD18C
:10785800E1E72046A04905220BF07CFF0546B8B9B0
:1078680029469E4870220BF028FF9D4B1968284630
:107878000E2303FB001301300022082883F82F2170
:1078880083F8302183F8312183F83221F0D119E1CE
:107898002046944904220BF05DFF05462046002D42
:1078A8004AD120210BF03FFF002800F00B81461C35
:1078B80030460BF046FF2C4607468B4B53F82450B6
:1078C8002DB98A480FB0BDE8F04001F0E1BC304660
:1078D8002946FAB20BF03EFF01340028EDD17B4A6D
:1078E80002F170011646002382F8D63082F8D230B1
:1078F80082F8D13082F8D03007328A42F3D17C49FD
:1079080001EBC40191F89022934210DAD1F89472F5
:10791800C3EBC302B0183A4400F1D0011768C0F8AD
:10792800D0709088888092798A710133E7E7294678
:10793800704801F0ADFC96E06F4907220BF00AFF92
:1079480005462046002D4AD120210BF0ECFE0646C4
:107958000BF0F7FEC4B274BB684801F099FC2146ED
:107968006748013401F094FC0E2CF8D1584801F016
:107978008FFC00246348214601F08AFC0025584A00
:10798800614811680E2202FB04120123D2F82F214C
:107998005E49AB4013425E4B05F1010508BF19462D
:1079A80001F076FC0E2DEAD14948013401F070FC53
:1079B800082CDFD186E0304656490BF01DFF2C46D7
:1079C800002852D0022C55D00BF012FF06AB5149BB
:1079D80043F8240000200BF00FFF0134F0E74D4975
:1079E8000BF00AFF002460B1082C3ED00BF000FF1A
:1079F80006AB484943F8240000200BF0FDFE013493
:107A0800F1E7082C31D1069B0F2B2ED8DDF81CE0AE
:107A1800BEF1070F29D8089F0D2F26D8099E06F119
:107A28006402C82A21D80A9DFF2D1ED80B98642805
:107A38001BD80C99642918D8884216DA0D9C032C97
:107A480013D8224AC3EBC303134483F8D0E083F866
:107A5800D17083F8D26083F8D35083F8D40083F8C8
:107A6800D51083F8D6402C4CC9E60FB0BDE8F040DD
:107A7800FEF798B8069B072B20D807990D291DD823
:107A88000278722A0DD06E2A18D1154A12680E2073
:107A980000FB032301228A40D3F82F1121EA0202B6
:107AA80009E00F4A12680E2000FB032301228A40D6
:107AB800D3F82F110A43C3F82F2101E0FEF772F81B
:107AC8000D4C9CE60FB0F0BDE76B0108801D00204F
:107AD80036760108126C0108BB690108501E0020A7
:107AE800200F0020E6690108DC4F0108EB69010856
:107AF8000C4E0108FA690108DF6B0108B26A010837
:107B08002E6C010895730108336C01089E780108F2
:107B18003E790108376C0108746701082DE9F743BD
:107B2800047805468CB9324D95F8A312B5F8A02211
:107B380095F8A2322F4800912146013401F0A8FBA4
:107B4800102C05F10405EFD14EE00BF051FE0F2883
:107B5800044636DC284620210BF0E5FD264EE4B22B
:107B6800D6F83480451CA400002728460BF040FEB8
:107B78005FFA87F9B9F1010F83B208D0B9F1020FA2
:107B88000BD0B3F5B47F24D2726B13530AE0FF2BEA
:107B98001FD8736B2344987004E0FF2B19D8736BBC
:107BA8002344D87028462C210BF0BDFD054608B1AA
:107BB800013502E0B9F1020F0BD10137032FD4D1FF
:107BC80012E00E4800210F2203B0BDE8F043FDF794
:107BD80066BF08EB0400002104220BF06EFD03B021
:107BE800BDE8F043FDF7DEBF03B0BDE8F08300BF9A
:107BF800801D0020396C010890120020946901084A
:107C08002DE9F04304788FB00546002C59D17C4B00
:107C18000021142209A807AED3F838800BF04DFDD7
:107C28000722304600210BF048FD05A80023A700D5
:107C3800059308EB070583801A467249B5F802E0F8
:107C480031F813C01CEA0E0F0AD00DF1380C0E31B2
:107C580002F1010E6244595C02F81C1C5FFA8EF2B4
:107C68000133072BE9D100210B46674AB5F802E03A
:107C780011F802C01CEA0E0F0AD00DF1380C0632BA
:107C880003F1010E63448A5C03F8242C5FFA8EF337
:107C980001310629E9D118F807305C498DE841001F
:107CA8006A78029209A81A0903F00F0301F0DBFAB7
:107CB8002146574809AA013401F0EAFA202CA6D136
:107CC8009BE00BF095FD1F28044600F389802846A9
:107CD8002021E4B20BF027FD1F2C02D9FDF762FF2B
:107CE8008BE0474B9B6B03EB8404451C002120462B
:107CF80004220BF0E2FC0027464B09AE3046002177
:107D08000A2217F803905FFA87F80BF0D6FC0023D5
:107D180015F8012B32B10A2B04D04A4502D0F2548F
:107D28000133F5E74A4561D108F1FF33032B09D840
:107D3800DFE803F0100502420DF1230037E00DF1F2
:107D480023011FE030460BF053FD2378C0B243EA0D
:107D5800001006E030460BF04BFD237800F00F00D2
:107D68001843207034E00133062B0BD02A4800F268
:107D78007B369E5D9642F6D1034493F8752363885B
:107D88001343638011F8012F12B30023EEE7013388
:107D9800072B0CD0204A02F26E369E5D8E42F6D139
:107DA80002EB4303B3F8602363881343638010F83E
:107DB800011F69B10023EDE730460BF019FD0F28CC
:107DC80004DC30460BF014FD607001E000236370A2
:107DD8000137052F90D1012400F032FE6CB97DE700
:107DE8000E4800211F22FDF75AFE06E0204600211A
:107DF80004220BF062FC0024EEE70FB0BDE8F0832C
:107E0800901200206C510108815101084D6C010845
:107E18005C6C01088D5101080C4E01089469010839
:107E28002DE9F0412DED048BB1498AB004460BF0E1
:107E38004DFCB049002820460CBF012607260BF050
:107E480045FCAD490028204608BF02260BF03EFC41
:107E5800002808BF0426F10740F1F080A748A84C85
:107E680007F0CCFA002007F0D1F8A64807F0C6FAC8
:107E7800A54807F0C3FA6279A44BA54803EB82032F
:107E88002546D3F8CC1101F003FAA24801F000FA14
:107E98004FF00008274695ED048AB5EE408AF1EECA
:107EA80010FA04D19C4801F0F3F9002570E09B48D2
:107EB800D5ED059A95ED069AD5ED078A414601F06C
:107EC800E7F9B5EEC08AF1EE10FA02D5202007F0E6
:107ED8008DFAB0EE480A06A801F05AF80146904813
:107EE80001F0D6F9F5EEC09AF1EE10FA02D520208D
:107EF80007F07CFAB0EE690A06A801F049F80146D5
:107F0800874801F0C5F9B5EEC09AF1EE10FA02D52E
:107F1800202007F06BFAB0EE490A06A801F038F8FD
:107F280001467F4801F0B4F9F5EEC08AF1EE10FA87
:107F380002D5202007F05AFAB0EE680A06A801F028
:107F480027F808F101080146764801F0A1F9B8F1CF
:107F58000C0F05F110059ED1A4E749B294F8D02082
:107F680094F8D130009194F8D310019194F9D41079
:107F7800029194F9D510039194F8D61004916A48A7
:107F88002946013501F084F9102D04F1070403D0C6
:107F980094F8D2100029E0D16448654C07F02EFA15
:107FA800D7F8088054F8041F19B1624801F070F935
:107FB800F8E70D46604B53F8254054B10123AB4018
:107FC80013EA080F03D05D48214601F061F9013535
:107FD800F0E75B4807F012FA21467B180AAA93F8E3
:107FE80088311344574A8A5C03F8102C0131082958
:107FF800F3D1002306A954488DF8203001F048F940
:10800800524807F0FBF95248FEF726FA514807F0A4
:10801800F5F94F48FFF7F4FD4F4807F0EFF94C48E2
:10802800FFF77CFD4D4801F033F94020FFF7F0FAE7
:108038004B4807F0E3F94648FDF7DEFFB20739D5AC
:10804800484807F0DBF9484807F0D8F9404807F0F6
:108058001DF8464807F0D2F93D48FDF72DFD444884
:1080680007F0CCF93A48FDF719FF424801F010F93A
:108078003748FDF79DFD404807F0C0F93448FFF741
:1080880019FB00270E257D4300243C4AD26B2A4465
:108098000123D2F80A20A34013421ED101340E2C2A
:1080A800F3D10137082FEDD12C4801F0F1F88020E9
:1080B800FFF7AEFA730716D5314807F09FF9314834
:1080C80007F09CF9224806F0BBFF244801F0E0F8CD
:1080D8004FF48070FFF79CFA05E0394622462A489B
:1080E80001F0D6F8DAE70AB0BDEC048BBDE8F08100
:1080F800686C0108B77001086F6C0108756C01089D
:10810800801D0020836C0108956C01080C4E010845
:10811800A16C0108AC6C0108B96C0108C66C0108B7
:10812800B16A0108DA740108DE6C0108CE6C010836
:1081380040500108FD6C0108445001080B6D01080E
:10814800186D01084E740108246D01082D6D010891
:10815800746701083C6D0108486D0108367601080E
:10816800566D0108636D0108766D0108846D01087C
:108178008E6D01089D6D0108AB6D010890120020FD
:10818800B76D0108C86D0108DA6D0108022803D02F
:10819800431E584258417047064B1B681B7823B151
:1081A800054B1868C0F3C0407047044B1878C0F3FB
:1081B800800070471C0D0020E40E0020E02A0020FB
:1081C80008B507480BF0BDFAC0B21428044B04D810
:1081D800421C20211954D0B2F7E700221A5408BDD6
:1081E800D0120020674B73B51878674DFFF7CEFFA4
:1081F8002B788342044620D0C8B1644B1B68E3B196
:1082080093F9000002230093614B1B685B780033ED
:1082180018BF0123019304214FF416530022FEF7DF
:1082280007F85C4B186040B101232B7005E0594EEC
:108238003068FDF7E9FF34602C70574B574D1878BC
:10824800FFF7A4FF2B788342044618D088B1544B1B
:108258001B68A3B10022012493F9000000944FF495
:10826800964301920821FDF7E3FF4E4B186028B9A9
:1082780005E04C4E3068FDF7C7FF34602C704A4B60
:108288004A4D1878FFF782FF2B78834204462E4622
:1082980042D0002837D0464B1A68002A3CD0D37900
:1082A80092F90000434C002B08BF022302220092DF
:1082B800002254F8233001921021FDF7B9FF3E4BFC
:1082C8000546186040B33D4C94F84A30022B0BD059
:1082D80094F89620022A01D14C3405E023B1002AF3
:1082E80004F14C0418BF0024354B1C6044B12046EF
:1082F80000214C220BF0E1F90223256084F84A3072
:108308000123337008E02C4E306806F07FFF306898
:10831800FDF77AFF34602C702A4B2B4D1878FFF745
:1083280035FF2B788342044629D000B3274B1B68BE
:108338002BB3274A93F9000012685278002A0CBF21
:10834800082209220323009301924FF4614320215C
:108358000022FDF76DFF1F4B186080B11E4A0123F4
:1083680013702B701D4B1A681D4B1A6007E0194ECD
:108378003068FDF749FF184B34601C702C7002B050
:1083880070BD00BF240D002029070020200D00200B
:108398003407002030130020250D00203807002066
:1083A8008C0700207C070020300D00209207002059
:1083B8002C0D00205C56010894070020E81C0020C2
:1083C800980700203C0D0020A0070020380D002051
:1083D800340D0020A4070020A8070020902A0020C0
:1083E800AC070020642928BF6421F8B510FB01F50B
:1083F8006424064695FBF4F40027E4B2FBB2A342DA
:1084080004D29F2004F0ADFF0137F7E7B4420BD246
:10841800C4EB84101421C4EB800095FBF1F5663D94
:108428002844C0B204F09DFF0134E4B2B44201D242
:108438009A20F7E7F8BD2DE9F743B74C06F0BCFAE8
:10844800A369C31A002BC0F26B8200F5433303F50E
:10845800A073A361B14B1E78237FC6F38006F31A7D
:1084680018BF012326774EB1002B00F05982AC4B80
:108478005A789A7001225A701A7025E0A84A2BB1CE
:10848800D37843F00203D37093785370D57805F00E
:10849800020101F0FF0339B9A1498968411A00298D
:1084A80003DB05F0010300E0012303F001079C4909
:1084B80017704BB1ED0707D50B799A4A013303F0D2
:1084C80003030B71D35C4B70954DDFF8B8822B78A2
:1084D8007BB3EB7823F00203EB70934B0344AE209D
:1084E800AB6005F051FD08B104F0CCFE88F800003F
:1084F800002800F01582B02005F046FD402005F068
:1085080043FD002005F040FD102005F03DFD4FF42F
:108518008067013F0020BFB205F031FD002FF8D180
:10852800384604F042FF6A78804B53F8220004F082
:1085380033FF98F80030002B00F0F2816B78052BA0
:1085480000F2AD81DFE813F00600AB0117007700F9
:1085580050016B017649774A774B6F4800F083FEEC
:10856800012004F022FF6C4804F016FF022004F0FA
:108578001CFF724891E1724F3B68990735D5DFF8C7
:108588000882DFF80892B8F8001063480A23B1FBA4
:10859800F3F203FB121399F80010009192B26949A3
:1085A8009BB200F060FEFFF70BFE012004F0FDFE19
:1085B800594804F0F1FE644B99F800201868B8F89F
:1085C8000030057905FB123164234B43C1784D1BFC
:1085D80055430220B3FBF5F5EDB204F0E6FE29465B
:1085E8001520FFF7FFFE032500E001253B681A056B
:1085F80040F15581554B56491F680968009164231D
:10860800544997FBF3F2444803FB127300F02BFE26
:10861800FFF7D6FD284604F0C8FE3F4804F0BCFE2C
:10862800FEF744FE0746681C04F0BFFE15203946D5
:10863800FFF7D8FE33E1012004F0B7FE464804F006
:10864800ABFE464B1A6812F0020F1F4617D0444A79
:108658003148B2F90210B2F900300091B2F90420A1
:1086680040490192404A00F0FEFDFFF7A9FD0220B3
:1086780004F09BFE284804F08FFE032500E0022545
:108688003B68DB0718D5394A2348B2F90210B2F91A
:1086980000300091B2F9042032490192344A00F0C6
:1086A800E2FDFFF78DFD284604F07FFE1A486F1C97
:1086B80004F072FEFFB23D462E4A2A49B2F9003054
:1086C800B2F9022000922C4A1348B2F90020019214
:1086D8002A4A2B4F00F0C7FDFFF772FD284604F029
:1086E80064FE0D4804F058FE97ED000A0A4800F0B1
:1086F8004FFC09480BF025F805F101085FFA88F8E6
:10870800C0B2092844D8431CDBB220222254E21804
:10871800002151701846F4E7D0120020E02A00200A
:10872800440E0020F0720108404B4C0050520108E2
:10873800F4720108FD7201083B6501080473010821
:10874800842A00200C730108DC110020440F00204B
:10875800E01100202473010839730108DC0E0020A1
:10876800040F00204F7301085E7301080A0F0020F0
:10877800627301083C0F0020400F00206673010857
:108788004C080020C9090020881200200801002098
:1087980097ED010A204400F0FBFBFFF711FD40466E
:1087A80004F003FE604804F0F7FD97ED020A5E4806
:1087B80000F0EEFB5C480AF0C4FF0235EDB2C0B22F
:1087C800092808D8431CDBB220222254E2180021D1
:1087D80051701846F4E79FED550A204400F0D8FB85
:1087E800FFF7EEFC284655E00025514F3B78AB4299
:1087F80055D90E2D53D06808013004F0D6FD28460F
:1088080005F0AAFE3B78AB4206D9202004F0A9FD6A
:10881800681CC0B205F0A0FE0235EDB2E5E7454D93
:10882800454995F8A827404800F01DFD012004F0AF
:10883800BCFD3D4804F0B0FD404B41491F783A4823
:108848003A4600F010FD022004F0AFFD364804F06F
:10885800A3FD0C2303FB07553A4995F8AB2795F878
:10886800AA37314800F0FFFCFFF7AAFC032004F008
:108878009CFD2D4804F090FD95F8B01795F8AE27AB
:1088880095F8AF37284800912F4900F0ECFCFFF726
:1088980097FC042004F089FD234804F07DFD002E98
:1088A8003ED12A4B93F82030052B9CBF284A9B18B1
:1088B8004FF0B00094BF1D7E3F2505F065FB0C20EE
:1088C80005F062FB162005F05FFB284604F049FD21
:1088D800B02005F059FB022005F056FB172005F0E3
:1088E80053FB1C4B1B78002B1B4B1B7814BF7220AF
:1088F8002120002B18BF522004F033FDB02005F0D2
:1089080043FB082005F040FB172005F03DFB657F81
:10891800124B585D013505F0030504F022FD65771B
:1089280003B0BDE8F08300BFD012002000000000B3
:1089380060250020801D00206A730108642700203C
:10894800767301088773010898730108942A002038
:10895800505201086C0D00201A0E0020AA7301085D
:1089680010B54B88DC0641BF2F4B14791B6853F8B0
:10897800244044BF2D4B43F820404B889B0641BF01
:10898800294B54791B6853F8244044BF274B43F8BC
:1089980020404B881C070ED5254B0C781B78B3EB71
:1089A800141FA1BF204BD4781B6853F82440A4BFE0
:1089B8001E4B43F820404B889B070ED51D4B0C7867
:1089C8001B78B3EB141FDFBF174B54781B6853F8A1
:1089D8002440DCBF154B43F820404B88DC070FD5FB
:1089E800154C0B78247803F00F03A342DFBF0E4B1E
:1089F80014781B6853F82440DCBF0C4B43F8204024
:108A08004B885B070FD50B780C49097803F00F03E7
:108A18008B42A1BF044B92781B6853F82220A4BF55
:108A2800024B43F8202010BDC4120020B4070020D8
:108A38004B08002049080020480800204A08002068
:108A4800254A264826490023F0B5156803708B7718
:108A58001C461A462E1976884EB92F5D3FB9037009
:108A680000238A77CB7707781C461A460CE0360530
:108A780048BF013204F1040403F1010348BFD2B234
:108A8800802CDBB2E6D1EAE7E0B2B8420CD215F8A6
:108A9800240006099E4200F00F00A8BF731C9042F4
:108AA800A8BF421C0134EFE781F82020CB77C2F33E
:108AB800470102F001020A444C1E0A490A480A709A
:108AC800C3F3470203F00103134404700749501E1F
:108AD800074A08701370F0BDC81200204008002033
:108AE800D01200204A080020480800204B08002027
:108AF800490800202DE9FF47704B714933F91030C0
:108B080004462BB902280CD06E4B1B88980708D056
:108B18006D4B002223F814206C4B1B8821F814306D
:108B2800C8E031F814301BB9694A02EB8402536279
:108B380001339BB221F814301BB2002B18DD022C34
:108B4800634A644809D1D66AB0F90450202095FBDD
:108B5800F0F505FB0060D0620AE002EB840230F910
:108B68001450566A802095FBF0F505FB00605062B2
:108B7800594F386890F85E20934240F09B80544AE1
:108B8800DFF8448102EB840200EB040E022C556AE4
:108B980095FBF3F39EF85750536208BF5E424FF0BF
:108BA800000221F8142007BFB6B214219EB20A2190
:108BB800002D7DD0002E7BD038F81420002A77D0E5
:108BC8000FFA86F90FFA82FCE14571D089EAE97259
:108BD8008CEAEC7AA2EBE972AAEBEC7ACAEB020215
:108BE800B9F1000F12B209B2DFF8F89003DDBCF159
:108BF800000F03DC20E0BCF1000F1DDA8A420BDD18
:108C0800022C90F85A2002D102F580720EE039F851
:108C1800141040320A4419E049428A4218DA022CF8
:108C280011D190F85A20C2F57F42C032B9F8041029
:108C38000A44A9F804200BE0002AB8BF52428A422D
:108C480006DD022C04D039F81420203A29F8142023
:108C580039F914209EF8549092114A4503DBAA4230
:108C6800A8BF2A4691461D4A126812031FFA89F5C1
:108C780008D5142001A98DF804400293ADF80C50D2
:108C880001F01EF8164B1B7873B12AB207EE902A32
:108C9800F8EEE77AB2EE047AC7EE877A3B6803EB20
:108CA8008403C3ED087A03E03B68234483F801900A
:108CB80028F8146004B0BDE8F08700BF80190020D0
:108CC800EC010020E00E0020E6010020DE0100207B
:108CD800D01200200A0F0020D8010020842A00208A
:108CE800DC010020E001002030B50B4C0B4D227850
:108CF8002B789A4285B00CD0684602A904F03AF95C
:108D08000123684602A9022204F0A4F900232B706B
:108D1800237005B030BD00BF321B0020311B00207E
:108D2800F0B50124B0FBF4F58D4201D34C43F9E7CB
:108D38000026D4B1B0FBF4F504FB1500B4FBF1F444
:108D48001EB9002D01DC002CF3D1092D03F1010E11
:108D5800EFB204DD002A14BF3725572500E030257F
:108D68003D441D7001367346E3E71C70F0BDF0B555
:108D78000124B0FBF4F58D4201D34C43F9E70026FA
:108D8800D4B1B0FBF4F504FB1500B4FBF1F41EB943
:108D9800002D01DC002CF3D1092D03F1010EEFB2F7
:108DA80004DD002A14BF3725572500E030253D444F
:108DB8001D7001367346E3E71C70F0BD03685A1C4A
:108DC8000260197070472DE9F843089E002B07468A
:108DD8008846144614BF4FF030094FF02009334637
:108DE80013F8012B0AB9254603E0002CFBDD013CF2
:108DF800F6E7002D04DD38464946C047013DF8E74F
:108E080024EAE4743546A01B284415F8011B11B167
:108E18003846C047F7E7BDE8F883024B186805F005
:108E2800BCBE00BFC00E002090ED017A07EE901A7C
:108E3800B5EE407AF1EE10FA01BFF8EEE77A9FED51
:108E48000E7A67EE877AB7EE007A04BFC7EE277A04
:108E5800C0ED017A90ED017AD0ED007A30EE877A94
:108E680030EE670AC0EE870AE0EE807AB0EE670A55
:108E7800C0ED007A704700BFDB0FC94010B502781B
:108E8800202A034600F10100F9D0092AF7D02D2A3B
:108E980003D10346BFEE000A04E02B2A08BF0346AD
:108EA800B7EE000ADFED387A1A46134612F8010BBE
:108EB800A0F13001CCB2092C0AD807EE101AB8EE8E
:108EC800C77AF2EE046AA7EEA67AF0EE477AECE7E4
:108ED8002E2816D1F2EE046A1146B0EE666A0B46E9
:108EE80011F8012B303AD0B209280AD807EE102A17
:108EF800B8EEC77A87EE267A66EE866A77EE877AC4
:108F0800EDE71A7802F0DF02452A35D15A782D2A82
:108F180002D10233012004E02B2A14BF01330233AB
:108F28000020013B002213F8011F3039CCB2092C74
:108F380003D80A2404FB0212F5E7B2F59A7F28BF8A
:108F48004FF49A721346B7EE007A072B05D9DFED76
:108F58000F6A083B27EE267AF7E702F007032BB1E2
:108F6800F2EE046A27EE267A013BF8E7F0EE476A4C
:108F780020B1C7EE877A03E0F7EE006A67EEA67ABB
:108F880020EE270A10BD00BF0000000020BCBE4C28
:108F980030B52DED028B87B0B0EE408A0C2200214F
:108FA800054603A80AF089FBB5EEC08ADFED2A7AE8
:108FB800F1EE10FACCBF38EE278A38EE678ADFED7B
:108FC800277A28EE278A6946FDEEC87A17EE904A76
:108FD80084EAE470A0EBE47005F0E4FA002CACBF7E
:108FE80020232D2368468DF80C300AF0AAFB0128AF
:108FF80007D130238DF80D308DF80E308DF80F30F5
:109008000CE0022805D130238DF80D308DF80E3094
:1090180004E0032804BF30238DF80D30694603A807
:109028000AF072FB03A80AF08CFB0338C4B222468C
:1090380003A928460AF0B2FB00232B552846084905
:109048000AF062FB03AB284619190AF05DFB2846B3
:1090580007B0BDEC028B30BD6F12033A00007A44B2
:10906800DC73010870B5064615460846B6FBF2F4EF
:1090780014B12046FFF7F6FF05FB1464024B1B5D95
:1090880000F8013B70BD00BFDE7301082DE9F04F09
:10909800814689B08A4616461C4600253178002943
:1090A80000F0DD80252902D00136484675E0727847
:1090B800302A08BFB278A2F1300319BFB71C4FF0AD
:1090C800000BF71C4FF0010B092B4FF0000819D8C3
:1090D800A2F13003D9B2092905D80A2202FB0838BF
:1090E80017F8012BF4E7A2F16103052B02D8A2F1CE
:1090F800570305E0A2F14103052B03D8A2F137037A
:109108000A2BEADD6C2A31D13A78642A07F1010684
:1091180000F083800BD8252A3DD003D8002A00F020
:109128009E80BBE7582A0CD0632A19D0B6E7732A69
:1091380022D002D86E2A37D0B0E7752A5CD0782AB8
:10914800ACD1271D2068A2F1580462424FF01001EB
:10915800624155E02CD9582A32D0632A2AD13E469A
:1091680048462178271DD04701350FE0642A64D08E
:109178000ED9732A14D13E462368009348465146B7
:1091880042460023FFF71FFE271D05443C4685E79E
:10919800252ADFD13E4648462521D04701357DE7BF
:1091A8000AD86E2A06D13E46236804341D6075E746
:1091B800002A54D03E4671E7752A26D0782AF9D17C
:1091C800A2F1580304F1040C5A422068CDF80CC0EF
:1091D8004FF010015A4105ABFFF7A2FDDDF80CC0B6
:1091E8003E46644605AB00934846514642465B46B8
:1091F800FFF7E9FD054451E72068271D0A210022F1
:1092080005ABFFF7B4FD3C46ECE704F1040CCDF8E0
:109218000CC020680A210022DDE72068002804F13C
:10922800040708DA2D238DF8143040420DF1150398
:109238000A210022E5E705ABFAE72068002804F1D7
:10924800040C0ADA2D238DF8143040420DF1150371
:10925800CDF80CC00A210022BEE705ABF8E7284686
:1092680009B0BDE8F08F0EB40FB505AB019053F807
:10927800042B0649039301A8FFF708FF019B00226E
:109288001A7004B05DF804EB03B07047C58D000890
:109298000FB413B50B4904AB08680B4953F8042BFA
:1092A80009680193FFF7F2FE0446084B186805F0B9
:1092B8006BFC0028F9D0204602B0BDE8104004B08D
:1092C800704700BF5C08002058080020C00E00202E
:1092D800B0EEE06AF0EEC05AB4EEE56AF1EE10FACC
:1092E800D4BFF0EE656AF0EE466AF5EE406AF1EE3C
:1092F80010FA0BD0B4EEE56AF1EE10FA54BFF0EEB6
:10930800657AF0EE467AC7EEA66A01E0DFED1F6ADD
:10931800DFED1F7A9FED1F7A9FED1F5AA6EEA77A01
:10932800DFED1E7AE7EE267A9FED1D7AA7EEA67A84
:10933800DFED1C7AE7EE267AF4EEC65AB1EE677ACC
:10934800DFED197AA6EEA75AF7EE007AE5EE267A4F
:10935800F1EE10FAC7EE277AC8BF9FED147AF5EE42
:10936800C00AC8BF77EE677AF1EE10FA48BF9FEDE2
:10937800107AB5EEC00A48BF77EE677AF1EE10FAB8
:1093880048BFF1EE677AB0EE670A70470000000048
:1093980039094E3DE3B59EBE69A2163E88FA16BE4F
:1093A80045FE7FBFA7DFA8B499FB243FDB0FC93F69
:1093B800DB0F4940FDEEC07A17EE903A2033402B80
:1093C80043D8DFED237AB4EEE70AF1EE10FA04DDB4
:1093D800DFED207A30EE670AF3E7DFED1F7AB4EEAF
:1093E800E70AF1EE10FA04D5DFED1A7A30EE270A13
:1093F800F3E7DFED1A7AB4EEE70AF1EE10FA04DDCE
:1094080030EE670A37EEC00A0AE09FED157AB4EE2F
:10941800C70AF1EE10FA44BF30EE270A37EE400AC9
:1094280060EE007ADFED0F6A9FED0F7AA7EEA67A5D
:10943800DFED0E6AE7EE876A9FED0D7AA7EEA67A52
:1094480020EE276AA6EE070A70479FED060A7047C6
:10945800DB0F4940DB0FC940DB0F49C0DB0FC93FB9
:10946800DB0FC9BF0000000092E741B99730083C04
:1094780015A82ABEDFED027A30EE270A9AE700BF68
:10948800DB0FC93F064B1A8822EA0000904210B54C
:1094980018801C4602D0012005F016FB208810BD5C
:1094A800E00E0020064B1A881043904210B5188031
:1094B8001C4602D0012005F007FB208810BD00BF24
:1094C800E00E0020024A936823EA0000906070478B
:1094D800801D0020024A936818439060704700BFBF
:1094E800801D002008B5104B1A780023D9B291428C
:1094F80007D20E4951F8231009680020086001338B
:10950800F4E7322005F074FA094B1B685A0309D5B1
:10951800084B9B685B0305D440F2DC50BDE808406B
:1095280005F066BA08BD00BF18260020E82500200F
:10953800842A0020801D00202DE9F34106F0A4FFB5
:10954800454A6F23137040F2DC735380BE231371B6
:10955800EF2382F8D837002382F8D9371946164600
:10956800F25C0133514040F2DC729342F8D13A4B3D
:1095780083F8D917394B1A69120604D5384A5A6044
:1095880002F188325A6004270020013F17F0FF07D4
:1095980050D0324B3422DA60002444B1002356F80C
:1095A8000480019305F09AF80428EED117E005F03D
:1095B80095F80428E9D1294D2B6943F002032B6162
:1095C800284B6B612B6943F040032B6105F086F84B
:1095D8002B69042823F002032B61DFD0D5E71F4D48
:1095E8002B6943F001032B6104F1006303F57C331D
:1095F8001FFA88F21A8005F071F8042810D11A4B66
:1096080023440193019B4FEA1848A3F8008005F012
:1096180065F82B69042823F001032B6105D0B4E712
:109628002B6923F001032B61AFE7043440F2DC73AC
:109638009C42B2D1094A1369042843F0800313619C
:1096480002D103F0C2FE10B9052005F055FA06F064
:1096580007FF02B0BDE8F081801D00200020024015
:109668002301674500F0030802F0030810B50E4C0B
:10967800206805F00BF92068047A002202FB02F347
:10968800193B634303F6C4135343192193FBF1F3C6
:10969800064921F812300132072AEFD10449BDE802
:1096A8001040FCF7A9BF00BF4C0F0020900E00200F
:1096B800C01E00202DE9F04103F087FE10B90420F8
:1096C80005F01AFAA74CA84D06F0DEFEA74940F2AD
:1096D800DC72204609F0E6FF94F8A837022B84BF15
:1096E800002384F8A83794F8A8274FF4CC7101FB1D
:1096F80002F303F5387023442044286093F84003AC
:10970800022801FB024284BF002083F8400392F83C
:109718004033974A13700C2202FB0343954A03F225
:10972800AA731360A26846F2090313401BB94FF4E9
:109738000050FFF7CFFEA368D80703D54FF40050B9
:10974800FFF7C0FEA368590409D50820FFF7BAFE41
:109758004FF40050FFF7B6FE0120FFF7B3FEA368F1
:109768001A0706D54FF40050FFF7ACFE0120FFF7AB
:10977800A9FEA3689B0402D54020FFF7A3FE01229F
:1097880084F8112294F8DE21764B2AB193F8E2216D
:1097980012B1002283F8E221774B784E1E604FF019
:1097A800000C674604EB0C03B3F8F2E14FEA5E01E4
:1097B80001F077314FEA9E0303F03333C1EB0E001B
:1097C800C11A4FEADE0303F01133CB1A03EB23135C
:1097D8001EF0010803F00F324FF0FF0392FBF3F382
:1097E800C3EB032318BF0137A2EB030318BFFFB273
:1097F800012B0ADD022B40F0B280B8F1000F00F017
:10980800AE801EF0BC0F00F0AA800CF1080CBCF171
:10981800200FC7D1013F012F00F2A180FFF726FFDB
:10982800302200215648574F09F047FF564BD5F8CC
:1098380000801F60554B002108F18500C3F80080A7
:1098480005F064F8524B80F001001870514B07F195
:1098580028021A60504B07F1D0021A6098F80000ED
:1098680002F03AFE4D4B94F8D601DFED4D6A07F150
:1098780096021A6064214B4BC82211FB00225A60E1
:1098880000229A60DA601A615A619A61DA6183F893
:10989800202083F82120444B07F12E021A602A6801
:1098A800424B92ED1B7A02F225111960404B02F2ED
:1098B800951119603F4B07F1080119603E4B1F6075
:1098C8003E4B07F1A201196067EE266A3C4B07F18F
:1098D800AC01B6EE007A196087EE267A39490E6037
:1098E800B4F86411181D07EE901AB4F86611F8EE72
:1098F800677AC3ED027A07EE901A92F86810197128
:1099080092F88410597194F8E1111974F8EE677A95
:10991800B2F82211C3ED037A07EE901A2A49F8EE3D
:10992800E77A08605A6183ED077A9FED287A1A6210
:10993800C7EE277A02F1700199612549DF62BDE817
:10994800F0419FED247A67EE877AC1ED007A02F143
:10995800740102F21D1259629A6206F081BD04F088
:109968008FFE5BE7801D0020200F002000F0030819
:10997800642700204C0F0020802A0020081F0020A8
:10998800500E0020C01E0020840E0020880E0020EB
:10999800050000200C1A00201C0D0020A82900201A
:1099A800DB0F4940942A0020741A0020CC120020B2
:1099B800E4020020E4260020E8260020F801002028
:1099C80000130020BC020020F01A002000006144AF
:1099D800F40100204C3D0F4408B5FFF7ADFDFFF73B
:1099E80069FE0120BDE8084005F06EB8284B294AF9
:1099F8001B68126810B51A60274A116859605168C7
:109A08009268DA60254A996011681961516892680C
:109A18009A61234A59611168D961516892685A62FA
:109A2800204A196211881985518859859188D288E8
:109A3800DA851D4A99851188198651885986928830
:109A48009A861A4A1188D9865188198719469288A0
:109A580021F83A2F164A10780022824206DA154C6D
:109A680034F8124021F8024F0132F6E7124A128800
:109A7800A3F86420114A1288A3F86620104A1288B5
:109A8800A3F868200F4A5289A3F85E2010BD00BFD2
:109A9800D4270020C42A0020D0190020DC19002077
:109AA800E8190020801900200A0F0020040F002068
:109AB80018260020240F0020FC110020B40E0020DE
:109AC800420F0020100F0020A0F17D03012B70B57C
:109AD80004460D460A4E05D830687D2105F05DF82C
:109AE80084F020043068214605F057F835B12B88FA
:109AF8001C4404EB142404F0FF042C8070BD00BF48
:109B0800A407002010B50A4C5E280146206805D13C
:109B18005D2105F042F820683E2105E05D2903D16A
:109B280005F03BF820683D21BDE8104005F035B848
:109B3800301300202DE9F8430E4B93E880030546C7
:109B48000E460024B44213DA7B1933F9140008EBEB
:109B5800050333F9142009EB050333F914301344D2
:109B6800022293FBF2F3C01A04F041F80134E9E74A
:109B7800BDE8F883D427002010B5104B93F8D037F0
:109B8800012B014612D10E4A0E4C1078431CDBB251
:109B980013701B0644BF00231370215403F016FAF8
:109BA8003F2809D9BDE8104003F0FCBA064BBDE8D0
:109BB8001040186804F0F1BF10BD00BF801D0020E0
:109BC800311B0020331B0020B82700207FB5264C0E
:109BD800264E274D2749284A284B20B12848008877
:109BE800B0F5805F32D230881F4E91F8201012787D
:109BF800ADF8040028788DF80600351D8DF807109B
:109C08008DF808201B788DF8093001A8294606220E
:109C180009F038FD30B30198BDF808307060AB80AA
:109C28005320FFF7A9FFA08803F0D1FFA07903F024
:109C3800CEFFE3790193237A029301A8637A039311
:109C480003F034FF0E4B00221A800BE03088A0800E
:109C580091F82010287812781B78A071E17122728F
:109C68006372DDE704B070BD30130020E00E002001
:109C7800EC1A0020942A00206C0D00201A0E0020F7
:109C88004C2900200A4A138801331380094A1368B3
:109C980001331360084A138801339BB2202B01BF9C
:109CA80000231380054A138808BF013313807047C7
:109CB8004C29002030290020342900203629002092
:109CC80038B5294B1B78083B012B05460C464AD86A
:109CD8004520FFF751FF2846FFF74EFF0E2D33D0E2
:109CE80003D83DB10D2D07D038BD142D20D0FF2D40
:109CF80032D038BD20682BE0637820789BB180F0A3
:109D08008000FFF739FFA568E8B2FFF735FFC5F314
:109D18000720FFF731FFC5F30740FFF72DFF280E97
:109D2800FFF72AFF04E0FFF727FF606803F05FFFF3
:109D38002078FFF721FF606803F059FF2489E0B21B
:109D4800FFF71AFF200A0BE0206803F040FF606865
:109D5800BDE8384003F03BBF044803F04CFF002047
:109D6800BDE8384008E738BDB6270020037401086D
:109D78002DE9F04FB44BB54F1A8889B01C46002A1C
:109D880040F09680B7F8CE07B14D42F20103C41AED
:109D980060426041FFF71AFFFFF728FE2C68492050
:109DA800FFF7EAFEAB4B2646186803F010FF56F89B
:109DB800040B03F00CFF304604F015FC04F110000E
:109DC80004F011FC04F11C094FF01008A24E012305
:109DD800326803FA08F3134203D0D9F8000003F0FD
:109DE80006FF08F10108B8F1130F09F10409EDD1D4
:109DF80004F1280004F0E7FBB7F84031B4F92E006D
:109E0800C01A03F0E4FE3368D90408D5934BB4F8BC
:109E180064001B88181AC0F30D0003F0D8FE3368DD
:109E28009A0403D5B4F8660003F0D1FE33681B0426
:109E380003D5B4F8680003F0CAFE04F13000A04668
:109E480004F0C1FB04F1360004F0BDFBB7F8403163
:109E580038F93C0FC01A03F0BAFE0127804B1B7873
:109E68009F4208DA38F9020FB4F93C30C01A03F0FF
:109E7800BEFE0137F2E73368980505D5B4F95E00F0
:109E8800A0F2DC5003F0B3FE2A6876486A60AA6044
:109E9800121A9110744A4A43531C032293FBF2F29C
:109EA80002EB42029A1A6C2303FB02032B6070E157
:109EB8006E4B6F4A1B6811688B4206D008A90020B8
:109EC80041F8203D1360FFF7FBFE97F8CE17238873
:109ED80097F8CF070B44013BB3FBF0F200FB1233BA
:109EE8008B4280F056815A4E0120FFF76FFEFFF734
:109EF8007DFD5020D6F800807768FFF73DFEB268F8
:109F0800336810681B68726803441068A3EB40004C
:109F180003F06DFE7A68D8F804309B1A0093BA688B
:109F2800D8F808309B1A0193FA68D8F80C306846BC
:109F38009B1A029304F057FB3A69D8F810309B1A21
:109F480000937A69D8F814309B1A0193D8F818301E
:109F5800BA6968469B1A029303F0A8FD08F11C0A27
:109F680007F11C0510243C4901230A68A340134249
:109F7800894605D0DAF800002B68C01A03F037FECE
:109F88000134132C0AF1040A05F10405EBD108F198
:109F9800260007F12601002330F9022F31F9024F7C
:109FA800121B4DF823200133042BF5D10322002581
:109FB8005DF82230AD00EDB26BB103F108010F2955
:109FC80002D845F0010506E08033FF2B94BF45F029
:109FD800020545F0030512F1FF32E9D22846FFF7E2
:109FE800CBFD0024EB46A24605F00303022B16D056
:109FF800032B1DD0012B4ED1BAF1000F05D1DBF890
:10A0080000402401E4B29A4645E0DBF8000000F085
:10A018000F002043FFF7B0FD4FF0000A3BE0BAF114
:10A02800000F0CD0DBF80000C0F3031020432CE035
:10A03800BAF1000F1ED19BF80100FFF79DFD9BF8B8
:10A048000000FFF799FD26E034290020801D00203C
:10A05800D427002030290020282900202429002086
:10A0680018260020E027002013DA4B683C2900203E
:10A0780038290020DBF80000C0F303302043FFF745
:10A088007BFDDBF80000C0F30710FFF775FDDBF878
:10A0980000402401E4B20BF1040B04AB9B454FEAEA
:10A0A8009505A1D1BAF1010F02D12046FFF764FD51
:10A0B800D9F8003013F480541FBFB8F86420B7F8FB
:10A0C8006410521A009218BF012499040AD508AAEC
:10A0D80002EB8401B7F86600B8F86620121A41F856
:10A0E800202C01341A040BD508AB03EB8402B7F813
:10A0F8006810B8F868305B1A42F8203C013400E078
:10A10800DCB1012C03D1009803F071FD15E0631E4A
:10A1180000205DF823204000C0B20AB140F00100E1
:10A12800013BF6D5FFF728FD00255DF8250008B1AD
:10A1380003F05DFD0135A542F7DB30200321FFF771
:10A14800F9FC36200321FFF7F5FC144B3C20197865
:10A15800FFF7F0FCD9F800309B0506D5B8F95E008A
:10A16800B7F95E30C01A03F042FD32680C487368D4
:10A178007260121A91100B4AB3604A43531C0322AF
:10A1880093FBF2F202EB42029A1A6C2303FB0203DE
:10A19800336003F079FC09B0BDE8F08F1826002081
:10A1A800E027002013DA4B682DE9F74F0E9F4D4C3E
:10A1B800C2EB030B0D9BFF1A6368002914BF4FF015
:10A1C80006094FF0040901338246164634D1226845
:10A1D8004A4580F08280DFF82881019158F82200F2
:10A1E80009F0AFFA0B3003F0EFFB0199054608B10F
:10A1F800012073E022683C48032A98BF514658F86A
:10A20800222003F08BFD394A1368181A636810601E
:10A2180001336360364B9D720EE00D9A92B103FBD9
:10A2280007F20D99895C01228A40324909680A427D
:10A2380008D163680133636063680C9A294D9342BF
:10A24800EBDB32E003FB0BF5236806EB050A2BB9C1
:10A25800705909F076FA00F1050801E04FF003089B
:10A26800404603F0B1FB0028C2D1204A204B1068B9
:10A27800C8EB000010609A7A1AB12C20FFF77CFC1A
:10A2880001E001229A72236843B9705903F0B3FCC4
:10A298009AF904104B1CCCD0174803E09A4417488D
:10A2A8009AF8041003F03AFDC3E710D1012003F037
:10A2B8008BFB60B90D4A13680A20013B1360FFF756
:10A2C8005BFC2B6801332B604FF0FF336B60206819
:10A2D80048452CBF0020012000E0002003B0BDE865
:10A2E800F08F00BF442900200E7401084029002087
:10A2F80030130020282900201D74010895730108D7
:10A308007052010830B585B004AC002524F8025D10
:10A318000091ADF8060021461020FFF7D5FB9DF807
:10A3280006002146FFF7D0FB9DF807002146FFF7FE
:10A33800CBFB9DF800002146FFF7C6FB9DF8010006
:10A348002146FFF7C1FB9DF802002146FFF7BCFB41
:10A358009DF803002146FFF7B7FB9DF80E00C043A8
:10A36800C0B22946FFF7B0FB05B030BD10B5054CAB
:10A37800206804F00FFC18B1206804F008FCF6E728
:10A3880010BD00BF7C07002030B50028104C114AD2
:10A39800B8BF40423C2590FBF2F304FB030068433E
:10A3A8000D4D90FBF2F22D682D7B25B903EB83034D
:10A3B80003EB830301E0C3EB031302EB83030B807E
:10A3C80004FB02024FF47A7392FBF3F24A8030BD29
:10A3D800806967FF809698003407002010B504460E
:10A3E800C0B2FFF78FFBC4F30720BDE81040FFF7AA
:10A3F80089BB024B5E21186804F0CFBB30130020E4
:10A4080038B5064C05465E21206804F0C6FB206876
:10A418002946BDE8384004F0C0BB00BF3013002017
:10A428002DE9F04F2DED0A8B87B08346039390F802
:10A438005030029101925BB1322BA8BF322307EE54
:10A44800903AB8EEE7BADFEDD67A87EE8BBA01E03C
:10A458009FEDD4BAD44BDFEDD5BA1B88D44CDFF8C6
:10A468006493002B08BF012307EE903AB8EEE79AF1
:10A47800238869EE2BBA13F0020F3BEE2BBA8BEE52
:10A488008BBA26D0B9F90030B9F9022083EAE37112
:10A4980082EAE270A1EBE371A0EBE2708842054624
:10A4A800B8BF0D46B5F5E17F16DA8842DFEDC1AADF
:10A4B80005DD002AD8BF524207EE902A04E0002B9F
:10A4C800D8BF5B4207EE903AF8EEE77AC7EEAAAA41
:10A4D80004E0DFEDB9AA01E0F7EE00AADFEDB69AD5
:10A4E800B64A59464FF0000AB0EE69AAB448B54DCD
:10A4F80030F81A00B4F800E003B207EE903AF8EE2C
:10A50800E77AB5EE047A67EE877A35F91A309FED67
:10A51800AE7AFDEEE77A06EE903AF8EEE77A1EF0AC
:10A52800030F5FFA8AF64FEA4A0767EE877AF8EE72
:10A53800E66A6FD036EEA67A019BBDEEC77AC3F104
:10A54800000817EE105A454503DBAB42A8BF2B465F
:10A5580098469E4D039B7D5F9FED9D5AC5EB08086D
:10A5680033F91A509BF81C30454407EE105A0AEE8E
:10A57800103A9BF80830B8EEC76A07EE103AB8EE02
:10A58800477AB8EE4AAA26EE077AF1EE045A27EE81
:10A59800057A6AEE255ABDEEC77A17EE108AB1EE33
:10A5A800657ABDEEC7AA1AEE103A984508DBBDEEEB
:10A5B800E5AA1AEE103A4345A8BF43460AEE103AF8
:10A5C800844D05EB8A0595ED007AA6EE2B7ABBEE55
:10A5D8000E6AB4EEC67AF1EE10FAB8EECAAA09D439
:10A5E800B3EE0E6AB4EE467AF1EE10FAC8BFB0EEDA
:10A5F800467A01E0B0EE467A85ED007A9BF8123093
:10A6080009EE903AF8EE699A27EE297ADFED729A08
:10A6180067EE299A1EF0010F50D100B20028B8BF8A
:10A628004042B0F5206F02DD0020106025E09FED6C
:10A638006B6A4B7826EE867A06EE103AB8EE466AD2
:10A6480087EE066A92ED007A36EE676AA6EE2B7AF6
:10A658009FED636AB4EEC67AF1EE10FA09D49FED65
:10A66800616AB4EE467AF1EE10FAC8BFB0EE467AE7
:10A6780001E0B0EE467A82ED007ACB7A92ED007A6C
:10A6880008EE103AB8EE488A1EF0020F28EE077A54
:10A698009FED558A27EE088A14D076EECA6AB0EE86
:10A6A8004A7AAAEEA67A38EE698AF0EE476AB0EEE0
:10A6B800697AAAEE887AB0EE478A03E0B0EE698A32
:10A6C800F0EE4A6A49489FED4A6A1AF80030059246
:10A6D80007EE103AB8EEC77A4FEA8A0827EE677A8B
:10A6E800051D4544E7EE066A049195ED007AC5ED2F
:10A6F800007A37EEC77A00F10C0587EE2B7A4544CD
:10A7080014301AF80030D5ED007A37EE677A08EE83
:10A71800903AEBEE077AF8EEE88AC5ED007A67EE34
:10A72800A87ADFED348A344D67EEA88A36EE880AB7
:10A73800B0EE66CA30EE680A09F0CEF9E853208810
:10A748000499059A10F4006F08D02C480078400747
:10A7580004D53046FEF7CEF9059A04992848294FC2
:10A76800FDEECC6AFDEEC87AF1EE688A16EE903AF4
:10A7780017EE906AFDEEE88A48F8003048F807605E
:10A7880018EE903A204E049648F80630043201310B
:10A798008046BAF1000F3BD14FF0010AA6E600BF90
:10A7A80083F9223EAF4C593CD00E0020BD37863588
:10A7B800E00E00200000E143000000003C130020F0
:10A7C8000A0F002080190020CDCC4C403C0F0020FF
:10A7D8006F12033C481300200AD7A33D0000A04392
:10A7E800000040C3000040430AD7233C5013002018
:10A7F800A69B443BF7CC9238C8190020E02A0020D9
:10A80800D0190020DC190020E819002000803B4501
:10A81800BDEEC99A5FED037A9BF853609049DFF863
:10A8280064A219EE103A23F0030309EE103A029BD2
:10A83800B8EEC99A9B7989EE279AB5EE000A002EE0
:10A848006DD0B9F904209BF80300002AB8BF524222
:10A858005A43844B92FBF3F364336422434393FBE0
:10A86800F2F308EE903AB1F9043007EE903AF8EEB8
:10A87800E77AF8EEE88A27EE800A09F02DF907EE64
:10A88800900AF8EEE77AB9F9043067EEA88ADFEDA6
:10A89800767AC8EEA78A80EAE072A2EBE072B2F597
:10A8A800207F07EE903AF8EEE77A77EEE88A05DC43
:10A8B80083EAE372A2EBE372642A03DD0023CAF899
:10A8C8000830A2E003EB83031A019BF8033092FBE4
:10A8D800F3F31B1A07EE903AF8EEE77ADAF8083045
:10A8E80067EE897AFDEEE77A17EE902A1A44134646
:10A8F800B2F57A5F5D4AA8BF4FF47A539342B8BF66
:10A908001346CAF808307D2293FBF2F39BF80D201A
:10A9180053439B1107EE903AB8EEE78A75E0544A24
:10A928005B00B2F90490283303FB09F9B1F904304C
:10A9380007EE903AF8EEE77A4FEA691927EE800AAF
:10A9480009F0CAF8B9F1000FC0EB090007EE900A48
:10A95800B8BFC9F10009B9F1320FB8EEE77A02DDE4
:10A96800CAF808601BE09BF80D3007EE903AF8EE45
:10A97800677ADAF8083067EE277A67EE897AFDEEAB
:10A98800E77A17EE902A13443A4A9342A8BF13462F
:10A99800394A9342ACBFCAF80830CAF80820DAF836
:10A9A80008305B13B3F5807FA8BF4FF480736FF056
:10A9B800FF029342B8BF134607EE903AB8EEE78A13
:10A9C800FDEEC77A9BF8032017EE903A53439B118C
:10A9D80007EE903A294B1B78032BF8EEE78A14D937
:10A9E800BBF84E20B2F5FA7F0FD2FDEEE87A53425B
:10A9F80017EE901A994204DB914217EE903AA8BFDD
:10AA0800134607EE903AF8EEE78A78EE887AFDEE7C
:10AA1800E77ACDED017ABDF80430AB801BB200EEC9
:10AA2800103AB8EEC00A09F057F82388A8801A052A
:10AA380006D5134B1B785B0702D50220FEF75AF8A0
:10AA4800FDEEE88ABDEEC88A049AC8ED028A0023A2
:10AA580087ED028A936007B0BDEC0A8BBDE8F08FE2
:10AA68000A0F00200CFEFFFF0000A04280C1FFFF7C
:10AA780080190020FEFFFF0F020000F018260020BA
:10AA8800E02A0020981900202DE9F04F87B0002611
:10AA98000593BA4B0491B3F90270B3F900300292EE
:10AAA800002FB8BF7F42002BB8BF5B429F42B8BFA0
:10AAB8001F46B7F5FA7F8046A8BF4FF4FA77009093
:10AAC800B3460196B2463446AD4B198811F00302DD
:10AAD8003DD0AA4B33F91400029B40005B429842D8
:10AAE8004FEA440503DB029B8342A8BF0346A548FF
:10AAF8002D5E05985B1B30F914501D4498F80830FA
:10AB080064206B4393FBF0F398F81C006FF0040A81
:10AB18000AFB00FA534504DB00EB800A9A45A8BFFC
:10AB28009A46994850F824302B4442F21075AB42AB
:10AB3800A8BF2B46954DAB42B8BF2B4640F82430F2
:10AB480098F8120043431B13012A019338D08B4B0A
:10AB58008F4833F914B0009B50F824E093F801C0F3
:10AB68008C4B33F9145085EAE573A3EBE573B3F521
:10AB7800206F4FEA840616DC0BEB8B031A0192FB5D
:10AB8800FCF3042295FBF2F55D1BAE44BEF57A5F3B
:10AB9800A8BF4FF47A5E804B9E45ACBF40F824E0D6
:10ABA80040F8243002E0002340F8243083597D2601
:10ABB80093FBF6F6009BDB7A7343402693FBF6F68D
:10ABC800880711D50198C7F5FA7307FB0BF907FB3E
:10ABD80006F54FF4FA7103FB0A9903FB005599FB3C
:10ABE800F1F295FBF1F505E0C9074DBF019D35462A
:10ABF8005A465246630069490393664B605C33F8D2
:10AC080014E020310FFA8EF34FF0040C93FBFCF99B
:10AC180009FB00F06FF04F0990FBF9F9914431F905
:10AC2800142021F814E098F850109B1A93FBFCF3B9
:10AC380079B107EE903A5A485A4BB8EEE70AD3ED85
:10AC4800000A00EBC400FEF7EFF8FDEEC07A17EE3D
:10AC5800903A554A554912F804C0039803EB430348
:10AC680009EB05020CFB03F34FF0200C93FBFCF3FC
:10AC7800D21A4252424A1288120508D54C4A127812
:10AC8800500704D520460393FDF734FF039B494A38
:10AC980049494A4841F824905B4242F82430009BD5
:10ACA80040F82450013300930D4681460CB9012425
:10ACB8000AE7324B3648B3F90410049B86689B793F
:10ACC8000F335B004B435B113249002B4FF00404F8
:10ACD800B1F9041091FBF4F1A3EB0101B8BF5B4299
:10ACE800322B98F80D400BDC354B04FB0164A34272
:10ACF800A8BF2346334CA342ACBF8360846001E005
:10AD080000238360304B98F803401B784C43032B97
:10AD18004FEAA4140CD9B8F84E30B3F5FA7F07D22D
:10AD280059428C4203DB9C42A8BF1C4600E00C46FB
:10AD3800866846F34F36B6F5807F6FF0FF03A8BFED
:10AD48004FF480769E42B8BF1E46184BA1199980D1
:10AD58000B4B1B88190508D5154B1B785B0704D5C9
:10AD680002200092FDF7C6FE009AAC600023C9F8E5
:10AD78000860936007B0BDE8F08F00BF801900201D
:10AD8800E00E00203C0F002068130020F0D8FFFFE1
:10AD9800981900200A0F002080C1FFFF50130020DF
:10ADA800B01900209419002064130020C81900204D
:10ADB800E02A0020E8190020D0190020DC19002022
:10ADC800FEFFFF0F020000F0182600202DE9F04FCB
:10ADD80087B080460493A94B03911C88029204F023
:10ADE8000204A4B294B1A64BB3F90240B3F90030FF
:10ADF800002CB8BF6442002BB8BF5B429C42B8BF6E
:10AE08001C46B4F5007FA8BF4FF40074C246002565
:10AE18009B4B9C4E33F915E09B4B33F8153001934F
:10AE2800BDF9040056F8253080EAE077A7EBE07713
:10AE38000421B7F5206F90FBF1F189B24FEA450B79
:10AE48004FEA4E0C0AB24FEA85090FDCC2EB0C023E
:10AE58001344B3F57A5FA8BF4FF47A538B4A9342F1
:10AE6800ACBF46F8253046F8252002E0002346F816
:10AE7800253056F809709AF80B30804AFF115F4365
:10AE880012889AF80130960703FB0CF34FEAA717CC
:10AE98004FEAA31340D0029A4FEA4E0E524296450B
:10AEA80003DB029A7245A8BF7246794EDFF814E2B6
:10AEB8003BF90660961B049A32F91520164459F896
:10AEC8000E2042F2107C32446245A8BF6246DFF889
:10AED800F8C16245B8BF624649F80E2098F808E004
:10AEE8000EFB06F698F81CE00EEB8E0EF611CEF16E
:10AEF800000C664503DB7645A8BF7646B44698F84D
:10AF0800126072431213BF1ACCEB03036743634307
:10AF180002EB67270CEB63235E4A565D243211FB74
:10AF280006F6A3EBA6163BF9023098F85010C01AA3
:10AF3800042390FBF3F0BDF804302BF8023079B10C
:10AF480007EE900A544B5548D3ED000AB8EEE70ACD
:10AF580000EBC500FDF768FFFDEEC07A17EE900A1A
:10AF68004F4B504A5B5D00EB400058434311F119C9
:10AF7800C91A2BF802104149088810F4006F8B4653
:10AF88000AD049490978490706D528460592019308
:10AF9800FDF7B0FD059A019B4448454949F8006012
:10AFA800444E49F801705B4249F806300AF1010A3B
:10AFB800074689460DB901252AE7314B98F80D0057
:10AFC800B3F90410039B9B790F335B004B435B1170
:10AFD8002D49002BB1F904104FF0040591FBF5F54C
:10AFE8002849A3EB0505B8BF5B42322B8C680BDC04
:10AFF800314B00FB05408342A8BF03462F488342DC
:10B00800ACBF8B60886001E000238B6098F8033048
:10B018005D432B4B1B78032B4FEAA5150CD9B8F8C9
:10B028004E30B3F5FA7F07D25842854203DB9D4282
:10B03800A8BF1D4600E005468C6844F34F34B4F5BC
:10B04800807F6FF0FF03A8BF4FF480749C42B8BFA5
:10B058001C462B199380BBF800301A0506D5124BF5
:10B068001B785B0702D50220FDF744FD0023BD6075
:10B07800C9F80840B36007B0BDE8F08FE00E0020C3
:10B0880080190020981900200A0F002080C1FFFFB6
:10B098003C0F00205013002094190020B019002004
:10B0A80064130020C8190020E02A0020D0190020CD
:10B0B800DC190020E8190020FEFFFF0F020000F055
:10B0C8001826002068130020F0D8FFFF2DE9F04F64
:10B0D8002DED028B85B000260293A44B0192B3F9A3
:10B0E8000270B3F900300090002FB8BF7F42002BE8
:10B0F800B8BF5B429F42B8BF1F46B7F5FA7F834689
:10B10800A8BF4FF4FA77B046B146B2463446984BDA
:10B118001B8813F0030045D0022C43D0934A32F920
:10B128001410019A4900524291424FEA440503DB48
:10B13800019A8A42A8BF0A468E4935F901900299B8
:10B148009BF81C5031F91410C9EB020202EB0109FB
:10B158009BF8081001FB09F2642192FBF1F16FF0F2
:10B16800040202FB05FA514505DB05EB8502914215
:10B17800A8BF11468A46804D804A55F8241042F2ED
:10B18800107E49447145A8BF714691429BF81290C0
:10B19800B8BF114609FB01F9012845F824104FEA08
:10B1A800293942D0764D714935F91450009A7548BD
:10B1B80031F9148092F801E050F8242085EAE57608
:10B1C800A6EBE576B6F5206F4FEA840120DC022C69
:10B1D80018D008EB8800000190FBFEFE042095FBC8
:10B1E800F0F5C5EB0E0E02EB0E0CBCF57A5F654868
:10B1F800654DA8BF4FF47A5CAC45ACBF41F800C0C0
:10B208000D5007E088EAE876A6EBE876642EE0DDE4
:10B21800002545505B48009A09587D2691FBF6F6B3
:10B22800D17A7143402691FBF6F69D0712D5022C80
:10B2380010D0C7F5FA7307FB06F507FB08F103FB07
:10B248000A114FF4FA7003FB095391FBF0F193FBD9
:10B25800F0F508E0D80704D5022C02D04D46514637
:10B2680001E035464146464B33F91400042390FB70
:10B27800F3F34648205C022C03FB00F36FF04F0009
:10B2880093FBF0F30B444FEA440C08EE103A0ED14E
:10B298003F4B4048D3ED000ACDF80CC0B8EEC80AC1
:10B2A8001E21FDF7C1FDDDF80CC0BDEEC08A344B90
:10B2B80039493CF803003CF901302CF801009BF8AF
:10B2C80050100FFA80FEC3EB0E034FF0040E93FBF1
:10B2D800FEF399B107EE903A30482D4BCDF80CC0EB
:10B2E800B8EEE70AD3ED000A00EBC400FDF79CFDB9
:10B2F800FDEEC07ADDF80CC017EE903A28492948CF
:10B3080011F804E018EE102A03EB430351190EFB61
:10B3180003F34FF0200E93FBFEF3C91A2CF800102C
:10B3280013490988090508D51F4909784A0704D52A
:10B33800E0B20393FDF7DEFB039B1C4918EE102ACD
:10B3480041F824201A4941F824501A495B4241F82F
:10B358002430009B01340133032C00937FF4D7AED3
:10B3680005B0BDEC028BBDE8F08F00BF801900204E
:10B37800E00E00203C0F002068130020F0D8FFFFEB
:10B388000A0F00209819002080C1FFFF50130020E9
:10B39800941900208C19002078130020B01900207F
:10B3A80064130020C8190020E02A0020D0190020CA
:10B3B800DC190020E8190020026BC168034610B5AB
:10B3C800406942B11A6C8C1A013A005D08BF0A46FE
:10B3D800C0B21A6410BD1A6A805C01328A4228BF62
:10B3E8000022C0B21A6210BD436B13B190F844003A
:10B3F8007047836A406A1B1A584258417047426A2C
:10B40800816A03698A4238BFD218521A416B21B146
:10B4180049680A44591E8A4203D2013B981AC0B2AD
:10B42800704700207047036B13B15B68016C01E043
:10B43800C369016A8B423CBFC2689B18581AC0B2E4
:10B448007047836A8169426B1944D160416A9942A5
:10B458009DBF0169CB1A5360CB1A96BF0023536076
:10B4680083624FF0000380F84430136888BF81621C
:10B4780043F0010313607047436A8269D154436AF9
:10B4880002690133934228BF00234362436B1BB117
:10B498001B68DB0705D4D4E7026D136843F080030B
:10B4A800136070474171F9F703BF8160F9F700BF76
:10B4B800026D036B70B50446D5699BB9A90611D511
:10B4C800C36A1BB1908C80B298470BE0E169928CFB
:10B4D80040694E1CD2B2E6614254E169E268914289
:10B4E80028BFE361616BA1B92A0612D5636AA26A13
:10B4F8009A42236D09D0501CA669A062B25C1A85D5
:10B508002369984205D3A16203E01A6822F08002F9
:10B518001A602B0742BF236D08221A6270BD0D4BBB
:10B528000D484FF400525A600C4A11684FF6FE73EA
:10B538000B401360426B11684FF6FE730B401360AB
:10B54800426A836A9A4200D07BE7012380F844303C
:10B55800704700BF00000240681C00204400024001
:10B568002DE9F0471E469F4B8CB09842894690467D
:10B578009DF850507ED19C4B9C4A1A609C4A5A6157
:10B5880002F580729A614FF48072DA601A61994A02
:10B598001A63143A5A63A2F54842203ADA6404322C
:10B5A8009A64C3F808801865934B9A6942F48042FC
:10B5B8009A615A6942F001025A6102238DF80830F3
:10B5C800032315F0010A8DF809304FF000038DF8B8
:10B5D8000A3014BF022301232C078DF80B3017D52E
:10B5E800864C402701978AF001038DF80A30236AB8
:10B5F80023F070632362236A43F0E06323622046EA
:10B6080001A9FBF77BFDBAF1000F23D1A76121E067
:10B61800B0070ED50CA9402341F82C3D7748036AA2
:10B6280023F070630362036A43F0E0630362FBF78D
:10B6380065FDF1070ED50CA9802341F82C3D6F4814
:10B64800036A23F070430362036A43F0E043036232
:10B65800FBF754FD0E238DF80030002201236846C5
:10B668008DF801308DF802208DF803305E4C02F021
:10B67800BBFE04E1624B984270D1624B5B4A1A6090
:10B688004FF48072DA601A615F4A5A6102F580727B
:10B698009A61594AC3F808801865D36943F400339E
:10B6A800D36102238DF80830032315F0010A8DF8C1
:10B6B80009304FF000038DF80A3014BF022301232C
:10B6C8002A078DF80B3017D54C4C082701978AF0BC
:10B6D80001038DF80A30236A23F470432362236A36
:10B6E80043F4E0432362204601A9FBF707FDBAF1C2
:10B6F800000F23D1A76121E0B3070ED50CA90823B9
:10B7080041F82C3D3D48036A23F470430362036A01
:10B7180043F4E0430362FBF7F1FCF7070ED50CA9ED
:10B72800102341F82C3D3548036A23F47023036243
:10B73800036A43F4E0230362FBF7E0FC26238DF859
:10B7480000300022012368468DF801308DF8022070
:10B758008DF803302B4C02F047FE90E02B4B9842BB
:10B7680040F00E812A4B214A1A604FF48072DA6049
:10B778001A61284A5A6102F580729A611E4AC3F812
:10B7880008801865D36943F48023D36102238DF8B8
:10B798000830032315F0010A8DF809304FF0000333
:10B7A8008DF80A3014BF022301232C078DF80B30C3
:10B7B80032D5124C4FF4806701978AF001038DF857
:10B7C8000A30636A23F470636362636A43F4E06374
:10B7D8006362204601A9FBF791FCBAF1000F3FD143
:10B7E800A7613DE000380140681C0020885201082C
:10B7F8008013002058000240001002400004004856
:10B8080000440040141C002080150020004800401F
:10B81800C01B002080170020B0070FD50CA94FF4DB
:10B82800806341F82C3D5848436A23F470634362AF
:10B83800436A43F4E0634362FBF760FCF1070FD50A
:10B848000CA94FF4006341F82C3D4F48436A23F498
:10B8580070434362436A43F4E0434362FBF74EFCA0
:10B8680027238DF800300022012368468DF8013027
:10B878008DF802208DF8033002F0B6FD434CC4F871
:10B888002C900027012384F844302762E761A762DF
:10B8980067626671C4F80880A5712046F9F708FD4B
:10B8A800F20734D5236B002B2AD001A8FBF7C2F985
:10B8B800E36C01934FF480530A9380230693E36863
:10B8C800ADF8103020230993206B636902930B971E
:10B8D8000597079708970397FBF7D7F901A9206BF6
:10B8E800FBF7B5F9236B216D1A6842F001021A6063
:10B8F8008A6842F040028A605B689BB2236406E073
:10B90800236D20221A621A6842F020021A60B307D7
:10B918002FD5636B43B301A8FBF78CF9A36C019394
:10B928004FF480530A93802306932369ADF81030AF
:10B9380000251023606B03930B95059507950895D3
:10B948000995FBF7A2F9606B01A9FBF780F9636B16
:10B958001A6842F002021A60226D5D605D609368A9
:10B9680043F08003936004E0226D136843F0800382
:10B978001360226D136843F001031360204600E052
:10B9880000200CB0BDE8F08700040048C01B002070
:10B998002DE9F04F2DED028B85B0814603938A4B3C
:10B9A80002921B889D0737D5109B8848DC89B0F91F
:10B9B80000301B1B03F2F31540F2E632954203D820
:10B9C800002BB8BF5B4201E04FF4FA73B0F90220D4
:10B9D800121B02F2F31440F2E630844203D8002A24
:10B9E800B8BF524201E04FF4FA729342B8BF13460F
:10B9F800C3F5FA73052293FBF2F30A22643B53431F
:10BA080099F81C20D2105343642293FBF2F3134499
:10BA180023EAE373DBB200E064230093CB1C0193B9
:10BA2800C8460025019B6A4813F8011F0193022D9F
:10BA38004FEA450A06D1B0F9040001F11B0444435A
:10BA480063112DE030F91520029B50005B429842AB
:10BA580003DB029B8342A8BF03465E4830F90A40D5
:10BA6800039830F915001B1B1844574B1E88F40720
:10BA780012D401F11B035A43B1074FEA22130FD521
:10BA880099F812409DF9001044434C43642294FBFA
:10BA9800F2F203EB221303E099F8083043431B1139
:10BAA8004D4A042432F90A2092FBF4F41C1B484B3B
:10BAB80003F108026421AF5C98F8012062437A43DD
:10BAC800022D92FBF1F24FEAE21208EE102A0AD197
:10BAD800B8EEC80A03F10C001E21D3ED050AFDF7E4
:10BAE800A3F9BDEEC08A3A4A3C4B98F80B601B8814
:10BAF80002F1180E03FB04F05EF82510C01206FBD5
:10BB08000016B6F5001F3649A8BF4FF4001602F11B
:10BB180024008E42B8BF0E4650F8251040F8254044
:10BB2800611A1B094FF6FF70B0FBF3F34B4399F80A
:10BB380050104EF825604FEA850B76139B1179B1AA
:10BB480007EE903A02F13000B8EEE70A00EBC500C4
:10BB5800D2ED050AFDF768F9FDEEC07A17EE903AC6
:10BB680098F815101F4A03EB43034B435F436423C4
:10BB780097FBF3F718EE103A3F1233443B4422F890
:10BB88000A30114B1B881A0506D5174B1B785B0723
:10BB980002D5E8B2FCF7AEFF144B18EE102A0135B7
:10BBA8004BF8032003F10C021833032D4BF8026005
:10BBB8004BF8037008F101087FF434AF05B0BDEC11
:10BBC800028BBDE8F08F00BFE00E0020C21C0020F1
:10BBD800801900203C0F00200A0F0020480F002089
:10BBE8000000E0FFC8190020E02A0020D01900203A
:10BBF8002DE9F04F2DED0A8B97B011F0FD080646A0
:10BC08000191A94C06D0A94B1B689A0700F1B08096
:10BC180000F041BCA36FA648DFF89492984700282B
:10BC2800F1D0A44F94F8882048464946FBF7A2FA79
:10BC38003B8804F1D802002B70D0D4F88C301B78E4
:10BC480008EE103A04F1900A04F19C05B7F800B028
:10BC580039F91800BBF57A7F02BF0023CAF8003013
:10BC68002B61DAF800300344CAF800302B6907EE7C
:10BC7800900A0133012B4FEA4801F8EEE77A2B616D
:10BC880006D10023C5ED017AC5ED007AAB601BE053
:10BC9800D5ED006A07EE103A37EEE66AB8EEC77AD5
:10BCA80086EE077A36EE877AD5ED026A85ED017A57
:10BCB80077EEC77A85ED007AE6EE276AF0EE667AC7
:10BCC800C5ED036AC5ED026A0023BBF1010F29F82F
:10BCD800013053522DD12B690392012BC3BF03F1BD
:10BCE800FF3300EE103AD5ED037A9FED730A029107
:10BCF800C4BFB8EEC00A87EE800A07F095FF029924
:10BD0800039A18EE103A5BB1F8EEC87AB4EEE70A77
:10BD1800F1EE10FA04DD4FF47A733B8000231CE047
:10BD2800DAF800304FF47A7003F5FA7393FBF0F306
:10BD3800535208F10108B8F1030F0AF1040A05F19A
:10BD4800140583D1BBF1010F04D15846029202F0C9
:10BD58008BFE029A3B88013BDFE739F8131032F873
:10BD68001300091A29F813100133032BF5D14AE7F8
:10BD7800019B002B00F08F8394F8DE704A4D6FB161
:10BD8800012F40F0808305F59470D5ED486A95ED54
:10BD9800497A05F59A730021804613E102F00CFEFA
:10BDA800D5F8E8309FED457AC5F8E000C31A07EEEC
:10BDB800903AF8EE677A424BC5F8E80067EE877A62
:10BDC8005B68C5ED397A05F1EC00984705F1EC0898
:10BDD800002800F0F1803B4B40461A784146FBF7BB
:10BDE800C9F9B5F8F230002B42D0D5F8F4103B462B
:10BDF800B4F8F22038F913702B4DB2F5C87F324AE7
:10BE080004BF002042F823004FEA830E52F80E00C8
:10BE1800384442F80E00002028F8130021F81300D7
:10BE28000133032BE4D1B5F8F230012B1BD1D5F83F
:10BE3800F8304FF4C87703F1C80292FBF7F20A8092
:10BE4800D5F8FC20C83292FBF7F24A801F4AD5F891
:10BE580000311288C83393FBF7F39B1A8B8030802C
:10BE68007080FDF7B9FDB4F8F230013BA4F8F23068
:10BE7800174B1B685B0740F18B80B4F804210A4B11
:10BE8800322A27D1D3F8F4201188A3F80611518853
:10BE98009288A3F80A213288A3F80C217288A3F8A3
:10BEA8000811A3F80E2117E080190020DC0E0020ED
:10BEB8000A0F0020DC2A002000000000BD3786356C
:10BEC80090270020E22A0020781A0020080000208D
:10BED800842A0020002A3BD0D4F8F4000023B4F8C8
:10BEE800042138F913E0C64D322AC64A04BF00219E
:10BEF80042F823109F00D1597144D151002228F8EB
:10BF0800132020F813200133032B1146E7D1B5F88D
:10BF18000431012B17D10C2085F81C2185F81D311F
:10BF280002F0A2FDD5F8F430B5F806211A80B5F86C
:10BF380008215A80B5F80A219A80B5F80C31338067
:10BF4800B5F80E317380B4F80431013BA4F804311C
:10BF580094F81E31AA4ADBB1D2F8F400D2F81031B5
:10BF6800002182F81E11322593FBF5F30380D2F8E5
:10BF7800143193FBF5F34380D2F81831A24A93FBAE
:10BF8800F5F312889B1A838031807180FDF724FDB8
:10BF9800D4F8F420B4F8EC3011885B1AA4F8EC302B
:10BFA8005188B4F8EE305B1AA4F8EE309288B4F8F1
:10BFB800F0309B1AA4F8F03094F8DE30013384F89E
:10BFC800DE30D9E68E4D914F05F1EC0232F81120A2
:10BFD80027F8112012B207EE902A8D4AF8EEE77A78
:10BFE80032F9112067EEA67A0131E0EC017A07EE0A
:10BFF800902AF8EEE77A032967EE877AE3EC017A6C
:10C00800E0D105F59A7005F5A071024602F0D1FF5E
:10C0180005F59A7005F5A67104AA02F0CAFF04A8EE
:10C0280095ED390ADFF8D8A1014602F0DBFFDDED16
:10C03800054ADDED047A9DED065A95ED594AD5ED90
:10C04800583A95ED563AB6EE007A64EE874A67EEAE
:10C05800875A64EEA47A25EE075AE5EEA57A07A872
:10C068000146B7EE008AE5EE057A0AAA0DAFF0EEB2
:10C07800482AE7EEC72A0AF5BC7965EE846AD5ED49
:10C08800577AE2EEA36A25EE236AE4EE836A23EE8A
:10C09800E57AB1EE452AE2EE276AA2EEA76AA4EE97
:10C0A800A77A67EEE57AF1EE641AE2EE837AA1EEFA
:10C0B800846AA2EE847AE1EEA37AA5EE836AA5EEFD
:10C0C800037AE2EE047A85ED576AC5ED567AB1EE49
:10C0D800466AC5ED586A85ED597AF1EE666AB1EEA1
:10C0E800477A8DED097A8DED076ACDED086A02F081
:10C0F80060FF95ED560A474810A902F073FF07A89C
:10C10800444913AA02F036FF13A810A93A4602F0D0
:10C1180050FF0AA8394613AA02F02CFF3D4813A97C
:10C128003A4602F046FFD5ED5A7A9DED0F7A95F81A
:10C138006C31B4EEE77AF1EE10FACCBF43F00803A5
:10C1480023F0080385F86C31D4F870311B78F0EED1
:10C15800489A0AF5C4753BB3DAED5D8A4846B0EEF5
:10C16800680A10A902F03EFF9AED618A0AF59470F8
:10C17800B0EE480A13A902F035FF4A4610A813A9E1
:10C1880002F017FF2846B0EE680A10A902F02AFF4D
:10C19800384613A9B0EE480A02F024FF10A813A9E4
:10C1A8002A4602F006FF07E098E8070089E807003A
:10C1B80097E8070085E80700D4ED4B7AD4ED4A6A82
:10C1C80094ED4C7A0E4D67EEA77A0023E6EEA67A38
:10C1D800E7EE077A9FED107AF4EEC77AF1EE10FADF
:10C1E80006DC9FED0E7AF4EEC77AF1EE10FA19D557
:10C1F800C4F84C31C4F85031C4F8543125E000BFBC
:10C2080080190020901A002008000020040F002048
:10C218000A0F0020AC520108B81E8D3F3D0A673F47
:10C228006F12833A05F5BC7005F5C47105F5A67261
:10C2380002F0A0FED5ED397A1FED070A05F5A670C4
:10C2480080EE270A014602F0CDFEB4F89431984DED
:10C2580001339BB2B3F57A7FA4F894312ED195EDD2
:10C26800570AD5ED566A95ED587AD5ED597A20EEEC
:10C27800000AA6EEA60AA7EE070AA7EEA70A07F085
:10C28800D3FC89EE800A0023A5F89431D5ED576ACE
:10C2980095ED587AD5ED597A95ED566A60EE266A8D
:10C2A80020EE077A60EE277A26EE000AC5ED576A77
:10C2B80085ED560A85ED587AC5ED597AD4ED578A39
:10C2C80094ED59AA94ED56BAD4ED58AA9FED799AEF
:10C2D80068EECA7AB7EE007AEBEE2A7A77EEA77A9A
:10C2E800F4EEE97AF1EE10FA0EDCFFEE006AF4EEF5
:10C2F800E67AF1EE10FA24D4F4EE477AF1EE10FA69
:10C30800C8BFF0EE477A01E0F0EE477A17EE900AE0
:10C3180004F074FA41EC100B07F024FC51EC100BFC
:10C3280004F0C0FA08EE100AB5EEC08AF1EE10FA71
:10C3380009DD78EE497AF5EEC07AF1EE10FA10DCF4
:10C3480023E09FED5D8AF1EE487A77EEC97AF5EE43
:10C35800C07AF1EE10FAB5EEC08A13DDF1EE10FAEC
:10C3680006DD38EE499ADFED557AB4EEE79A03E038
:10C378009FED527AF4EEC77AF1EE10FA4CBF012322
:10C38800002312E0F1EE10FA06DD38EE499ADFEDEF
:10C398004C7AB4EEE79A03E09FED497AF4EEC77A57
:10C3A800F1EE10FACCBF0123002353B1B0EE4A0AD4
:10C3B800F0EE4B0AFCF78CFF9FED42CA70EE008A44
:10C3C80041E02AEE8A0A6AEEAABAABEE280AB0EE73
:10C3D8006B7A30EE000AA8EEA87AB5EE400AF0EEC5
:10C3E800007AF0EE690AF1EE10FAE7EE670AB0EEAD
:10C3F800679A04D1F5EE400AF1EE10FA04D0FCF782
:10C4080067FFB0EE40CA01E09FED2ECA28EEAA0AE7
:10C41800EAEE0ABAABEE0A0AF0EE690A30EE000A52
:10C42800EBEEC90AB5EE400AF1EE10FA04D1F5EECA
:10C43800400AF1EE10FA04D0FCF74AFFF0EE408A09
:10C4480001E0DFED208A9FED209A204D2CEE090AAD
:10C4580007F042FB28EE090A288007F03DFBDFEDD4
:10C468001C7A1C4A688068EEE78AFDEEE88ACDED02
:10C47800018ABDF8043013F4004F18BF03F5B473F4
:10C488001380002300E00123002284F8DE20002B23
:10C498007FF472AC06E00023A4F8EC30A4F8EE3088
:10C4A800A4F8F03017B0BDEC0A8BBDE8F08F00BFE0
:10C4B80080190020DB0FC93FDB0FC9BF35FA0E3CDE
:10C4C80035FA0EBC000000004D3D0F443C0F002023
:10C4D800E12E6542400F002001380A4B042804D899
:10C4E800DFE800F00507090B0D00074A08E0074AD6
:10C4F80006E0074A04E0074A02E0074A00E0074A64
:10C508001A60704700010020D5B0000899B90008EA
:10C51800BDFE0008D5AD000891AA000829A40008AE
:10C52800704708B50B4B002093F82C10FAF7CEFA99
:10C53800094B1B68187A082801BF084B4FF4805232
:10C548001A80102208BF5A80A0F1090358425841A6
:10C5580008BD00BFD0000020BC1C0020181B002014
:10C56800704770477047FEE7FEE7FEE7704730B553
:10C578000024E3B293420DD2030F092B94BF30334A
:10C58800373301F8143001EB4403002500015D70D6
:10C598000134EEE730BD30B5002202F1805303F5D7
:10C5A800B8539B0042F400441D6840F60F7144F0F4
:10C5B8008004294001322143042A1960EDD1024B3D
:10C5C80040F08000186030BD4C5C00402DE9F34716
:10C5D800884D894C2B68894E9BB2A380A2883188EC
:10C5E8000A40970507D54FF6FF53854A2B60137805
:10C5F8000133DBB21370A3880B40180440F10083A9
:10C608000023ADF802302B687B4F9AB21804A28041
:10C6180040F1F682BB8803F00F03BB71002B40F09A
:10C62800C182784A13689BB23B803B8803F0300391
:10C638007B803B8803F440533B8011684BF6BF7303
:10C648000B4083F4005383F0200343F4004343F08A
:10C6580080031360BB88D90621D4116848F60F738C
:10C668000B40694913600B681A7A022A884601D080
:10C67800042A02D1FAF7B6F95AE2062A40F06B8288
:10C688005A78052A08D11A78520605D1D878FFF7C2
:10C6980082FFBB681B6A9847E3689B685AE2136885
:10C6A8009BB2ADF80230BDF802301F0540F1D081D1
:10C6B8001168554F40F68F730B40544913600A6850
:10C6C800534B92B213445B0088461A683B68187A49
:10C6D800092817D092B2520002F1804202F5C042F6
:10C6E80011781970517859709188C8B2090A41EACD
:10C6F800002159801189C8B2090A41EA00219980AC
:10C708009289DA8001221A72DA8893F80190002A55
:10C7180040F0DC801A7812F07F024AD1B9F1090F93
:10C728000FD1DA78012A00F2B8809978002940F010
:10C73800B4809988002940F0B0809A72A3685B6839
:10C74800A9E0B9F1050F10D193F90320002A01DA05
:10C758000823B9E09A78002AFAD19A88002AF7D1F2
:10C768009B7A002B00F0A280F2E7B9F1030F0ED1FB
:10C77800DA78012A40F091809A88002A40F08D806A
:10C788005A7A42F020025A72A368DB6983E0B9F151
:10C79800010F40F08280DA78012A7ED19A88002A37
:10C7A8007BD15B7A980678D5FAF7B2F900287DD064
:10C7B80073E0012A2ED1B9F10B0F6ED1E2685879D6
:10C7C8009269D97890473B689A7A002A65D0002800
:10C7D80063D11A79002A60D19B78002B5DD1064B72
:10C7E8009B68DB689847084B1B685A79DA72DA78D5
:10C7F8001A735BE0445C0040181B00209829002055
:10C80800E42A0020005C0040BC1C0020505C004072
:10C8180004300020022A40D1B9F1010FC4D0B9F187
:10C82800030F3AD1587920F0800E4FEA8E0202F1B8
:10C83800804101F5B84110F0800F096814BF01F07C
:10C84800300101F44051BEF1030F26D8B3F802E0DD
:10C85800BEF1000F21D101B39B7AF3B102F18042FE
:10C8680002F5B842010613684BBF23F4E04323F4F2
:10C87800804323F0400323F070034BBF9BB29BB26D
:10C8880083F0100383F4805343F4004343F08003A0
:10C898001360A3689B69984708E0E36848465B69AA
:10C8A800984703280FD000287FF452AFD8F800200B
:10C8B800A14B92B213445B001A6800221A6030231D
:10C8C8006380062300E009233A6847E1B9F1060FBF
:10C8D80012D11A78520678D19B78012B02D1E368DD
:10C8E800DB6967E0022B02D1E3681B6A62E0032B75
:10C8F8006BD1E3685B6A5DE0B9F1000F38D1598804
:10C90800002962D15A6822F47F42B2F5003F5CD117
:10C918001A7812F07F0204D19B88002B00F0D58191
:10C9280053E0012A08D1E2685879926990470028B3
:10C938004BD13B689B7A17E0022A46D15A7902F01C
:10C948000F010BB29B0003F1804303F5B84312F0CB
:10C95800800F1B6814BF03F0300303F4405303290E
:10C9680033D812F0700F30D1002B40F0AE812CE09C
:10C97800B9F1080F04D11B785B0600F0A88124E008
:10C98800B9F10A0F21D11A7802F07F02012A1CD1CD
:10C998009A7AD2B15988C1B95A6822F47F42B2F55D
:10C9A800803F12D1E268587992699047002800F0D8
:10C9B80090810AE04BB13A684FF00008A2F8128063
:10C9C80093614046984740460BE0E3683A681B6924
:10C9D80050789847032804D1584B1B6809221A72CB
:10C9E800BDE03A68138A4FF6FF718B4201D10923E3
:10C9F800B4E0022800D00BB90823AFE092F9001088
:10CA080000291FDAD18801910198834202D9019B3C
:10CA1800138210E08B420ED2E16891F82C00834219
:10CA280001D2002105E093FBF0F100FB113313B9AB
:10CA38000121434B1970E36893F82C309382F9F77E
:10CA4800D1FF8CE0032313724FF44053238086E018
:10CA5800BDF802301BB2002BBFF6D5AD116840F609
:10CA68008F730B401360354A17683B7A022B904648
:10CA780071D0042B6FD0032B01D0052B66D1BB6975
:10CA88003A8A8BB9398A00293BD04FF44053238026
:10CA98002C4B1A68284B92B213445B001A68002288
:10CAA8001A60302363802CE0002AEBD0B7F814908A
:10CAB800914528BF91461FFA89FA504698473B8A04
:10CAC800CAEB03033B827B8A53447B821D4B1A6863
:10CAD8001D4B92B213445B0009F101021B689BB223
:10CAE80003F1005303F5405352105B004FF0000E62
:10CAF8009645C7D053F82E1020F81E100EF1010EDF
:10CB0800F6E7BB8A8B42D8F8003001D8032201E04F
:10CB180011B105221A720BE006221A72094B1A6823
:10CB2800054B92B213445B001A6819603023638086
:10CB3800D8F800301B7A0FE002300020BC1C00201F
:10CB4800E32A0020505C004004300020072B02D16B
:10CB5800E368DB6898470823D8F800201372FFF7CA
:10CB6800E0FC5E4B1A684BF6BF7313402288D7046B
:10CB7800228848BF83F480539004628848BF83F4B6
:10CB88000053D106628848BF83F01003920648BF5D
:10CB980083F0200343F4004343F080034F4A9BB2E1
:10CBA80013602DE09A0002F1804202F5B842116844
:10CBB80089B2ADF80210BDF8021009B2002909DAED
:10CBC800106840F68F7101401160013B444A52F8E9
:10CBD80023309847BDF802301F067FF514ADA179C0
:10CBE8008B0003F1804303F5B84348F60F721868C9
:10CBF80002401A603A4B03EB81039B69984702E5B0
:10CC0800A28833881340590505D54FF6FF332B60AA
:10CC1800344B5B689847A28831880A40920444BF25
:10CC28004DF6FF732B60A3882F4A0B40DB0452D5C7
:10CC38004EF6FF732B6000231374137C052B41D829
:10CC4800DFE803F0030D1418222D6369264D1BB984
:10CC580001F0EEFD062300E005232B743BE001F014
:10CC6800E7FD042323740123636134E00223637422
:10CC7800032328E0637C013BDBB26374637C53BB12
:10CC8800194B04221A7426E0184A13689BB243F021
:10CC980010031360052323740A2363741BE0637C69
:10CCA800114A013BDBB26374637C03F0FF0093B964
:10CCB8000E490C684FF6EF7323400B60062313747C
:10CCC800506108E00623237405E0094B73E6094B1D
:10CCD80071E6094B6FE602B0BDE8F087005C0040E2
:10CCE800B8520108D0000020181B0020405C00400A
:10CCF800956600084D67000829670008FF207047FF
:10CD080090F844305A1C0344D2B22DE9F04380F81D
:10CD1800442083F8301090F845300BB1132A4FD9CE
:10CD2800002380F84430002A4AD0264B196800298D
:10CD380046D01B68052B43D12349202A144628BF17
:10CD48002024651C0E686D10204F3B6883BBDFF8FC
:10CD58008CC000F13203AE4613F8019C13F8028C24
:10CD6800BEF1010E48EA09282CF8048C03F10203ED
:10CD78000CF1040CF0D1164B1B681FFA83FE154BFF
:10CD880073445B00A646D3F800C01C603B6823448C
:10CD98003B60114F3B6823F4E04323F040039BB210
:10CDA80083F0300343F4004343F080033B6001E029
:10CDB8004FF0000E964503D00B689B1B312BC3D94F
:10CDC800BDE8F083C82A0020902A0020942900207A
:10CDD800505C00400A300020045C00408461004040
:10CDE800014B1868C0B270475029002001207047D5
:10CDF80070477047F7B51C4B1A680AB91C6800E001
:10CE080001241A490E780022D0B2A04202F1010290
:10CE180007D202AD2F18164D3544285C07F8040CCC
:10CE2800F2E71A68121B1A600A781D6822440A7011
:10CE38009DB903204021F9F749FE0E4A136823F4EF
:10CE4800804323F070039BB283F4405343F40043C0
:10CE580043F080031360054B1D70002CCBD09DF868
:10CE6800040003B0F0BD00BF50290020301B002093
:10CE7800542900200C5C004070B5044601F089F884
:10CE8800B4F5807F0ED0BB2C0ED8612C0ED8292C7F
:10CE98000ED8132C0ED8092C0ED8002C14BF06253A
:10CEA80000250AE0002508E0012506E0022504E047
:10CEB800032502E0042500E00525154C8021A36820
:10CEC8006B209847642001F093FDA36803216B2031
:10CED8009847104AA3681178192098470F2001F045
:10CEE80087FDA36829461A209847A36818211B20A4
:10CEF8009847A36810211C209847A368022137206F
:10CF08009847A36838200121BDE87040184700BF42
:10CF1800D4090020E409002008B501F03AF8074BCD
:10CF28005B7813B1012B03D008BD4FF4006201E018
:10CF38004FF48052024B1A8008BD00BFD009002070
:10CF480008000020094A13781844C0B210F0800F76
:10CF580018BF803810701346054A1978137899421B
:10CF680001BF00231370014A13707047321B002061
:10CF7800311B002010B50A4B0A4A1B7842609C18E6
:10CF8800094A046012789A4225BFD31A0B60C3F18C
:10CF9800800300232EBF4B600B604A6010BD00BFAA
:10CFA800321B0020331B0020311B00201FB56846B0
:10CFB80002A9FFF7DFFF044B02981B68034403989C
:10CFC800184405B05DF804FB400D0020054A064BE7
:10CFD80010781B7883422EBF181AC0F18000C01841
:10CFE800704700BF321B0020311B00200F4B73B568
:10CFF80018781C4698B105230D4D8DF800304FF474
:10D00800805600238DF8013001A82E85694602223A
:10D0180001F0B4F9AE619DF8050000F0010000F0E0
:10D028000100207080F0010002B070BD3D0D0020AD
:10D0380000040048064B70B51D6806461C46FFF7FD
:10D04800D5FF18B923685B1BB342F8D970BD00BF80
:10D05800902A00202DE9F04F89B0824601930023E1
:10D06800029103929946039A934205DA029A52F87A
:10D07800232001339144F6E7019B4D46002B56D1FE
:10D08800FFF7B4FF002852D101987CE002223F4EFE
:10D098008DF81C201A0C4FF480578DF81D2006209F
:10D0A8001A0A8DF81E208DF81F30FFF7C3FF378549
:10D0B800062001F03BF9364BB76101221A700020B7
:10D0C800378507A9042201F059F9029FD046264660
:10D0D8004FF0000B039B9B451EDABC4657F8042B08
:10D0E8004FEA8B03002A47D0B24235D332465AF86A
:10D0F8000310CDF814C00020049301F03FF9049BFD
:10D10800DDF814C05AF8032032444AF80320DCF84A
:10D1180000309E1BCCF800601C4B4FF480529A6183
:10D128001C4A13682D1B1C44019B14604BB345B368
:10D13800184B1B68DCB22A19B2F5807F164AD268F0
:10D148008CBFC4F580742C4693429FD3134A0023A6
:10D158001370134A137014E00020D8F8001001F07F
:10D168000DF957F8043CD8F80020F61A1344C8F80B
:10D178000030002347F8043C0BF1010B08F10408C8
:10D18800A8E7C5EB090009B0BDE8F08F0004004826
:10D198003D0D0020400D00200C000020311B002018
:10D1A800321B002030B50E4D0E4C2A7823789A4257
:10D1B80085B011D0684602A9FFF7DCFE002302A95A
:10D1C80002226846FFF746FFFFF7BCFE20782B785F
:10D1D8001B1A5842584100E0012005B030BD00BF7D
:10D1E800321B0020311B002038B50E4C4FF48055FF
:10D1F80045F20820FFF71EFF2585062001F096F866
:10D20800094BA56101221A70C720258501F08EF807
:10D21800064AA56100231370054A1370054A136076
:10D2280038BD00BF000400483D0D0020311B002020
:10D23800321B0020400D0020F7B503238DF8043081
:10D24800030C8DF805308DF80700030A06200F46F9
:10D2580014468DF80630FFF7EDFE78B1084D4FF40F
:10D26800805601A904222E85002001F087F838464F
:10D278000021224601F082F8AE61204603B0F0BDDD
:10D288000004004810B5D42000F07EFE802000F095
:10D298007BFEA82000F078FE3F2000F075FED3202A
:10D2A80000F072FE002000F06FFE402000F06CFEDF
:10D2B8008D2000F069FE142000F066FEA12000F029
:10D2C80063FEC82000F060FEDA2000F05DFE122048
:10D2D80000F05AFE812000F057FECF2000F054FEE7
:10D2E800D92000F051FEF12000F04EFEDB2000F0C6
:10D2F8004BFE402000F048FEA42000F045FEA6208A
:10D3080000F042FEAF2000F03FFEA62000F03CFEF9
:10D31800AE2000F039FE202000F036FE002000F09C
:10D3280033FEB02000F030FE402000F02DFE00203B
:10D3380000F02AFE102000F027FE4FF48064013C24
:10D348000020A4B200F01BFE002CF8D1812000F0D0
:10D358001BFEC82000F018FEAF2000F015FE0120CB
:10D3680010BD70B500EB8000094CA0F1A1059C38F8
:10D3780025440444074B15F8010F1E78704000F04F
:10D38800FEFDA542F6D13046BDE8704000F0F7BD7D
:10D39800F4520108E52A002010B5441E14F8010FC4
:10D3A80010B1FFF7DEFFF9E710BD08B55038C0B27D
:10D3B80000F0EAFD002000F0E7FD1020BDE808407D
:10D3C80000F0E2BD0846FCF7D7BB0F4B1A786F2A6E
:10D3D80017D1598840F2DC72914212D11A79BE2ACB
:10D3E8000FD193F8D827EF2A4FF000000BD113F88C
:10D3F800012B5040054A9342F9D1B0FA80F0400918
:10D40800704700207047704700F00308DCF70308F6
:10D418002DE9F04F2DED028BF14C85B0002140F243
:10D42800DC72204606F049F9EE4B04F538721A60B2
:10D43800ED4B00261E70ED4B04F2AA721A606F23A2
:10D448002370012003236371FCF744F80220FCF7E2
:10D4580041F84FF48070FCF73DF820224FF4167322
:10D4680084F868216E22A4F8643184F87A21FA23BA
:10D478000A22A4F8663184F87B214FF4FA732B2230
:10D48800A4F86C3184F87D210123212284F85E31CF
:10D4980084F8693184F86A3184F87C3184F87E2113
:10D4A80084F884312322002384F87F21C4F81432BD
:10D4B800C4F818324FF4C872052384F8A867A4F892
:10D4C8007061A4F86E61A4F8726184F8556184F8FB
:10D4D800566184F85761A4F85861A4F85A61A4F811
:10D4E8005C6184F85F61A4F88261A4F88021A4F8E3
:10D4F800866184F8116284F8106284F81C6284F8EA
:10D508001D6284F81F3240F2DC53A4F8963140F2D1
:10D518004C43A4F8983140F26C73A4F89A3140F265
:10D528007533A4F89C3140F64303A4F89E3184F87F
:10D538001E6284F8906184F8916125462346032E83
:10D54800CCBF0122002206F1010683F8A02114BFF6
:10D558001E220522122E83F8A12103F10203EED127
:10D5680040F27E42A4F8402140F23A724FF4FA6346
:10D57800A4F8422140F27E52A4F8C631A4F8CA3178
:10D58800A4F8CE31A4F8D231A4F84821052340F2FA
:10D59800EA5284F8E031A4F84A21C82340F2B45290
:10D5A800002601274FF47A7B4FF01E0840F2DC502A
:10D5B8004FF0190AA4F8E431A4F84C214FF4C873C9
:10D5C8003222A4F8E831A4F846010390A4F84E21C9
:10D5D800A4F8503184F8938184F8DF7184F8E1A1CC
:10D5E80084F8E27184F8E37184F8E67184F8EC71E8
:10D5F80084F8926184F89461A4F8C4B1A4F8C8B11D
:10D60800A4F8CCB1A4F8D0B184F8D46184F8DE6170
:10D6180084F8EA61A4F844B1A4F85221029284F88B
:10D62800546101F02DF8DFF8BCC12673DCF8003036
:10D63800029A83F80B804FF05F0E83F803E04FF0F7
:10D648000F0E83F805E04FF0220E83F806E04FF046
:10D658000E0E83F810E04FF0350E83F81AE04FF005
:10D66800210E83F811E04FF0530E83F81BE04FF0C2
:10D678005A0E83F808E04FF0780E83F80AE04FF06E
:10D688002D0E4FF02809142183F80C8083F807A089
:10D698004FF00A084FF0640A83F814E04FF4FA7E5A
:10D6A800CDF804C01F70597599755A731A719F7710
:10D6B80083F8019083F8029083F817809E731E7692
:10D6C800DE735E7683F8128083F81CA083F80990D5
:10D6D800A3F84EE0DFF830E1C3F838E0C3F83CE0E7
:10D6E800DFF828E1C3F828E0DFF824E1C3F834E0E4
:10D6F800DFF820E1C3F848E0DFED3D7A9FED3D8A91
:10D70800C3ED0B7A4FF04B0E83F84CE04FF4E17EFB
:10D71800C3ED0C7AA3F85CE0B7EE087AF1EE047A70
:10D728004FF0100E83F85EE083F8509083ED087A8E
:10D7380083ED097A83ED108AC3ED117A83F853607B
:10D7480083F8548083F8558083F8568083F857A06F
:10D7580083F858A083F859A083F85A60039884F88E
:10D76800AC274FF0460E042284F8B21784F8ABE7D2
:10D77800A4F8B40784F8AAA784F8AD6784F8B16759
:10D7880084F8AE6784F8AF6784F8B06783F86820D8
:10D79800152283F87420184A9A67184ADA67184AD3
:10D7A800C3F8802083F88470A3F86460A3F86660E7
:10D7B800A3F86260C3ED1B7A83F8709083F87190C8
:10D7C800104800F09DFFDDF804C0DCF800204FF49D
:10D7D800487382F8207182F81D6182F81E611BE08F
:10D7E800801D0020200F0020642700204C0F0020FF
:10D7F800CDCCCC3E000000009A99193FF6287C3F1A
:10D808003D0A773F417401088FC2F53C0000604033
:10D818006666663F0000404082F81F9182F82461E6
:10D82800A2F82231114684F8D68184F8D781A4F869
:10D83800D8B184F8DA61A4F8DCA167460E2303FBAB
:10D8480006236FF0170083F82501032083F82601CB
:10D858006FF02F0083F82701072083F828016FF065
:10D86800230083F82901052083F82A01642381F81D
:10D878002B3101365A2381F82C3181F82D31082EAD
:10D888004FF0FF0381F82E3101F10E01D6D10023AC
:10D8980082F895312D4B18EE102A45F8102F9D422D
:10D8A800F9D12B480021402205F007FF0023294D1C
:10D8B800294C59591A1904330868C2F8A002382BA0
:10D8C800F5D104F508700021802205F0F6FE05F177
:10D8D8003801702204F5087005F0E4FEFBF7B0F893
:10D8E8003E6800230125314604F58F604FF4CC7261
:10D8F80084F8D03784F8CE5784F8CF5705F0D2FE95
:10D9080004F5C26031464FF4CC7205F0CBFE134BE0
:10D918001B681A68C4F8B6275A68C4F8BA279A6800
:10D92800C4F8BE271A68C4F8C2275A68C4F8C627BC
:10D938009A68C4F8CA27022384F8D85484F8703641
:10D9480005B0BDEC028BBDE8F08F00BF401E002083
:10D958002020002098550108801D00204C0F002031
:10D968001549D1F8883043F47003C1F88830134B57
:10D978001A6842F001021A605868114A02405A6057
:10D988001A6822F0847222F480321A601A6822F42B
:10D9980080221A605A6822F4FE025A60DA6A22F07B
:10D9A8000F02DA62186B074A02401A6300229A6073
:10D9B8004FF000638B60704700ED00E000100240FC
:10D9C8000CC07FF8CCFC00FF38B5144B1B6898429C
:10D9D80005461ADD124B93F8D04714B1012C09D033
:10D9E80017E0104B1B68186988B1A842CCBF01200A
:10D9F800022038BD7F280CDCFFF7E8FAC0F17F0071
:10DA0800854208DDFFF7CEFB05E0002038BD012088
:10DA180038BD022038BD204638BD00BF402900204F
:10DA2800801D0020B8270020074B93F8D037012B22
:10DA380008D1064A064BD0681B68834234BF0020D1
:10DA48000120704700207047801D00200C00002036
:10DA5800400D002038B5094B93F8D05765B9084CEC
:10DA68002068F8F7D1FB074B25601B78022B03D100
:10DA7800BDE8384000F0C4BD38BD00BF801D00209F
:10DA8800B8270020B7270020064B93F8D0371BB1E2
:10DA9800012B05D1FFF786BB034B186801F074B85A
:10DAA80000207047801D0020B8270020F8B5011F0E
:10DAB80006460023083051F8042F02F120043F2CB9
:10DAC8003BD802F108040F2C06D80232032A04D9E5
:10DAD800002B08BF012300E002238142EBD1012B78
:10DAE80030680ED0022B1AD0736803F003039B0032
:10DAF80000F0030043EA0010B36803F0030318437F
:10DB080017E000F00F0040F04000FCF735F8B0686F
:10DB1800736800F00F0040EA0310C0B209E000F09B
:10DB28003F0040F08000FCF727F83079FCF724F834
:10DB3800307ABDE8F840FCF71FB806F10C07344608
:10DB48003A46002552F8043D03F18001FF294FEAC7
:10DB5800850510D903F50041B1F5803F02D245F0A3
:10DB6800010508E003F50003B3F1807F34BF45F0F9
:10DB7800020545F00305B242E4D165F03F00C0B2AA
:10DB8800FBF7FAFF05F00303022B207807D0032BDD
:10DB98000CD0012B13D1FBF7EFFF60780FE0FBF7F8
:10DBA800EBFF6078FBF7E8FFA07808E0FBF7E4FFFD
:10DBB8006078FBF7E1FFA078FBF7DEFFE07804343C
:10DBC800FBF7DAFFBC424FEAA505DBD1F8BD10B57B
:10DBD80004467F2C06D964F07F00C0B2FBF7CCFF67
:10DBE800E409F6E7E0B2BDE81040FBF7C5BF430023
:10DBF80083EAE070EBE72DE9F047314B93F8D03733
:10DC0800012B86B0074601D004464AE005F099FD8D
:10DC180003A9054606466846FFF7ACF9039B049A34
:10DC2800029713442B443F2B059519D900236846C6
:10DC380003A90322FFF70EFA039B3BB9049B2BB9F8
:10DC4800204A13705370059BABB301E0FFF77AF9D4
:10DC5800039B049A059E134433447F2B2BD8029FC1
:10DC6800DFF86090CA4639461AF8024BC4F18008BA
:10DC7800B04528BFB0460AEB04004444E4B242462B
:10DC880005F010FD802C89F8004014D1C8EB060679
:10DC9800504607EB0801324605F004FD89F800609C
:10DCA80009E0254614F8011B21B1074B186800F05C
:10DCB80074FFF6E7ED1B284606B0BDE8F08700BF05
:10DCC800801D0020311B0020B82700200FB437B575
:10DCD80006AC482054F8045BFBF74EFF2020FBF706
:10DCE8004BFF2A4623460B4901940020FBF7CEF947
:10DCF80004460A20FBF740FF074BC4F1FF241A68CB
:10DD080004F57F04FD3414441C6003B0BDE83040C2
:10DD180004B07047CDD30008402900200FB407B5E0
:10DD280004AB064953F8042B01930020FBF7AEF926
:10DD380003B05DF804EB04B0704700BFCDD3000812
:10DD4800054B1A7802F0FF0122B10122027000226D
:10DD58001A70704701707047B41B002037B5104B1C
:10DD680004465D68187806216A46A847A8B19DF858
:10DD780000209DF8013043EA022323809DF8022009
:10DD88009DF8033043EA022363809DF804209DF840
:10DD9800053043EA0223A380012003B030BD00BF51
:10DDA800D409002013B5104B04465B683B200621BC
:10DDB8006A469847A8B19DF800209DF8013043EACB
:10DDC800022323809DF802209DF8033043EA0223B2
:10DDD80063809DF804209DF8053043EA0223A38060
:10DDE800012002B010BD00BFD4090020094B0A4928
:10DDF8001B681B6923F01F0010B50122445803F06B
:10DE08001F0302FA03F31C421EBF4350034B1A7050
:10DE180010BD00BFE009002014040140B41B00201D
:10DE280003460A4668201946F7F7AABDF8B52F4DEC
:10DE38002F4C06464FF420432868636087693F04E7
:10DE480004D51F46013B002FF8D111E04768294B44
:10DE58003B4043F4903343F0D00343604FF42043F6
:10DE680063608769BF070AD41F46013B002FF8D1BA
:10DE78006360F7F773FD003018BF0120F8BD4FF459
:10DE88002043866263608669770604D41E46013B98
:10DE9800002EF8D1ECE76360164E43681E40164B1F
:10DEA800334343EA014343604FF4204363602868E7
:10DEB80059B1866976070CD41E46013B002EF8D16D
:10DEC800D6E71A46013B002AD2D082699206F8D5D5
:10DED80006E063600139436A02F8013BC9B2E3E72F
:10DEE80063602023C3610120F8BD00BFD40E002069
:10DEF800B41B0020009800FCD02400022DE9F0415A
:10DF08000369C76805460E461F40002F35D0B7FA8B
:10DF180087F24FF00043D340DB432B611F40A2F14F
:10DF28001B03042BF1D8DFE803F0221F1C190300A0
:10DF3800746A24B1013C0023A4B2736201E0EC6A64
:10DF4800A4B2D6F82080B8F1000FDED0D8F800309F
:10DF5800404621469847D8F80480F4E73068696B52
:10DF680007E07068A96B04E0B068E96B01E0F0684D
:10DF7800296C036889B29847C7E7BDE8F081024673
:10DF880040213C20F7F7FCBC024680213C20F7F7F3
:10DF9800F7BCF0B5364D2B7A85B0002B66D1354CE1
:10DFA8002368002B62D01A68334E12B171690A4394
:10DFB80072619A889868ADF80020694602220027A5
:10DFC8008DF803208DF80270F7F7B2FBB36921686A
:10DFD80043F00103B3610B7D0E7B03F0030203F0F2
:10DFE800FC0303F1804303F58033920098684FF0F7
:10DFF8000F0E0EFA02FE20EA0E009860986806FAE4
:10E0080002F202439A601D4B4A7D596819B138469D
:10E0180000F072FD02E01A4959601A70226813690B
:10E02800012623F01F0103F01F0306FA03F0154B26
:10E03800C8501369029308230DEB030000278DF8DD
:10E048000D308DF80C708DF80E6000F017FA23680B
:10E058008DF806705B7D8DF8043001A803238DF8D8
:10E0680005308DF8076000F0BFF92E7205B0F0BDDD
:10E07800B41B0020E009002000100240D025002039
:10E08800F5DD0008140401400148024936E700BFE5
:10E0980000480140BC260020014802492EE700BF85
:10E0A80000400140942600200148024926E700BFAD
:10E0B800000400406C2600204FF0804000491DE716
:10E0C800442600200148024918E700BF002C0140FF
:10E0D8001C2600200148024910E700BF002C01401F
:10E0E8001C260020224B10B5224C5A43224BB3FB6E
:10E0F800F2F203880139013AA04289B292B29BB286
:10E108000ED004F50064A0420AD0B0F1804F07D0C9
:10E11800A4F59834A04203D004F58064A04202D14B
:10E1280023F070039BB2154CA04206D004F580641E
:10E13800A0421CBF23F440739BB203800D4BC16205
:10E14800984202850FD003F5006398420BD003F57F
:10E158004063984207D003F58063984203D003F5E3
:10E168008063984201D1002303860123436110BDD7
:10E1780040420F00002C014000A24A040010004059
:10E188000E4B800A984216D007D8B0F5801F0CD0E5
:10E198004A3B98420DD102207047094B984206D05D
:10E1A8000233984205D104207047012070470320AC
:10E1B8007047FE2070470020704700BF4B001000DA
:10E1C80050001000F8B50468064620460F4615466C
:10E1D800FFF7D6FF04284BD8B27A910847B9022333
:10E1E8008B40D4F80CE0DB439BB203EA0E03E360F8
:10E1F8000A23204A03FB001342F82370043342F831
:10E20800235015463FB1B17AE268890802238B4052
:10E218009BB21343E360282202FB00522032EFF343
:10E228001286502383F3128803B203EB8303DB00C7
:10E2380003F10C011C3329442B4451F8047F17B116
:10E2480017600A6804329942F7D100231360F3B2C9
:10E2580083F31188282303FB0050036A1BB1E3688A
:10E2680043F0010303E0E2684FF6FE731340E360F6
:10E27800F8BD00BF1C2600200148FDF719B900BFF2
:10E28800C01B00200148FDF713B900BF141C002073
:10E298000148FDF70DB900BF681C002020B9034BE9
:10E2A8001B6808221A82704701487047BC1C00206E
:10E2B8007400002020B9034B1B6808221A8270479B
:10E2C80001487047BC1C00207400002021B90128B7
:10E2D8008CBF0220002070470220704710B5094B00
:10E2E8001A68D378042B0BD8074C518ADB002344D7
:10E2F80018B99B895B1A138210BD9B68581810BD0A
:10E30800002010BDBC1C002074000020054B1968BB
:10E31800054B4A8A18B99B8D9B1A0B827047986ADD
:10E3280010447047BC1C00207400002040F2E93300
:10E338000F4A1289920704D4013B9BB2002BF7D1F4
:10E348000BE00C4A40F2E933107009490989C90702
:10E358000AD4013B9BB2002BF7D1074A93880133BB
:10E368009BB29380FF2070471078C0B2704700BFFF
:10E37800003800400C380040BC1C002030B5174B5A
:10E388009B894FF47A733AB311B10D78013107E0E4
:10E39800FF2505E0013B9BB24FF6FF74A3420FD067
:10E3A8000E4C2489A407F5D50D4C25700B4D2D89ED
:10E3B800ED070BD4013B9BB24FF6FF75AB42F5D18D
:10E3C800084A938801339BB2938005E0247808B10A
:10E3D80004700130013AD6E7012030BD0038004012
:10E3E8000C380040BC1C00200C4B0D49DA684378FF
:10E3F800D243C2F30222C2F10402934002781B0105
:10E408000A44DBB282F8003303780122580903F08A
:10E418001F0302FA03F341F82030704700ED00E0D3
:10E4280000E100E073B50546002100680122FFF70E
:10E4380059FE2A6813889BB243F001031380EB7AD4
:10E448008DF804300124002601A88DF805408DF8C8
:10E4580006608DF80740FFF7C7FFEB7A1B2B0BD13F
:10E46800192301A88DF804308DF805408DF8066051
:10E478008DF80740FFF7B8FF02B070BD036823F0BE
:10E488001F0202F1804202F5823270B503F01F01CB
:10E498001468012303FA01F124EA010111600268FA
:10E4A8002A4C22F01F0502F01F02295903FA02F232
:10E4B80021EA02022A510279016802F1804221F020
:10E4C8001F0402F5823201F01F01155903FA01F108
:10E4D8002943115102681E4D22F01F0402F01F0249
:10E4E800615903FA02F221EA020262510268194CE8
:10E4F80022F01F0602F01F02315903FA02F221EA44
:10E508000202417932511029026812D122F01F010A
:10E5180002F01F024E5903FA02F232434A510268CE
:10E5280022F01F0102F01F020859934003430B51C8
:10E5380070BD01F1804122F01F0001F5823102F027
:10E548001F020C58934023430B5070BD0404014034
:10E55800080401400C040140104B10B50446185C37
:10E56800FEF7FFFE0E4800EB4400B0F90610B1F5C7
:10E578007A7F05DBB1F5FA6FA8BF4FF4FA6101E0C5
:10E588004FF47A71A1F57A710A23092091FBF3F10E
:10E59800BDE81040C9B2F9F725BF00BF4E740108A5
:10E5A800BC1C0020031EB8BF2D2210B5B8BF5842AE
:10E5B8000C46B8BF01F8012B0A22FAF753FD0023D5
:10E5C8000370204610BD10B50446B0F90000FFF7EF
:10E5D8000EFBB4F90200FFF70AFBB4F90400BDE82A
:10E5E8001040FFF704BB10B504460068FFF7FFFAB8
:10E5F8006068FFF7FCFAA068BDE81040FFF7F7BABB
:10E608002DE9F74F0120F7F7EFFF002488B3012C1D
:10E618002FD8194E4FF04C0909FB04FA06EB0A08EB
:10E6280008F17407BD7815B10134E4B2EEE790F94A
:10E63800003090F804E01846104B03228DE82400BF
:10E6480001212A4653F82E30F7F7F2FD834660B1D0
:10E6580006F12C00504429464A4605F02EF80123BD
:10E668001C44C8F82CB0BB70E4B20120F7F7A0FF37
:10E67800CCE703B0BDE8F08FBC1C00205C56010855
:10E6880008B522221148002105F017F8104B002286
:10E6980010490420515C83F8F0110132052183F8F8
:10E6A800F501042A4FF0000083F8F41183F8F7010C
:10E6B80083F8F61103F10803EAD1074B0122A3F806
:10E6C800B622522283F8B22208BD00BF6E1F002076
:10E6D800801D00204A740108BC1C002010B5F8F702
:10E6E8004DFB4FF43024012806D11CB1F8F746FB46
:10E6F800013CF8E7052010BD002C08BF052010BD1F
:10E7080070B50646441E14F8011F89B1094D284604
:10E7180005F009F80028F6D005F1080398423FBF34
:10E72800054B401BC018A31B38BF80F84C32EAE7E2
:10E7380070BD00BF4E740108BC1C002007B51C4BFF
:10E7480003F6A402C3F8A02893F854225AB1012A68
:10E7580014D1032183F8A618072183F8A82883F881
:10E76800A7180C2208E0022183F8A618032183F8D1
:10E77800A82883F8A718072283F8A4280D4B0E4A67
:10E788001A634020F7F730FF70B10122002390F997
:10E79800000040218DE80C00084A4FF4E133F7F7F8
:10E7A80047FD003018BF012003B05DF804FB00BF2F
:10E7B800BC1C002074000020296800085569000866
:10E7C8000120002100F074BDF0B5184A92F8A9386C
:10E7D800D2F8AC781546032B11D807EBC3025E1CA0
:10E7E800941CF6B209D013469288D10705D5104279
:10E7F80003D008E00131042908D13346EBE785F856
:10E80800A9380020F0BD93F802E00021074C0C2243
:10E8180004F50B6C02FB01F31CF803209645E9D1C3
:10E82800234484F8A968D3F8B408F0BDBC1C0020C0
:10E838000B4B10B519684FF6FB720A401A60094A6B
:10E8480092F8EA281C46084B0AB1052200E001228A
:10E858001A60FFF785F84FF43643236010BD00BFF8
:10E86800405C0040BC1C0020C82A00204FF09043A8
:10E87800012208B19A6170471A8570474FF090439A
:10E88800012208B11A8570479A61704710B544781B
:10E898000078002202FB02F3193B634303F6C4131A
:10E8A800534340F6C411434393FBF1F3034921F862
:10E8B80012300132072AEDD110BD00BFBC2500205F
:10E8C8000430114B33F91000B0F5617F10B506DB49
:10E8D80040F6330398420246A8BF1A4601E04FF4B7
:10E8E80061720C78192340F2833013FB04049442BC
:10E8F80007DA497813FB01039342B4BF00200120D3
:10E9080010BD002010BD00BFC21C002010B500F1D2
:10E91800500302788A4203D18478C278944204D39F
:10E9280004309842F5D1002010BD012010BD0B4BDA
:10E938001B6813F4805F0A4BB3F9063005D0C08911
:10E94800421A934207DD084400E0008A8342B4BFBC
:10E958000020012070470120704700BF842A002052
:10E96800C21C00201FB5094B1B681B030AD58DF874
:10E97800040001230D2001A98DED030A8DF805304F
:10E98800FBF79EF905B05DF804FB00BF842A002060
:10E998001FB5084B1B681B0309D58DF804000291AD
:10E9A80000230D2001A98DF80530FBF789F905B082
:10E9B8005DF804FB842A002010B50A4A0A4B116846
:10E9C8009B6800BF12689142F7D1084A14694FF456
:10E9D8007A7000FB04F2D31AB3FBF4F300FB0130A6
:10E9E80010BD00BF902A002010E000E0BC250020E8
:10E9F80038B5044654B1FFF7DFFF0546FFF7DCFFE3
:10EA0800401BB0F57A7FF9D3013CF3E738BD024AE1
:10EA18001368013313607047902A0020044A9369F1
:10EA280023B192F91420282A00D11847704700BF53
:10EA3800BC250020014B1B68184700BFCC2A0020CA
:10EA480010B50020FFF7F6FF054B00241C7001F0FD
:10EA580031FD044B1C771C629C849C6210BD00BF76
:10EA6800B82A0020BC25002010B5E0B1124B1B6865
:10EA780013F0020304D0114B1B78012B13D9002388
:10EA88000C225A430E4C1119125D824203D00133F5
:10EA9800102BF5D110BD0B4B986A38B14A784078E5
:10EAA800824203D310BDBDE81040C9E70022996235
:10EAB8009A841A6210BD00BF842A00200801002031
:10EAC8001C570108BC25002010B540001428A8BF19
:10EAD80014200023074A022199540B44991814243E
:10EAE800834201F8014CF5DBFF21D1540F20BDE82A
:10EAF8001040B9E79C2700202DE9F84307460B246E
:10EB0800013C35D01D4B20229A617D1C32264FF0E6
:10EB18000508DFF86890B9F814309BB283F0200339
:10EB2800A9F814300120FFF785FF3046FFF760FF92
:10EB3800B9F814309BB283F020030020A9F81430F0
:10EB4800FFF778FF3046FFF753FFB8F1000F08D002
:10EB5800B8F10108DDD14FF4FA70FFF749FFFA2642
:10EB6800D7E7013DD5D14FF47A70FFF741FFC7E7EA
:10EB7800034B044ADA60BDE8F88300BF000400488C
:10EB880000ED00E00400FA0503685B6918470368B4
:10EB9800DB68184703685B68184703681B681847F1
:10EBA8002DE9F84FB0F90230934218BF00232DED3C
:10EBB800048B18BF0370057804460E469146002D55
:10EBC80040F0978007EE902ADFED7D8AF8EEE77A2D
:10EBD800B6EE009A67EEA88ADFED7A7A68EEA78A21
:10EBE800A04668EE898A2746B0EE680AFAF7E2FB83
:10EBF800B0EE408AB0EE680AFAF73CFC88EE000AEC
:10EC080040F2DC5363651023A4F852301823A4F8AB
:10EC18005030DFED6D6A60EE266AB7EE006AB0EE3E
:10EC2800667AA0EE007AD0EE006A37EE067A76EEC3
:10EC3800866AC6EE077A84ED046A27EE807AB0EE1B
:10EC4800498A27EE007A77EE075A84ED017AC4EDF7
:10EC5800025A70EE005A84ED037AB8EE007AA5EEF7
:10EC6800807A27EE877A67EEA67A84ED057AC4ED76
:10EC7800067ADFED567A98ED047A27EE277AF0EED9
:10EC8800678AB5EEC07AF1EE10FA4CBF77EE487A93
:10EC980077EE087A013517EE900A01F06FFED8ED8D
:10ECA800017A67EEA87AC7E90E01F5EEC07AF1EEAF
:10ECB80010FA4CBF77EEC87A77EE887A08F1040824
:10ECC80017EE900A01F05AFE032DC7E9080107F173
:10ECD8000807CED1A6F2DC531B042367E3676367FA
:10ECE800C4F88030A367C4F884300123A4F80290E4
:10ECF8002370D4F85490B4F95280636A276A206F5D
:10ED0800E26FD4F840C0D4F88010C4F88020C9EB72
:10ED1800060606FA08F64FEAE67B734307FB0B3351
:10ED28002667A7FB06671F44636C656F60674FEA39
:10ED3800E27B53430CFB0B3EACFB02237344B61A35
:10ED480067EB0307E36AA26AC4F884104FEAE07B22
:10ED5800434302FB0B3EA2FB00237344B6185F41FA
:10ED6800E36CA06CB4F95020A5674FEAE17B4B43F4
:10ED780000FB0B33A0FB01011944636B361A206BAF
:10ED88004FEAE57B05FB03F300FB0B3367EB010759
:10ED9800A0FB050119448019794101F0BDFB08F178
:10EDA800FF3201239340E067C01841EBE37142460C
:10EDB80001F0B2FBBDEC048B4844BDE8F88F00BFFE
:10EDC8006F12833ADB0F4940F404B53F0000804BD3
:10EDD8002DE9F8430024234B93F85C60E0B2B0427D
:10EDE8000CD203EB8003204ADB6A32F810101BB107
:10EDF8000B2801D8DB6898470134ECE71B4B1B68EC
:10EE08005B032DD500242346E2B2B24228D2DFF8B4
:10EE1800549009F12C074FEA840857F824205568C4
:10EE28009D4215D02846FFF7ABF9EFF31283502225
:10EE380082F3128828216A6A01FB00900132C0F827
:10EE480084206A6942F001026A61DBB283F31188A7
:10EE580057F808301B6800221A6001342B46D3E7A4
:10EE6800BDE8F883BC250020240F0020842A002058
:10EE780008B50E4B1B6813F4805F0D4B14BFD3F815
:10EE88002821D3F82C2193F85C1092880023D8B25B
:10EE9800884204D2074820F813200133F7E7FFF728
:10EEA80097FF3220BDE80840A2E500BF842A002071
:10EEB800BC250020240F00200A4B1A680A4B30B5E5
:10EEC80002F48052D3F82841D3F82C5100230AB118
:10EED800A18800E0A988054820F8131001330C2BFD
:10EEE800F5D130BD842A0020BC25002066270020EB
:10EEF80070B5124D0024214605F23110702285F8B4
:10EF0800304104F0DAFB2146D5F8A4310B4A0B4412
:10EF180093F9020080B102F231141E680E510819EB
:10EF28009C8884809B79837192F830310731013352
:10EF3800702982F83031E7D170BD00BFBC250020B0
:10EF4800094B1A680E2303FB0020437AFF2B07D0D6
:10EF5800064A12789A4203D9054A32F8130000E0AB
:10EF6800808800B2704700BFCC12002060250020C6
:10EF7800C21C0020D0ED024A91ED016A90ED015AC1
:10EF880091ED027AD0ED005AD1ED007A66EE646A0E
:10EF9800E5EE076A27EE657AC2ED006AA4EEA77A65
:10EFA80067EEC57A82ED017AE5EE867AC2ED027ADD
:10EFB8007047D0ED017A91ED017AD1ED026A91EDB9
:10EFC800006A37EE877AD0ED027A77EEA67AD0ED2E
:10EFD800006A82ED017A76EE866AC2ED027AC2EDA7
:10EFE800006A704790ED017AD0ED027AD0ED006AA0
:10EFF80020EE077A60EE277A26EE800A81ED017A04
:10F0080081ED000AC1ED027A704700BF07B5064BD3
:10F018000093064B01930649064A074B0748FAF73F
:10F0280037F903B05DF804FB636501083B65010827
:10F0380004730108FD72010857650108637401082B
:10F0480008B5037833B90C4B0C481978BDE808406B
:10F05800FAF71EB904F0CCFB02280CD8064B18703E
:10F06800074B0C2202FB0030064B02301860FAF7FF
:10F07800FDFA0548E5E708BD642700208974010802
:10F08800282500204C0F00207467010808B5037874
:10F098003BB90B4B0B4893F8A817BDE80840FAF7A3
:10F0A800F7B804F0A5FB022808D8054B83F8A80791
:10F0B800FAF742FAFAF7FEFA0348E8E708BD00BF94
:10F0C800801D00208D7401087467010838B5037825
:10F0D80003BB214B1B6801330F2B07D81F490C2298
:10F0E80002FB03121C4695682DBB00E01C46013448
:10F0F8000F2C01DD002400E005D818490C2202FB82
:10F1080004129568BDB99C42F1D11548BDE8384054
:10F11800FAF7BEB804F06CFB0F28044605D80F4A6E
:10F128000C2303FB00239D682DB921460D48BDE83B
:10F138003840FAF7ADB8084B1C60FFF781FC214650
:10F148002A460948FAF7A4F80C235C43034B185DD8
:10F15800BDE83840FFF788BCC40000201C570108F0
:10F168009A740108B0740108C874010873B503786B
:10F1780013B9F6F717FD3DE01F4901AA04F099FB02
:10F18800002401462646254699B134B1012C08D100
:10F19800084604F02DFB064603E0084604F028FB69
:10F1A80005461549002001AA04F083FB01340146F5
:10F1B800EAE70B2D02D911480C220BE0022C10D1E2
:10F1C800A6F57A73B3F57A7F07D90D484FF47A71AB
:10F1D8004FF4FA62F6F763FC0CE00A4B03EB4503C5
:10F1E8005E80084B084803EB45032946B3F9022023
:10F1F800FAF74EF802B070BD376C0108946901083F
:10F208000270010864270020DF74010838B50D4C2E
:10F2180023688342054606D1F6F7F6FF204600210B
:10F228004C2204F04AFAE36CAB4209D12846F6F7BF
:10F23800EBFF054800214C22BDE8384004F03DBAF8
:10F2480038BD00BFE81C0020341D0020034BDA69DC
:10F25800D379591C1344D171187A70476427002058
:10F2680010B5FFF7F3FF84B2FFF7F0FF04EB0020BF
:10F2780080B210BD10B5FFF7F3FF0446FFF7F0FFAB
:10F2880004EB004010BD38B5054D04462146286AF8
:10F29800FFF783FCEB6998796040987138BD00BF2F
:10F2A80064270020014BDB699879ECE7642700208C
:10F2B80038B5044624200D46FFF7E5FF4D20FFF73B
:10F2C800E2FF002C084C14BF21203E20FFF7DBFF93
:10F2D800E369002228469A71FFF7D5FFE36993F89E
:10F2E8004900BDE83840CEE76427002001460020E9
:10F2F800DEE710B50446C0B2FFF7C5FF200ABDE837
:10F308001040C0E710B5044680B2FFF7F2FF200CAA
:10F31800BDE81040EDE737B58288836804461006DB
:10F328000D4641BF2B4991F8A8174FF4CC7000FB4C
:10F338000133D10544BF2849097802F03F0244BF90
:10F3480001EB410103EB8103042A12D006D8012AFC
:10F358000DD0022A32D193F9001030E0102A0AD0D9
:10F36800202A0AD0082A29D1B3F9001027E01978F1
:10F3780025E0198823E0196821E093ED000A684622
:10F38800F9F706FE01461548F9F782FF05B3D4EDF3
:10F39800037A6846B8EEE70AF9F7FAFD014610481D
:10F3A800F9F776FF94ED040A6846B8EEC00AF9F753
:10F3B800EFFD01460A48F9F76BFF09E0002109480B
:10F3C800F9F766FF25B10848E1682269F9F760FF97
:10F3D80003B030BD801D002064270020B16A0108F9
:10F3E800AA6A010895730108EE740108024B0146E8
:10F3F800586AFFF7D2BB00BF6427002010B5441E2F
:10F4080014F8011F21B1034B586AFFF7C6FBF7E751
:10F4180010BD00BF6427002010B503781BB90A4847
:10F42800BDE81040EAE704F0E3F90446082899BF6C
:10F438002146064806480821F9F72AFF601EC0B28F
:10F44800BDE81040F6F77CBEF57401083C7501086C
:10F45800687501082DE9F3412B4E2C4B96F82800CE
:10F468002B4D1C682B4B05EB80001A882A4BD0F8D3
:10F47800C0101B78294800914FF47A71B4FBF1F160
:10F48800F9F706FF26484821F9F702FF254BD3F87C
:10F4980000800027FBB205EB8302D2F8D010E9B157
:10F4A80001249C4014EA080F16D0220714D01E4AE3
:10F4B800D25C0B2000FB0323154A1C4802EB830394
:10F4C800D3F8F020F9F7E4FE022C05D196F83410B1
:10F4D80011B11748F9F7DCFE0137DBE71548FFF7EC
:10F4E8008DFF154B15481A68154B9A420CBF154BE2
:10F4F800154B1A88154B198892B240F2DC7302B08A
:10F50800BDE8F041F9F7C4BE64270020902A002026
:10F518001C57010888120020080100209375010873
:10F52800D6750108DC0E002004010020E6750108EC
:10F53800EE75010836760108D40E0020F275010830
:10F5480000540040D80E0020DA0E0020D00E002013
:10F558002DE9F0410024804625460F4EA759414623
:10F56800384604F02DF958B139460C48F9F790FEA1
:10F5780030190021FFF7CFFE0948FFF73FFF01359B
:10F58800143440F6CC339C42E7D11DB90548BDE898
:10F59800F04133E7BDE8F081BC580108476B01082A
:10F5A80036760108EB6901082DE9F04F2DED028B45
:10F5B80083B0054604F0C5F8064620B1012818D1E5
:10F5C8002B782A2B15D15C48FFF718FF00245B4DD8
:10F5D8005B486159F9F75CFE28193146FFF79BFE35
:10F5E8005848FFF70BFF143440F6CC339C42EED159
:10F5F8009CE028463D2104F096F8002800F08F8012
:10F608000346994613F8012D202AFAD0441C2046B7
:10F6180004F0EEF880462046F9F730FCC5EB0909FE
:10F62800B0EE408A0026DFF834A1142202FB06F46B
:10F638000AF5D07B54F80B70384604F082F803467C
:10F648001A4628463946019304F084F8019B00289D
:10F658005BD15FFA89F29A4257D10AEB0402D2EDE4
:10F668006B7AF8EEE77A0BEB0405B4EEE78AF1EE75
:10F6780010FA48DBD2ED6C7AF8EEE77AB4EEE78A56
:10F68800F1EE10FA3FD8B2F8A431D2F8A82113F05D
:10F69800200F08BF08EE108A1C0641BF2A4991F8BE
:10F6A800A8174FF4CC7404FB0122D90544BF27499D
:10F6B800097803F03F0344BF01EB410102EB8102EB
:10F6C800042B18EE100A0BD004D8013B012B0ED8DE
:10F6D80010700CE0102B05D0202B06D0082B06D17B
:10F6E800108004E082ED008A01E082ED008A39464C
:10F6F8001748F9F7CDFD2846002103B0BDEC028B71
:10F70800BDE8F04F07E6134803E00136972E8AD18B
:10F71800114803B0BDEC028BBDE8F04F6EE62846F9
:10F7280003B0BDEC028BBDE8F04F11E703B0BDECB0
:10F73800028BBDE8F08F00BF24760108BC58010891
:10F74800476B010836760108801D002064270020D9
:10F758003976010844760108EB6901081C5701084D
:10F7680010B50A48FFF74AFE094B5C6A2046FFF7C6
:10F778000BFA18B90A20FFF73BF9F7E7FFF778FB10
:10F78800F9F7B0FE034B044ADA6010BD647601084D
:10F798006427002000ED00E00400FA0508B50548DC
:10F7A800FFF72CFEFDF734FEF9F7C6FEBDE808406A
:10F7B800D6E700BF7076010808B50448FFF71EFEBB
:10F7C800F9F7BAFEBDE80840CAE700BF8676010827
:10F7D8002DE9F04FAB490B7813F0010F85B003F01A
:10F7E800040200F04181002A40F06E81A6480768B3
:10F7F80017F0806740F06881980700F1358143F081
:10F8080004030B70A14BA24C1B882380A14BA24D73
:10F818001A6812F4002F984600F016819F4B80203A
:10F828001F70FEF7D1FF08B1FFF7F0FCA678012E94
:10F8380040F00A8195F8CE272AB1974B93F8CF3735
:10F848000BB19A4203D3012385F8CE370FE018464F
:10F85800114630B191FBF0FE00FB1E1E01467046BA
:10F86800F7E792FBF1F285F8CE2793FBF1F385F8E1
:10F87800CF3795F8D037012B82BF874B002283F80A
:10F88800D02795F8D097B9F1000F03D0B9F1010F3F
:10F898002ED036E08020F6F7A7FE824688B3802176
:10F8A800F6F77CFE9AF806207D4BE07053F822307C
:10F8B8009AF90000B3F5613F0CBF02220022022131
:10F8C8008DE806004A468021F6F7B2FC754B606069
:10F8D8001B684FF4FA7203EB4303B3FBF2F31BB15B
:10F8E800402BA8BF402300E00123237258B908E049
:10F8F8006D4BDB682BB1FEF797F810B940232372E4
:10F9080001E000239FE000211422684803F0D5FE9F
:10F91800674B236203F16C02D833A362654BD8F8B6
:10F9280000101B88A4F8703195F8923195F8CE979D
:10F93800614895F884A16262002B6B790390A3F16A
:10F94800190CC1F3C03818BF4FF00108DCF1000EE4
:10F958004EEB0C0E012B95F8CF37D0F800C008BF3E
:10F968004FF0010E9945554B1B780293C1F3400B9C
:10F9780028BF4FF0000901F4006138BF4FF00109BA
:10F98800721ED2B2531E132B37D8DFE803F00C0CCB
:10F998000C0C0C0C0C0C0A39397429397612121219
:10F9A800333973466AE0029B9342B4BF00230123B4
:10F9B80022E09CF80030022B0BD10CEB820353EDB4
:10F9C800027AF5EE407AF1EE10FA14BF0123002313
:10F9D80012E00CEB02035B79003318BF01230BE044
:10F9E80021B10AF1FF304342434100E00B4603F0E6
:10F9F800010343E04B4641E013B1012393401F4309
:10FA0800142E02D80136F6B2BAE7039BC4F8747113
:10FA1800186819218530FEF779FF0023C4F87C3176
:10FA2800A4F88031A4F88231C4F88C31C4F890313C
:10FA3800234BD4F888211B68C4F8943184F87801E2
:10FA4800C4F884210223A3701D4B95F8E0211B689C
:10FA58004FF47A7101FB02331A4A0520136005B08E
:10FA6800BDE8F04FFFF700B872BB012005B0BDE854
:10FA7800F04FFFF729B85B4600E04346002BBCD1A6
:10FA8800C0E700BFE02A0020E40E0020400F00205D
:10FA9800B4270020842A0020801D0020652500202E
:10FAA8005C560108480F00200C000020C0270020E9
:10FAB800E0270020FC110020200F0020182600203D
:10FAC800902A00203C0E002005B0BDE8F08F10B54C
:10FAD800154A1378590725D523F004031370134BDF
:10FAE8001B681B0319D5124CA378A3F10802012A3D
:10FAF8000BD8FF200021FAF7E3F80E4B1B68C4F877
:10FB08009431FDF7C1FF0A2306E0012B05D90A2B22
:10FB180003D0FDF79FFF0123A3700420BDE8104028
:10FB2800FEF7A2BF10BD00BFE02A0020842A0020F3
:10FB3800B4270020902A0020054B1968054B4A8AF3
:10FB480018B99B889B1A0B82704718681044704735
:10FB5800BC1C0020C8000020074B1B681B7803F062
:10FB68007F03212B06D100F0DF00022814BF0220FA
:10FB78000020704702207047BC1C0020212810B5C7
:10FB880008D1114B1B681B7803F07F03212B10D081
:10FB9800022010BD2028FBD10B4B0C4A1B681070AB
:10FBA8001B7803F07F03212B094B18BF00230BB9E7
:10FBB800EEE7084B044A12680024936154822046F9
:10FBC8009847204610BD00BFBC1C0020E62A002034
:10FBD800A5E20008BDE200087047034B1A78202A06
:10FBE80004BF00221A707047E62A0020014B042245
:10FBF8001A607047C82A0020034B9B7A13B1034B45
:10FC080005221A60704700BF9C250020C82A0020E2
:10FC18000D4B0E491A680E4B92B213445B000D4A05
:10FC28001B68C3F3090310B5136013689BB2013353
:10FC38005B1000229A4206D0074851F8044B20F87E
:10FC480012400132F6E710BD505C004020620040CF
:10FC58001E3000205029002054290020014B00228A
:10FC68005A647047502900202DE9F843664B674EC7
:10FC78001B68DFF8B881664A00254FF0C0099D72FD
:10FC880083F80990DD723560D8F8003023F4EC432E
:10FC980023F0700343F400739BB2C8F80030D8F81F
:10FCA800003023F4E04323F040039BB248F2800481
:10FCB80083F010032343C8F80030336812FA83F343
:10FCC8005B0040271A681F6033689BB203F100533A
:10FCD80003F540535B0028461A6880221A60D8F85A
:10FCE800003023F4F8731B051B0D2343C8F80030BC
:10FCF800484B93F83410F6F7E9FED8F80030464A36
:10FD0800464923F4804323F070039BB283F44053A5
:10FD18002343C8F80030136823F4EC4323F070033E
:10FD28009BB21360336811FA83F35B0003201968F0
:10FD3800C3F8009013683A4923F4E04323F04003E2
:10FD48009BB283F0200323431360136823F480439A
:10FD580023F0700323439BB21360536823F4EC43EE
:10FD680023F0700343F4C0639BB25360336811FA05
:10FD780083F35B0019684FF480711960536823F4AA
:10FD8800804323F0700323439BB25360536823F4EA
:10FD9800E04323F040039BB283F0200323435360E6
:10FDA800D8F80C301F4A23F4EC4323F070039BB2BD
:10FDB800C8F80C30336812FA83F35B0039461A68C6
:10FDC8004FF488721A60F6F781FED8F80C3023F4E5
:10FDD800804323F070039BB283F440532343C8F855
:10FDE8000C30D8F80C3023F4E04323F040031C43D4
:10FDF800A4B2C8F80C402846FCF7CDFB0A4B0122F8
:10FE08001A60BDE8F88300BFBC1C0020505C0040AD
:10FE180004300020C8000020045C004008300020A6
:10FE2800103000201C300020C82A0020005C004050
:10FE3800134A144B50681B68181810B5146808D07A
:10FE480011490822FCF793FB204610490422FCF7CD
:10FE58008EFB0F4B1A68002393720E4A0121116022
:10FE68000D4913604FF4E0500B6010600B480B60B5
:10FE78004FF43641A0F848101160094A136010BDCC
:10FE8800B0F7FF1FACF7FF1FAA000020BA00002040
:10FE9800BC1C0020405C0040445C0040502900200D
:10FEA800C82A0020024B4FF480221A60704700BF16
:10FEB800140401402DE9F04F2DED088BCB4D83B094
:10FEC800044601932B8813F0020F0AEE102AF7EE6E
:10FED800009A4CD0149BC648DE89B0F900309B1BB1
:10FEE80003F2F31740F2E632974203D8002BB8BF6B
:10FEF8005B4201E04FF4FA73B0F90220921B02F260
:10FF0800F31640F2E630864203D8002AB8BF5242C0
:10FF180001E04FF4FA7294F84C0058B39342B8BF1A
:10FF28001346C3F5FA7307EE903A9FEDB27AF8EEEE
:10FF3800E77A6423C7EE877A93FBF0F307EE103A6B
:10FF480077EEE97AB8EEC77AB0EE699AA7EE879AA3
:10FF5800F7EE006AB5EEC09AF1EE10FA0AD4B4EEE4
:10FF6800669AF1EE10FAC8BFB0EE669A04E0B0EEF9
:10FF7800699A01E09FEDA09AA04E01F10308A346FB
:10FF88004FF0000ABAF1020F18F8010F9C4F4FEA20
:10FF98004A09F2EE04AA0ED100F10A01B7F90400E9
:10FFA8009FED987A00FB01F307EE903AF8EEE77AB6
:10FFB800C7EE877A51E0B8EE4A7ADFED8E6A37F9F4
:10FFC8001A1087EE267A07EE901A1AEE103AF8EE13
:10FFD800E77A5B4227EE877A07EE903AF8EEE77AFF
:10FFE800B4EEE77AF1EE10FA08D4F8EECA7AB4EE75
:08FFF800E77AF1EE10FAD8BF20
:020000040801F1
:10000000F0EE477A824F37F909302F8807EE103A21
:10001000019BB8EEC77A33F91A3077EEC77A07EE4C
:10002000103AB8EEC77AFB0737EE877A87EE2A7A5E
:1000300004D5D4ED117A67EE277A12E0143001FB73
:1000400000F307EE903ADFED716AF8EEE77AB90750
:10005000C7EEA67A42BFD4ED126A27EE267AE7EE03
:10006000097A6C496C4F31F909306C499BED08BA3B
:10007000D1ED046A9FED6A8A07EE103AB8EEC77AAE
:10008000684BE7EE667A1AF80330BAF1020FF0EE29
:10009000678A67EE8B7A0BEE103AB8EECBBAF0EEC9
:1000A00048BA27EE8BBA8BEE08BA09D1B0EE4B0AEC
:1000B0005D48D7ED000A1E21F8F7BAFEB0EE40BA4F
:1000C000D7ED000A9BED0B7A68EEA07A67EE877A8F
:1000D00096ED007AA7EEAA7ADFED547AB4EEE77ACD
:1000E000F1EE10FAF0EE47AA09D4DFED517AB4EE42
:1000F000677AF1EE10FAC8BFF0EE67AA01E0F0EE01
:1001000067AA89EEA08A4B494FEA8A07394491EDE4
:10011000000AC6ED00AAC1ED008A38EEC00A94F8C4
:10012000501020EE080A21B1434800EBCA00F8F74E
:100130007FFE3C4BDBED0E7A13F80A3060EE277A37
:1001400000EE103AB8EEC00A27EE800ADFED3B7AE7
:1001500080EE2B8AB4EEE78AF1EE10FA09D4DFEDD7
:10016000387AB4EE678AF1EE10FAC8BFB0EE678A4B
:1001700001E0B0EE678A3BEE2A0A30EE080A03F08F
:10018000AFFC3049B0F57A7FA8BF4FF47A7088424F
:10019000B8BF08462C4921F8090029880A0507D567
:1001A0002A4909784B0703D55FFA8AF0F8F7A6FCCD
:1001B000BDEECBBA26491BEE103AFDEEEAAA7B5003
:1001C000BDEEC88A23491AEE903A0AF1010A7B5023
:1001D000214918EE103ABAF1030F7B500BF1040BD2
:1001E00006F104067FF4D2AE03B0BDEC088BBDE887
:1001F000F08F00BFE00E0020C21C00200000FA4378
:10020000000000003C13002080190020000048423C
:100210003C0F00200A0F002094190020F419002040
:100220000000C842881900208C19002000007AC301
:1002300000007A439C290020B0190020000096C3DA
:100240000000964318FCFFFFC8190020E02A002098
:10025000D0190020DC190020E8190020044B0022EE
:100260001A605A60034B00221A605A60704700BF40
:10027000681300204813002010B50B4C0123E370D5
:100280004FF48060022384F82030F9F70FF9074A11
:10029000074BD2681B685178642212FB01336361FB
:1002A00023880133238010BD942A00209C2900203C
:1002B000902A00200A4BDFED0B7A53F8213007EE2D
:1002C000103AB8EE477AF6EE046AE7EE267A82B084
:1002D000FCEEE77ACDED017ABDF8040002B070477C
:1002E000AC29002000005C44024B03EB4101B1F853
:1002F00048007047AC290020024B03EB4101B1F8E4
:100300006C007047AC290020024B03EB4101B1F8AF
:100310006C007047AC2900200020704738B50446B7
:10032000FEF74EFB274A2749D2F88430C2F88400F2
:10033000C31AB3F57A6F84BF002382F8883092F82D
:10034000883033B9A82C3BD181F88930A1F88A30A4
:1003500006E0022B02D181F88C4001E0242B02D868
:10036000D11881F88D4092F88C10164D013302316E
:10037000DBB249008B4282F8883018DAB5F88A304F
:10038000E0B283EA0020082310F4004F4FEA400057
:1003900018BF80F4815003F1FF3318BF80F00100D3
:1003A00013F0FF0380B2EFD1A2F88A0038BD01310B
:1003B0008B4201BF002385F88830012385F88930FE
:1003C00038BD00BFAC29002010B50446FEF7F8FA8E
:1003D000104AD2F8B43040F6AC51C31A8B42C4BFB5
:1003E000002382F8B83092F8B830D11881F8B940BB
:1003F00023B90F2C0DD10749C1F8B4000133DBB28A
:10040000192B044982F8B8300CBF0123002381F86E
:10041000D23010BDAC290020114910B5D1F8D4302C
:1004200003EB4002147E14B1022C10D00BE0022822
:1004300005D9032807D1D1F8D820D20401D5D8890D
:1004400010BD988A10BD074B33F8100010BD507EC8
:1004500000EB800000EB800000F2EE2080B210BDC7
:10046000AC290020C21C002008B5FEF7A9FA074BF2
:10047000022283F8E020D3F8E420C3F8F020012220
:10048000C3F8DC0083F8092108BD00BFAC290020B7
:1004900008B5FEF795FA084B022283F8E020D3F85E
:1004A000F02000F5B71000F5587002F2DC52C3F8E6
:1004B000DC00C3F8F02008BDAC290020104B93F8F5
:1004C0000C21012A10B51C460DD008D3022A0DD1EB
:1004D0000C4A938A9BB283F02003938206E0094B77
:1004E00020229A6102E0074B20221A85FEF768FA63
:1004F00000F5F42000F59070C4F8100110BD00BFA5
:10050000AC2900200004004808B5044B1B7803F018
:100510000503052B01D1FEF7AFFCFEE7C02A002042
:10052000D0400B1C1141203A03D49C461341184380
:100530006346524293401843704700BF81F0004128
:1005400002E000BF83F0004330B54FEA41044FEAB8
:10055000430594EA050F08BF90EA020F1FBF54EA53
:10056000000C55EA020C7FEA645C7FEA655C00F0EF
:10057000E2804FEA5454D4EB5555B8BF6D420CDDC0
:100580002C4480EA020281EA030382EA000083EA43
:10059000010180EA020281EA0303362D88BF30BDE3
:1005A00011F0004F4FEA01314FF4801C4CEA113139
:1005B00002D0404261EB410113F0004F4FEA033398
:1005C0004CEA133302D0524263EB430394EA050F23
:1005D00000F0A780A4F10104D5F1200E0DDB02FA92
:1005E0000EFC22FA05F2801841F1000103FA0EF226
:1005F000801843FA05F359410EE0A5F120050EF1EC
:10060000200E012A03FA0EFC28BF4CF0020C43FA1C
:1006100005F3C01851EBE37101F0004507D54FF029
:10062000000EDCF1000C7EEB00006EEB0101B1F579
:10063000801F1BD3B1F5001F0CD349085FEA3000BF
:100640004FEA3C0C04F101044FEA445212F5800FCA
:1006500080F09A80BCF1004F08BF5FEA500C50F167
:10066000000041EB045141EA050130BD5FEA4C0C4A
:10067000404141EB010111F4801FA4F10104E9D1D3
:1006800091F0000F04BF01460020B1FA81F308BFCA
:100690002033A3F10B03B3F120020CDA0C3208DD96
:1006A00002F1140CC2F10C0201FA0CF021FA02F171
:1006B0000CE002F11402D8BFC2F1200C01FA02F1E1
:1006C00020FA0CFCDCBF41EA0C019040E41AA2BF06
:1006D00001EB0451294330BD6FEA04041F3C1CDACE
:1006E0000C340EDC04F11404C4F1200220FA04F0EE
:1006F00001FA02F340EA030021FA04F345EA030198
:1007000030BDC4F10C04C4F1200220FA02F001FA59
:1007100004F340EA0300294630BD21FA04F02946DB
:1007200030BD94F0000F83F4801306BF81F4801174
:100730000134013D4EE77FEA645C18BF7FEA655CE7
:1007400029D094EA050F08BF90EA020F05D054EAB9
:10075000000C04BF1946104630BD91EA030F1EBFBE
:100760000021002030BD5FEA545C05D140004941C2
:1007700028BF41F0004130BD14F580043CBF01F5B5
:10078000801130BD01F0004545F0FE4141F470019B
:100790004FF0000030BD7FEA645C1ABF1946104676
:1007A0007FEA655C1CBF0B46024650EA013406BF77
:1007B00052EA033591EA030F41F4002130BD00BF36
:1007C00090F0000F04BF0021704730B54FF48064F3
:1007D00004F132044FF000054FF0000150E700BF74
:1007E00090F0000F04BF0021704730B54FF48064D3
:1007F00004F1320410F0004548BF40424FF00001C0
:100800003EE700BF42004FEAE2014FEA31014FEA02
:1008100002701FBF12F07F4393F07F4F81F0605151
:10082000704792F0000F14BF93F07F4F704730B5C0
:100830004FF4607401F0004521F0004120E700BF53
:1008400050EA010208BF704730B54FF000050AE0DA
:1008500050EA010208BF704730B511F0004502D5DB
:10086000404261EB41014FF4806404F132045FEADD
:10087000915C3FF4DCAE4FF003025FEADC0C18BF82
:1008800003325FEADC0C18BF033202EBDC02C2F178
:10089000200300FA03FC20FA02F001FA03FE40EA0A
:1008A0000E0021FA02F11444C1E600BF4FEA4102F2
:1008B000B2F1E04324BFB3F5001CDCF1FE5C0DD9BE
:1008C00001F0004C4FEAC0024CEA5070B2F1004F08
:1008D00040EB830008BF20F00100704711F0804F0B
:1008E00021D113F13872BCBF01F00040704741F4D0
:1008F00080114FEA5252C2F11802C2F1200C10FAD4
:100900000CF320FA02F018BF40F001004FEAC123B7
:100910004FEAD32303FA0CFC40EA0C0023FA02F35B
:100920004FEA4303CCE77FEA625307D150EA013331
:100930001EBF4FF0FE4040F44000704701F0004001
:1009400040F0FE4040F40000704700BF7BB972B930
:100950000029BEBF00204FF0004106E008BF00287C
:100960001CBF6FF000414FF0FF3000F073B882B051
:10097000EC462DE9005000F03DF8DDF804E002B04F
:100980000CBC704707EE900AF5EEC07AF1EE10FA53
:1009900001D400F009B808B580F0004000F004F878
:1009A000404261EB410108BDD0B5FFF72BFF0022AB
:1009B0000E4B06460F4600F04FF800F05FFA044673
:1009C000FFF7FEFE00220A4B00F046F802460B46F7
:1009D00030463946FFF7B6FD00F050FA23460022B4
:1009E00042EA000210461946D0BD00BF0000F03DAB
:1009F0000000F0412DE9F041069C154606460F46E1
:100A0000984600F05BFA05FB01F300FB0838A5FBF4
:100A10000023B21A434467EB0303C4E90023BDE893
:100A2000F08100BF2DE9F041069C904606460F4636
:100A30001D4600F091FB00FB05F5A0FB082308FB19
:100A40000155B21A2B4467EB0303C4E90023BDE848
:100A5000F08100BF704700BF70B54FF0FF0C4CF441
:100A6000E06C1CEA11541DBF1CEA135594EA0C0FEC
:100A700095EA0C0F00F0DEF82C4481EA030621EA27
:100A80004C5123EA4C5350EA013518BF52EA033562
:100A900041F4801143F4801338D0A0FB02CE4FF014
:100AA0000005E1FB02E506F00042E0FB03E54FF044
:100AB0000006E1FB03569CF0000F18BF4EF0010E3C
:100AC000A4F1FF04B6F5007F64F5407404D25FEA38
:100AD0004E0E6D4146EB060642EAC62141EA5551EB
:100AE0004FEAC52040EA5E504FEACE2EB4F1FD0C2D
:100AF00088BFBCF5E06F1ED8BEF1004F08BF5FEAAB
:100B0000500E50F1000041EB045170BD06F000465C
:100B100046EA010140EA020081EA0301B4EB5C0409
:100B2000C2BFD4EB0C0541EA045170BD41F4801101
:100B30004FF0000E013C00F3AB8014F1360FDEBF26
:100B4000002001F0004170BDC4F10004203C35DA02
:100B50000C341BDC04F11404C4F1200500FA05F385
:100B600020FA04F001FA05F240EA020001F0004226
:100B700021F0004110EBD37021FA04F642EB06019C
:100B80005EEA430E08BF20EAD37070BDC4F10C04C6
:100B9000C4F1200500FA04F320FA05F001FA04F28A
:100BA00040EA020001F0004110EBD37041F1000176
:100BB0005EEA430E08BF20EAD37070BDC4F1200581
:100BC00000FA05F24EEA020E20FA04F301FA05F2E9
:100BD00043EA020321FA04F001F0004121FA04F291
:100BE00020EA020000EBD3705EEA430E08BF20EA61
:100BF000D37070BD94F0000F0FD101F0004640009B
:100C000041EB010111F4801F08BF013CF7D041EA1C
:100C1000060195F0000F18BF704703F00046520020
:100C200043EB030313F4801F08BF013DF7D043EAF1
:100C30000603704794EA0C0F0CEA135518BF95EAA7
:100C40000C0F0CD050EA410618BF52EA4306D1D12E
:100C500081EA030101F000414FF0000070BD50EA4D
:100C6000410606BF1046194652EA430619D094EAD7
:100C70000C0F02D150EA013613D195EA0C0F05D1C1
:100C800052EA03361CBF104619460AD181EA030115
:100C900001F0004141F0FE4141F470014FF00000CD
:100CA00070BD41F0FE4141F4780170BD70B54FF068
:100CB000FF0C4CF4E06C1CEA11541DBF1CEA1355E8
:100CC00094EA0C0F95EA0C0F00F0A7F8A4EB0504CA
:100CD00081EA030E52EA03354FEA013100F08880C1
:100CE0004FEA03334FF0805545EA131343EA12638A
:100CF0004FEA022245EA111545EA10654FEA00263F
:100D00000EF000419D4208BF964244F1FD0404F5F7
:100D1000407402D25B084FEA3202B61A65EB030553
:100D20005B084FEA32024FF480104FF4002CB6EB10
:100D3000020E75EB030E22BFB61A754640EA0C0090
:100D40005B084FEA3202B6EB020E75EB030E22BFD0
:100D5000B61A754640EA5C005B084FEA3202B6EB11
:100D6000020E75EB030E22BFB61A754640EA9C00D0
:100D70005B084FEA3202B6EB020E75EB030E22BFA0
:100D8000B61A754640EADC0055EA060E18D04FEA5E
:100D9000051545EA16754FEA06164FEAC30343EAFE
:100DA00052734FEAC2025FEA1C1CC0D111F4801FCB
:100DB0000BD141EA00014FF000004FF0004CB6E7C4
:100DC00011F4801F04BF01430020B4F1FD0C88BF63
:100DD000BCF5E06F3FF6AFAEB5EB030C04BFB6EB6E
:100DE000020C5FEA500C50F1000041EB045170BD61
:100DF0000EF0004E4EEA113114EB5C04C2BFD4EB8E
:100E00000C0541EA045170BD41F480114FF0000E11
:100E1000013C90E645EA060E8DE60CEA135594EA8D
:100E20000C0F08BF95EA0C0F3FF43BAF94EA0C0F90
:100E30000AD150EA01347FF434AF95EA0C0F7FF405
:100E400025AF104619462CE795EA0C0F06D152EA59
:100E500003353FF4FDAE1046194622E750EA41063D
:100E600018BF52EA43067FF4C5AE50EA41047FF44E
:100E70000DAF52EA43057FF4EBAE12E74A0011D200
:100E800012F5001211D20DD56FF47873B3EB6252E4
:100E90000ED44FEAC12343F0004343EA505323FAF0
:100EA00002F070474FF00000704750EA013002D165
:100EB0004FF0FF3070474FF00000704700292DE9D8
:100EC000F043C0F2A6800026002BC0F29C8088462A
:100ED00094469E46154604460F46002B3DD18A4255
:100EE00059D9B2FA82F33BB1C3F120029F4020FAF4
:100EF00002F29D4017439C40290C220CB7FBF1FEE7
:100F0000A8B201FB1E7742EA074700FB0EF3BB4283
:100F10000AD97F190EF1FF3280F00581BB4240F201
:100F20000281AEF1020E2F44FF1AA4B2B7FBF1F317
:100F300001FB137744EA074700FB03F0B84208D9E6
:100F40007F1903F1FF3280F0F080B84240F2ED806B
:100F5000023B43EA0E43002203E08B420FD90022FA
:100F60001346341C18BF012460424FF0000565EBA6
:100F700045015840514000196941BDE8F083B3FA7A
:100F800083F2002A40F086808B4202D3844500F22F
:100F9000DB800123E5E712B90123B3FBF2F5B5FAD3
:100FA00085F000283BD1781B4FEA154E1FFA85FCCF
:100FB0000122B0FBFEF8210C0EFB180741EA07479F
:100FC0000CFB08F3BB4207D97F1908F1FF3102D2AD
:100FD000BB4200F2BD808846FF1AA4B2B7FBFEF305
:100FE0000EFB137744EA07470CFB03FCBC4507D90B
:100FF0007F1903F1FF3102D2BC4500F2A7800B46F6
:1010000043EA0843ADE752426FEA060663EB430347
:101010005DE7404261EB41014FF0FF3654E7C0F11C
:10102000200224FA02F107FA00F385404FEA154E38
:10103000D7401943B7FBFEF20B0C0EFB12771FFAD9
:1010400085FC43EA07430CFB02F79F4204FA00F4D5
:1010500007D95B1902F1FF3074D29F4272D9023A6C
:101060002B44DF1B89B2B7FBFEF80EFB187341EA75
:1010700003430CFB08F79F4208D95B1908F1FF31C5
:101080005CD29F425AD9A8F102082B44D81B48EAE7
:1010900002428EE7C2F120032CFA03F10EFA02FE9F
:1010A00020FA03F741EA0E0E08FA02F028FA03F1DB
:1010B0004FEA1E453843B1FBF5F8030C05FB181148
:1010C0001FFA8EF743EA014107FB08F38B420CFA43
:1010D00002FC09D911EB0E0108F1FF3930D28B4225
:1010E0002ED9A8F102087144C91A80B2B1FBF5F3F8
:1010F00005FB131140EA014107FB03F78F4208D9B2
:1011000011EB0E0103F1FF3016D28F4214D9023BCE
:10111000714443EA0843C91BA3FB0C89494509D321
:1011200005D000221DE79646FEE6134611E79440DF
:101130004445F6D2013BF4E70346EAE78846A5E7D3
:10114000C846D1E702468CE713460AE7023B57E759
:10115000A8F102082F443FE72DE9F041002B44D1CC
:101160008A42154604464FD9B2FA82F70E464FB16D
:10117000C7F12003B94020FA03F602FA07F50E433F
:1011800000FA07F44FEA154E230CB6FBFEF0AFB29F
:101190000EFB106143EA014307FB00F1994209D9B4
:1011A0005B1900F1FF3280F0EC80994240F2E98057
:1011B00002382B445A1AA4B2B2FBFEF30EFB1322E0
:1011C00044EA024207FB03F7974208D9521903F198
:1011D000FF3180F0D880974240F2D580023B43EA4D
:1011E000004000263146BDE8F0818B4247D8B3FA73
:1011F00083F6002E48D18B4202D3824200F2CD808A
:1012000001203146BDE8F08112B90125B5FBF2F5A8
:10121000B5FA85F8B8F1000F77D14A1B4FEA154EA1
:10122000AFB20126B2FBFEF0230C0EFB102143EA05
:10123000014107FB00F38B4207D9491900F1FF3246
:1012400002D28B4200F2BA801046C91AA4B2B1FB96
:10125000FEF30EFB131144EA014407FB03F7A74218
:1012600008D9641903F1FF3280F08F80A74240F261
:101270008C80023B43EA00403146BDE8F081002605
:1012800030463146BDE8F081C6F1200422FA04F56B
:10129000B3402B4320FA04FC01FA06F721FA04F5C7
:1012A0004FEA134E4CEA0707B5FBFEF8390C0EFB6C
:1012B00018551FFA83FC41EA05450CFB08F1A942C9
:1012C00002FA06F204D9ED1808F1FF3467D3A046FC
:1012D0006D1ABFB2B5FBFEF40EFB145547EA05418B
:1012E0000CFB04FC8C4504D9C91804F1FF355CD310
:1012F0002C4644EA0844CCEB0101A4FB02239942AA
:1013000048D344D0204600266CE7C8F1200401FAF7
:1013100008F305FA08F520FA04F7E1404FEA154E04
:101320001F43B1FBFEF63A0C0EFB16111FFA85FCAB
:1013300042EA01430CFB06F29A4200FA08F407D98C
:101340005B1906F1FF3137D29A4235D9023E2B4460
:101350009B1ABFB2B3FBFEF00EFB103347EA034308
:101360000CFB00F1994207D95B1900F1FF3221D241
:1013700099421FD902382B445A1A40EA064667465A
:1013800050E7104616E70B4629E7134672E7B040D0
:101390009042B7D2601E002624E7304622E7A942D9
:1013A00095D9A8F102081D4492E78C45A0D9023CCA
:1013B00019449EE71046DFE70E46C9E70238294484
:1013C00043E700BF4FF0FF3C06E000BF4FF0010CC9
:1013D00002E000BF4FF0010C4DF804CD4FEA410C84
:1013E0007FEA6C5C4FEA430C18BF7FEA6C5C1BD051
:1013F00001B050EA410C0CBF52EA430C91EA030FD2
:1014000002BF90EA020F0020704710F1000F91EA2E
:10141000030F58BF994208BF90422CBFD8176FEAFC
:10142000E37040F0010070474FEA410C7FEA6C5CCA
:1014300002D150EA013C07D14FEA430C7FEA6C5CD1
:10144000D6D152EA033CD3D05DF8040B704700BFFD
:101450008446104662468C461946634600E000BF4B
:1014600001B5FFF7B7FF002848BF10F1000F01BD1D
:101470004DF808EDFFF7F4FF0CBF012000205DF8E8
:1014800008FB00BF4DF808EDFFF7EAFF34BF01206D
:1014900000205DF808FB00BF4DF808EDFFF7E0FF06
:1014A00094BF012000205DF808FB00BF4DF808ED57
:1014B000FFF7CEFF94BF012000205DF808FB00BFBE
:1014C0004DF808EDFFF7C4FF34BF012000205DF8A0
:1014D00008FB00BF11481249026800608A4218D018
:1014E000002103E00F4B5B58435004310E480F4B73
:1014F00042189A42F6D30E4A02E0002342F8043B17
:101500000C4B9A42F9D3FCF72FFA00F019F8704708
:10151000FEE70948D0F800D040680047FC9F002053
:10152000EFBEADDE608101080000002078010020E0
:1015300078010020EC2A002000D8FF1FFEE7000001
:101540002DE9804895B0EEF71FFEB34CB34E2378DB
:10155000316843B1B24B1B68CB1A002BA1BFB14A13
:10156000002323701370DFF810A3DAF8000042F2B2
:10157000010303400BB9AA4A1371030740F1938199
:10158000A94B1B681B7A062B00F27C81DFE813F065
:10159000070007003400D40010013C013C01A34BBC
:1015A0001A78002A00F06E8100221A70A04B93F87E
:1015B00000E0A04B1B6893F800C09F4B93F800809D
:1015C00002229E4FBB5C43FA0EF303F00F03634508
:1015D00002F101090CD20B2B9FBFBD5C17F80970FB
:1015E00005EA080507EB05259CBF954F47F82350F2
:1015F0000232102AE5D10CE1924B1A78002A00F051
:10160000418100221A70904B904A93F802C093F8DF
:1016100003E05D780CF0070745EA07250EF03F0769
:101620007F0147EADC0715601D7957605F7993F801
:1016300006C0AD0045EA9E1507F0010E45EA8E256D
:10164000956093F807E00CF00F05ED0145EA5705AA
:101650000EF07F07D5603F011D7A47EA1C1793F80B
:1016600009C017616D000CF0030745EADE1545EA75
:10167000472593F80AE05561DD7A0EF01F07BF0198
:10168000ED0047EA9C0745EA5E1593F80DC093F814
:101690000EE0D5611D7B97610CF0070745EA072531
:1016A0000EF03F077F0147EADC071562DD7B5762DA
:1016B0001F7C93F811C0AD0045EA9E1507F0010E9E
:1016C00045EA8E25956293F812E00CF00F05ED01C6
:1016D00045EA57050EF07F073F0147EA1C17D56220
:1016E000DD7C176393F814C06D0045EADE150CF03D
:1016F000030793F815E045EA472555630EF01F07E9
:101700009D7DDB7DBF0147EA9C07ED0045EA5E1544
:101710009763DF07D5634CBF40F21475AD251564A0
:101720009D074CBF40F21475AD2513F0080F5564AA
:1017300014BF03230123A6E0454A1378002B00F0D1
:10174000A18000231370434ADFF830E11778424D3F
:101750000EEB470CB5F800809CF803909CF8045001
:1017600045EA0925A84540F08D809EF80150012DDD
:1017700004D0812D40F08780032300E02B46102FFA
:1017800084BF10251570354D92F800E00022D7B2C5
:10179000774505F1020576D215F802CC15F8017CE3
:1017A00047EA0C27DFF8D8C02CF812700132EEE7B8
:1017B0002B4B1A78002A65D000221A70294B1A7810
:1017C000A82A1F465ED1DA7C002A5BD107EB4205CE
:1017D0009FED257A95F803E02B7903EB0E2307EEB6
:1017E000903AF8EEE77A214BC7EE877A9FED207AA0
:1017F00077EEC77AFCEEE77A17EE905A43F822505C
:101800000132082AE2D104E01A4B1A78D2B300223E
:101810001A70012337E000BF6C0D0020C42A00209D
:10182000780100206D0D0020802A00208D110020FD
:10183000622500205C250020632500207D1100200A
:10184000F81000207E2A0020652A0020AC29002004
:10185000352A0020382A0020362A00203C2A002081
:10186000AE11002099110020CDCCCC4028110020D1
:101870000080BB43F4100020842A0020392A002075
:10188000481100200023DA070DD5A14A0125157162
:10189000A04DC3F340032B7083F00103237001F5C7
:1018A000C333A0331360470411D59B4A13780BB19F
:1018B00000251570964A13714BB101232370954B87
:1018C00000241C7001F5433303F5A0731360C507B2
:1018D0000FD58F4B5C799A79A2420AD08F4A9C71BE
:1018E000012515708E4A0025157001F5C332A0320E
:1018F0001A60840409D500238A4A32F81320002A8A
:1019000041F0628601330C2BF6D1DFF804B29BF86C
:10191000043023B9844B1B68CB1A002B10DBDBF897
:101920000830C91A11F1500F02D4794B1B7B3BB11F
:10193000F0F73CFA01238BF80D308BF80C3010E0F7
:10194000DBF810305A1CCBF810201BB9800301D5EE
:10195000F6F775FDDBF81030002BC2BF6C4B002290
:101960001A61FDF72DF8714B30600DACDB68204635
:1019700098479DF834303BB96D4BDBF808201B6865
:101980009B1A642B00F133876A4F33683A686A4DBB
:101990001344CBF8083000238BF80C30674B2868D1
:1019A0001988643001B10221FAF726F9FDF708F829
:1019B000D7ED007ADBF814303060F8EE677A604ECD
:1019C0009FED607ADFF89481CBF81400C31A33805E
:1019D00067EE877A5C4BC8ED007A224603F1080E69
:1019E00018685968174603C7083373453A46F7D154
:1019F00018689B883860BB80BDF840C053490022FE
:101A000000230F46184637F802EF34F8039027F802
:101A100002EC02330C2B1EFB0900F4D14C4F37F8BB
:101A200012308B8113FB0C004FF4807390FBF3F0AA
:101A300027F812000132032A01F10E01E0D1F1F77B
:101A400041FA3388324FD8ED000ABBF8424000EE2D
:101A5000103A07F14400B8EE400A0121F7F7E8F91F
:101A6000BCEEC00A9BF80D308DED040ABDF81000E5
:101A7000B4FBF0F0441CA4B2ABF84C4033B3B7F85D
:101A80004E30049300232249324ABDF8109032F8B8
:101A900013C001F1580E01F150083EF8137038F8E8
:101AA00013202EF813C0C7EB0C0712FB09F20FFA34
:101AB00084F992FBF9F23A4428F813200133042BFD
:101AC000E1D100234B73A1F84E0004E0B7F84E308B
:101AD000013BA7F84E30BBF84E000D4A03B2002B75
:101AE0004FF000033CDDB2F94C401B4931F81320A4
:101AF000083112FB00F231F8131092FBF4F28A1A4B
:101B0000144921F813200133042BEED12AE000BF41
:101B10007801002003000020C60E00206D0D00207B
:101B200004000020182A0020440D0020F419002091
:101B3000C42A0020480F0020200F0020E00E0020C3
:101B4000D00E0020BD3786359C440108900100204E
:101B50000A0F002080190020C801002094190020DD
:101B6000A2F84E30BA4BBB4C1B68BB4F13F4801F1E
:101B700000F09480B4F8008008F400681FFA88F838
:101B8000B8F1000F77D1B54B1B78590773D54FF4D7
:101B90000060F7F78BFC3B68CBF860301978B04AEF
:101BA000022906BF012182F8641082F86480B3F82C
:101BB0005C209BF864804FF47A735343328893FB24
:101BC000F2F3A84A5B4292F800C0DBF860209BB2B7
:101BD000ABF8663002F12006002092F857E092F848
:101BE0005410BEF1000F01D0714504D8BCF1030FB1
:101BF00005D8022803D14FF0000E82F857E0DFF835
